:1000000002CFE1FFFFFFFFFFFFFFFF0267CEFFFF11
:10002000FFFFFF0204AFFFFFFFFFFFFFFFFFFFFF28
:10004000FFFFFFFFFFFFFFFFFFFFFF02CEF0FFFFFD
:10005000FFFFFF02D0DFFFFFFFFFFF02D19DFFFF89
:10007000FF2365FFFFFFFFFFFFFFFFFFFFFFFFFF06
:1000800090F009E4F090F008E4F002CFE1FFFFFF08
:10010000E4F5B875A890F54AF55EF55FF55CF55D28
:1001100090F0087406F0E4FFFE055DE55DAC5C70F0
:1001200002055C14F5828C83E493FD055FE55FAA0C
:100130005E7002055E14F5828A83EDF00FBF000148
:100140000EE4B507D4EEB420D090F0097402F0A309
:10015000E4F090F0097403F0E4F55EF55FF55CF50A
:100160005D1205478F59E559B42E0B7E047F81122D
:1001700003CFC2AF80FEE559B42103120189C2AF9B
:10018000D2AED2BED2AF80D922E4F5541203858F0D
:10019000681203858F641203858F65E4F56112038D
:1001A0008574412561F8A6070561E561C39408409F
:1001B000EDE4F561120385744B2561F8A60705612E
:1001C000E561C3940840ED12038EEF655460067F2D
:1001D0006212051822AF687401A807088002C333B1
:1001E000D8FCF561554A706CC2AF90F00AE568F032
:1001F000C2431203FD50067F4512051822D2431256
:1002000003FD50067F4512051822E561424AE4F5D8
:1002100066F567C2AFD2AED2BED2AFF561E4F56289
:100220000567E567AE667002056614F5828E83E0A9
:10023000B4FFBD0567E567AE667002056614F5821A
:100240008E83E0B4FFAA0562E562B480D30561E560
:1002500061B480C9C2AFD2AED2BEE564FE7C00E418
:100260002565FFEC3EF5668F67E4F56190055574F2
:10027000AAF09002AA7455F090055574A0F074414C
:100280002561F8E6856782856683F08567828566E5
:1002900083E05480FF74412561F8E65480B507EB94
:1002A0000567E567700205660561E561B408BDE4B0
:1002B000F56190055574AAF09002AA7455F0900566
:1002C0005574A0F0744B2561F8E6856782856683D6
:1002D000F0856782856683E05480FF744B2561F862
:1002E000E65480B507EB0567E567700205660561B2
:1002F000E561B408BD74F02567F56774FF3566F5F0
:1003000066E4F5610567E567AE667002056614F59B
:10031000828E83E0FF74412561F8E6FEEF6E601681
:10032000AF687401A807088002C333D8FCF4524AAE
:100330007F62120518220561E561C3940840C5E497
:10034000F5610567E567AE667002056614F5828E95
:1003500083E0FF744B2561F8E6FEEF6E6016AF6830
:100360007401A807088002C333D8FCF4524A7F62A4
:10037000120518220561E561C3940840C5D2AF7F1C
:100380003F1205182212038EEF2554F55422E5087A
:10039000700F3025F9C225C2AFD2AED2BED2AF8027
:1003A000ED7400250CF582E434FDF583E0FFBF0D0C
:1003B000057800E214F2E50C04547FF50C150822D0
:1003C000EF1FAC0670011E4C6004000080F2227822
:1003D00098EEF208EFF27898E2FE08E2F5828E835A
:1003E000E49360181808E2FF2401F218E23400F2E6
:1003F0008F828E83E493FF12051880DA22900555D0
:1004000074AAF09002AA7455F09005557480F074A7
:10041000AAF09002AA7455F030430890400074305E
:10042000F080069000007430F0D2AF900000E054ED
:1004300040FDE4F569D2AED2BE900000E05440FF2A
:100440006D6012AD077FD07E071203C00569E569B4
:10045000C394C840E0E569C394C840097E047F8B1B
:100460001203CFD3227E047F9D1203CFAF69120502
:100470007A7E047FAB1203CF7F327E001203C0C3AB
:10048000225265626F6F74210D0A002044656C650D
:1004900074652054696D656F75740D0A002044659C
:1004A0006C65746554696D653A2000200D0A00C0C2
:1004B000E0C083C082C0D0C000C007309829C29875
:1004C000E508D3947F5020AF997400250AF582E4A3
:1004D00034FDF583EFF0BF0D057800E204F2E50A84
:1004E00004547FF50A0508309921C299E50960197D
:1004F0007480250DF582E434FDF583E0F599E50D72
:1005000004547FF50D15098002D200D007D000D029
:10051000D0D082D083D0E032C3747F9509C3940ACF
:1005200040F6E509D3947F501D7480250BF582E4D5
:1005300034FDF583EFF0E50B04547FF50B0509302E
:100540000004C200D29922E50860277400250CF54A
:1005500082E434FDF583E0FFFEBF0D057800E21470
:10056000F2E50C04547FF50C1508EE640A60D8AF70
:1005700006227F00227800E2FF22AE07EEC4540F6D
:100580009005BD93FF120518EE540F9005BD93FF23
:1005900012051822120547EF541F24CEF582E434C9
:1005A00005F583E493C454F0FD120547EF541F246E
:1005B000CEF582E43405F583E4932DFF2230313209
:1005C0003334353637383941424344454600000A12
:1005D0000B0C0D0E0F0000000000000000000001D9
:1005E0000203040506070809E478A0F690F00CF071
:1005F0007557F0A374F0F090F000E0783AF2C2AFD3
:10060000E4F5A8F5B8758680D2AED2BED224C2B5C4
:100610000090F00A04F090F008E4F012847C7E0070
:100620007FE07D007B027AEC790012D40E7E007FA1
:10063000E07D007B027AED790012D40E759204758C
:1006400083F0758201E4F592C28C438901758CF5C3
:10065000758A95D28C75C84575C10A75A90C75B98E
:1006600004C2C27F0B1291CB129A3C43B110759019
:100670000353B1EF12CE7212850E75B80675A892AB
:1006800090F001E030E00C783AE230E70312823378
:10069000127E841283B5126E0012B6AD7B057A9D70
:1006A0007997E4FD1285AE7B057A9D79A67D1012BF
:1006B00085AE7B057AA079867D191285AE751925E0
:1006C000751801129820C224754B35754C01E4F55C
:1006D0004D20210312519CE47801F2781BE660075B
:1006E000D24412527B80F47FA87E611203C0C2AF55
:1006F000D2AED2BED2AF7801E204F2E2C3940A4095
:10070000DA1284FAE47876F208F2780174FFF2786B
:1007100003740AF2087432F27882740CF27802746C
:1007200019F2C2AFD2AED2BED2AF90ECE07403F0F9
:100730007834E2A3F0A374FFF0E4A3F0A374FFF015
:10074000E490ECE9F090ECE8F0203D06129D2A12CE
:100750003406781BE67003302A05D24412527B120D
:100760000575EF605E20215B1208D27887E6648011
:1007700070030208C7301A4B1284FA7B057A9D7900
:10078000B2E4FD1285AE7B057A9D79BB7D101285A2
:10079000AE7E9D7FC41203CF1299F9E55744A0F5B0
:1007A0005790F00DF0D214D2451297DCC2AFD2AE02
:1007B000D2BED2AF7FA87E611203C07F06129A3CE0
:1007C000120100303505127799C2357884E6FF7042
:1007D000030207497885E630E411EFD39401400B1A
:1007E000785CE2FEEFD39E4002EFF27884167876D2
:1007F00008E22401FFF218E23400FEF2BE031EBF3D
:10080000201BE4F208F2D2451297DC7882E2600DF8
:1008100014F270099091C0F012CC57D2367877E27A
:10082000B4900818E2B4010312971A7801E2600A42
:1008300014F2700674FFF21279A7202164789FE603
:10084000600E16E6700A780D74FFF27F0D1205181F
:100850007802E2600A14F270067419F2127CA5782C
:1008600004E2603414F270307404F27885E630E10A
:100870000578047428F230420712B19BC2428018F6
:10088000D242909150E0FEA3E0FF122BB090917302
:10089000E0FEA3E0FF122BB01231FF302B03124118
:1008A0001D7803E2600B14F270071294D57803EF01
:1008B000F2202503020749C22575A0FCC2AFD2AEC3
:1008C000D2BED2AF0207497E9D7FD01203CF129BCA
:1008D000AD22C24330330412C6BF221205478F59DE
:1008E000E4F552F553F554E5596463600BE559643A
:1008F000766005E559B46905D2435359DFE559647B
:1009000043604BE55964566045E559644C603FE5EA
:100910005964576039E559644F6033755A091205B7
:1009200047744B255AF8EFF6640D6007155AE55ADF
:10093000B4FFEBE55AB4FF161205477867EFF2648F
:100940000D600B120547EF640D6003022905E559A0
:1009500024BFB41A0040030228FB900961F828283C
:10096000730211640215E90209AF020B5E0226D17F
:1009700002163B020A0402291F020D0402291F026B
:100980001B910225EE021D12021ECB020A00021F5D
:100990000C0223F80223F8021FDC02291F02202F79
:1009A000022470020A1102110702291F020B197892
:1009B00085E620E30302291F1205948F4B1205944C
:1009C0008F4CE54C540FF559E4F55BE55BC3955945
:1009D000500E120594744D255BF8A607055B80EB5D
:1009E000304319534C0F78E07CEC7D027B047A0095
:1009F000794B7E007F0A12D316D22A2212519C22F2
:100A000012C9F8227885E620E30302291F12C7C91C
:100A100022120547EF24BD601E24FA601624E07000
:100A200003020AE524FA604D24206003020B191228
:100A3000C5472212C61C22120547EF644C60030210
:100A4000291F120547EF6445600302291F1205475D
:100A5000EF6441600302291F120547EF64526003EF
:100A600002291FD22212B6ADC2227F2A1205187F98
:100A70000D12051822D207E4F55AE55A541F7005E5
:100A8000780BF208F275F02CE55AA4240DF582E5F6
:100A9000F0344EAF82F55E8F5F7F571205187F6985
:100AA000120518AF5A12057AE4F559855F82855E02
:100AB00083E0FF12057AE55F2401FFE4355EF55E11
:100AC0008F5F0559E559C3942840E0E509D3943F69
:100AD00050F97F0D1205187F0A120518055AE55ABC
:100AE0007098C20722D207E4780BF208F2F55A1286
:100AF00005948F54E554655A60F57E9D7FDB1203A3
:100B0000CF754B35754C01754D0D12519C12519C92
:100B100012519CD2AED2BE80FEE4F559301E034382
:100B20005901201403435902300903435904302268
:100B3000097885E630E303435908435980789CE6F9
:100B4000FF30E003435920EF30E1034359107F5A4F
:100B5000120518AF5912057A7F0D12051822E554B7
:100B6000646F7023E553B4771EE552B46E19E551F6
:100B7000B46C14E550B46F0FE54FB4610AE54EB4A0
:100B80006405D21A022905E5546465702BE55364A7
:100B9000627025E552B45F20E551B4451BE550B4C1
:100BA0006D16E54FB47011E54EB4660CE54DB421F9
:100BB0000778877680022905E55464656003020C96
:100BC0006BE55364626003020C6B7F0D1205187FA6
:100BD0000A1205187F07122B387885A6077887A692
:100BE000507F04122B387887A6077885E6FF120518
:100BF0007A7887E6FF12057A785CE2D39401402088
:100C00007F201205187F421205187F471205187FB2
:100C100054120518785CE2FF12057A785C7401F2D0
:100C20007F0D1205187F0A1205187885E620E70364
:100C300002291FC2AFE4F5C8F5C190F00B740CF0A7
:100C4000C290C291D2AED2BE7F0A7E001203C0D241
:100C5000907F057E001203C0D29100000000C29078
:100C60007F087E001203C0C29180D9E5546465708C
:100C700040E553645A703A7F0D1205187F0A120539
:100C8000187F07122B387881EFF27F05122B387806
:100C90004DEFF27881E2FF12057A7F201205187875
:100CA0004DE2FF12057A7F0D1205187F0A12051812
:100CB000227885E6700302291F7F0D1205187F0A2E
:100CC0001205187885E6FF12057A7887E6FF120587
:100CD0007A785CE2D3940140207F201205187F428D
:100CE0001205187F471205187F54120518785CE228
:100CF000FF12057A785C7401F27F0D1205187F0AE5
:100D0000120518227885E620E30302291FE4F5592D
:100D1000F55DD207E554640D700302107F7F091260
:100D20002B388F5AE55A541F7005780BF208F2E5FC
:100D300009D3942050F975F02CE55AA42418F582B3
:100D4000E5F0344EF583E0FF12057A75F02CE55A94
:100D5000A4241AF582E5F0344EF583E054C0F55929
:100D600030E6077F6E1205188011E55930E7077FDE
:100D70006D12051880057F7A12051875F02CE55A5A
:100D8000A4240DF582E5F0344EF583E04430FF12E3
:100D900005187F2012051875F02CE55AA4241EF5BD
:100DA00082E5F0344EF583E0FF12057A75F02CE50C
:100DB0005AA4241DF582E5F0344EF583E0FF1205B8
:100DC0007A7F20120518204303020F2375F02CE5CB
:100DD0005AA42409F582E5F0344EF583E0FEA3E041
:100DE000AA06F97B02126D0F75F02CE55AA4240BAC
:100DF000F582E5F0344EF583E0FEA3E0AA06F97B28
:100E000002126D0F7E9D7FE31203CF75F02CE55A21
:100E1000A42419F582E5F0344EF583E0FF12057A3B
:100E20007E9D7FE71203CF75F02CE55AA4241AF5B6
:100E300082E5F0344EF583E0FF12057A7E9D7FEB6C
:100E40001203CF75F02CE55AA4241BF582E5F0348B
:100E50004EF583E0FF12057A7E9D7FEF1203CF757A
:100E6000F02CE55AA4241CF582E5F0344EF583E01D
:100E7000FF12057A7E9D7FF31203CF75F02CE55AA1
:100E8000A4241FF582E5F0344EF583E0FF12057AC5
:100E90007E9D7FEF1203CF75F02CE55AA42420F538
:100EA00082E5F0344EF583E0FF12057A7E9D7FF7F0
:100EB0001203CF75F02CE55AA42421F582E5F03415
:100EC0004EF583E0FF12057A7E9D7FFB1203CF75FE
:100ED000F02CE55AA42422F582E5F0344EF583E0A7
:100EE000FF12057A7E9D7FFF1203CF75F02CE55A25
:100EF000A42423F582E5F0344EF583E0FF12057A51
:100F00007E9D7FFF1203CF75F02CE55AA42424F5B3
:100F100082E5F0344EF583E0FF12057A7E9E7F0372
:100F20001203CF7F07122B38055AEF655A60030270
:100F30000D24E550640D700302107CE4F559755AD8
:100F400001E559C39405400302107CE559B404033C
:100F5000E4F55AE509D3942050F97E9E7F061203EA
:100F6000CF75F007E55AA42449F582E5F03491F5F0
:100F700083E0FEA3E0AA06F97B02126D0F75F0076D
:100F8000E55AA4244BF582E5F03491F583E0FEA305
:100F9000E0AA06F97B02126D0F75F007E55AA4244A
:100FA0004EF582E5F03491F583E0FEA3E0AA06F960
:100FB0007B02126D0F75F007E55AA4244DF582E50A
:100FC000F03491F583E064AA601A7F211205187548
:100FD000F007E55AA4244DF582E5F03491F583E05D
:100FE000FF12057A7E9E7F0A1203CF75F007E55A3D
:100FF000A4246CF582E5F03491F583E0FEA3E0AA29
:1010000006F97B02126D0F75F007E55AA4246EF500
:1010100082E5F03491F583E0FEA3E0AA06F97B02B5
:10102000126D0F75F007E55AA42471F582E5F034CE
:1010300091F583E0FEA3E0AA06F97B02126D0F751D
:10104000F007E55AA42470F582E5F03491F583E0C9
:1010500064AA601A7F2112051875F007E55AA424C6
:1010600070F582E5F03491F583E0FF12057A7E9EFB
:101070007F031203CF0559055A020F41C20722E52B
:1010800009D3943F50F9E559540F70147F0D1205A0
:10109000187F0A120518AF5912057A7F3A120518FF
:1010A0007F20120518AF5D055DA807E6FF12057ADF
:1010B0000559E55970C97F0D1205187F0A120518E8
:1010C000E4F559F55DE509D3943F50F9E559540F1E
:1010D00070147F0D1205187F0A120518AF591205FA
:1010E0007A7F3A1205187F20120518A85DE2FF12D8
:1010F000057A055D0559E55970CB7F0D1205187FFE
:101100000A120518C207227885E620E30302291F88
:10111000E554B40D08E47884F208F2801EE554B476
:10112000620B78847400F2087418F2800EE554B4EF
:1011300061097884744EF2087409F27884E2FE083A
:10114000E2FF1205187884E2FF120518788408E29D
:10115000FF2401F218E2FE3400F28F828E83E0FF5A
:1011600012051822E552640D60030212B57F411288
:1011700005187F09122B388F5912057A75F02CE566
:1011800059A42409F582E5F0344EAF82F5608F61F1
:10119000F583E5822411F582E43583F583E054C0BC
:1011A00060087E9E7F0E1203CF22E5612410F58237
:1011B000E43560F583E030E712E561241AF582E456
:1011C0003560F583E0FF12057A8049E561240BF56F
:1011D00082E43560F583E0540FF559E5612413F599
:1011E00082E43560F583E0FF30E003435910E561A8
:1011F0002410F582E43560F583E0FE30E0034359C6
:1012000020EF30E203435940EE30E303435980AF0F
:101210005912057AE5612415F582E43560F583E01D
:101220005407FF25E025E0FFE5612416F582E4354B
:1012300060F583E05430FEC4540F4FF559E5612446
:1012400013F582E43560F583E0FF30E30343592072
:10125000EF30E403435940EF30E503435980AF5981
:1012600012057AE5612415F582E43560F583E0FF27
:10127000C454F0FE25E025E0FEEF54304EF559FF52
:1012800012057AE4F559E561240EF582E43560F53E
:1012900083E030E503435901E5612410F582E4352C
:1012A00060F583E030E703435902AF5912057A7FB6
:1012B0000D12051822E553644D600BE553644E6032
:1012C00005E553B45A097F07122B388F5980077FE1
:1012D00008122B388F59E553644D6009E553644E6D
:1012E0006003021384E554645760030213847F4152
:1012F000120518E4F54BE553B44D2AE559C3944063
:10130000400302291F75F005E559A42409F582E57B
:10131000F03490AF82F5648F657F571205187F4DCA
:10132000120518804475F00BE559A42409F582E5EF
:10133000F0347AAF82F5648F657F05122B38EF3079
:10134000E70EE42565F565740B3564F564754B802F
:10135000856582856483A3A3E030E003434B017F6E
:10136000571205187F4E120518AF5912057AAF4B68
:1013700012057A856582856483E0FF12057A7F0D08
:101380001205182275F02CE559A42409F582E5F020
:10139000344EAF82F5608F61F583E5822411F582CA
:1013A000E43583F583E0F55154C0F5398F82E58249
:1013B0002410F582E43560F583E0F54B30E7317FAA
:1013C000411205187F57120518E539600302291FDD
:1013D0007F5A120518AF5912057AE561241AF58271
:1013E000E43560F583E0FF12057A7F0D12051822BF
:1013F000E539B44015E559D3947F400EAF61AE6036
:10140000AD59122B52400302291F7F411205187F4C
:1014100046120518E561240BF582E43560F583E09A
:10142000F552E53970087F5A12051853520FE53905
:10143000644070337F4E120518E551540CFFBF080D
:1014400010E5521313543FF552D3941C40037552C8
:101450001CE551540CFFBF040EE552131313541F27
:10146000F552B40F021552E539B480187F4D1205BC
:1014700018E552131313541FF55253520FE552B48B
:101480000F021552AF5912057AAF5212057AE4F5E0
:1014900059E54B30E103435901E54B30E203435931
:1014A00002E551540CFFBF0403435904BF08034332
:1014B0005908BF0C0343590CE5612413F582E43548
:1014C00060F583E0FF30E003435910E54B30E00363
:1014D000435920E5397007EF30E203435940E539BD
:1014E000B44012E5612411F582E43560F583E03003
:1014F000E103435940E54B30E303435980AF5912B0
:10150000057AE5612413F582E43560F583E0FFC3D5
:1015100013F559E561241AF582E43560F583E0306E
:10152000E003435980AF5912057AE5612417F5822B
:10153000E43560F583E0FF12057AE539706FE56107
:101540002415F582E43560F583E05407FF25E02596
:10155000E0FFE5612416F582E43560F583E0543060
:10156000FEC4540F4FF559E5612413F582E435604C
:10157000F583E0FF30E303435920EF30E4034359A0
:1015800040EF30E503435980AF5912057AE56124F5
:1015900015F582E43560F583E0FFC454F0FE25E0E4
:1015A00025E0FEEF54304EF559FF12057AE4F55967
:1015B000E561240EF582E43560F583E030E5034310
:1015C0005901AF5912057AE539B44017E561241A7B
:1015D000F582E43560F583E0FFC313F559540FFF3E
:1015E00012057A7F0D120518221229208F5975F0E5
:1015F0002CEFA42409F582E5F0344EAF82F5608F1C
:1016000061FEAD59122979500302291FE539B44012
:1016100015E559D3947F400EAF61AE60AD59122BE2
:1016200052400302291F7F07122B38E5612417F56A
:1016300082E43560F583EFF0021C97C24412292042
:101640008F5975F02CEFA42409F582E5F0344EAFE4
:1016500082F5608F61FEAD59122979500302291F6E
:10166000E539B44015E559D3947F400EAF61AE60C3
:10167000AD59122B52400302291F7F07122B388FBE
:10168000547F05122B388F59E55930E411E5612458
:1016900013F582E43560F583E04401F0800FE561E5
:1016A0002413F582E43560F583E054FEF0E559300B
:1016B000E511E5612410F582E43560F583E044012D
:1016C000F0800FE5612410F582E43560F583E05485
:1016D000FEF0E5396440704FE5612410F582E43591
:1016E00060F583E0FF5408FEE5595480FD6E6014F8
:1016F000D244E5612411F582E43560F583E030E100
:1017000003435B10ED6011E5612410F582E4356060
:10171000F583EF4408F0800FE5612410F582E4358D
:1017200060F583EF54F7F0E5612410F582E435604D
:10173000F583E0547FF04440F0E55930E011E56175
:101740002410F582E43560F583E04402F0800FE573
:10175000612410F582E43560F583E054FDF0E5592D
:1017600030E111E5612410F582E43560F583E04451
:1017700004F0800FE5612410F582E43560F583E024
:1017800054FBF0E539644060030218247F03122BF8
:10179000388F5AE561241AF582E43560F583E0FF5D
:1017A00030E733E5612413F582E43560F583E0FE2C
:1017B000C313F55CEF30E003435C80E55A655C6081
:1017C00015E561240FF582E43560F583E0FFAD5C3B
:1017D000129AF5435B02E5612413F582E43560F566
:1017E00083E05401F0E5612413F582E43560F5836C
:1017F000E0FFE55A25E0FEEF4EF07F01122B38EFB7
:10180000540FFF25E0F54EE55A30E703434E01E55E
:1018100061241AF582E43560F583E054E0F0454E2A
:10182000F0435B07E5612410F582E43560F583E061
:1018300030E014E561240AF582E43560F583E020A8
:10184000E0057411F0D243E5612410F582E43560BF
:10185000F583E020E014E561240AF582E43560F5C3
:1018600083E030E0057412F0D243E5396440706DD6
:1018700053590CE5612411F582E43560F583E0F5F8
:1018800051E559600A5351F34251E551F08006E5A4
:1018900051540CF559E559B40409E554C454F0F514
:1018A00054801BE559B4080BE55433333354F8F531
:1018B00054800BE559B40C06E55425E0F554E56178
:1018C0002420F582E43560F583E0455BF0E5612492
:1018D00008F582E43560F5837402F08049E53964E7
:1018E00080703C53590CE5612411F582E43560F5B4
:1018F00083E0F551E559600A5351F34251E551F047
:101900008006E551540CF559E554C454F0F554E5FE
:10191000612408F582E43560F583740AF08007E5F8
:1019200054C454F0F554E5612412F582E43560F5B1
:1019300083E554F0E5612416F582E43560F583E033
:10194000540FC454F0FFE561240CF582E43560F5D2
:1019500083E0540F2FF0E561240EF582E43560F545
:1019600083E0FF20E61D4440F0754B34754C22E5C2
:1019700061240FF582E43560F583E0F54DE4F54E22
:1019800012519CE5612404F582E43560F583E0643E
:10199000016009AF61AE607D01124E0E754B42755C
:1019A0004C06E561240FF582E43560F583E0F54DE2
:1019B000E5612410F582E43560F583E0F54EE561DC
:1019C0002411F582E43560F583E0F54FE561240BE1
:1019D000F582E43560F583E0F550E5612413F58286
:1019E000E43560F583E0F551E561241AF582E435CC
:1019F00060F583E0F55212519CE5612411F582E413
:101A00003560F583E020E003021B81E5612410F5D9
:101A100082E43560F583E0F55A85605E85615FE4B8
:101A2000F559E55F2406F582E4355EF583E0FEA313
:101A3000E08E5EF55F4E700302291FE55F65617001
:101A400004E55E6560700302291FE55F2411F582DD
:101A5000E4355EF583E020E00302291FE55F2410F2
:101A6000F582E4355EF583E054D1FFF0E55A542E5B
:101A70004FF0E55F2412F582E4355EF583E554F01E
:101A8000E561240CF582E43560F583E0FFE55F2431
:101A90000CF582E4355EF583EFF0E5612417F582FD
:101AA000E43560F583E0FFE55F2417F582E4355EF9
:101AB000F583EFF0E55F2420F582E4355EF583E001
:101AC0004401F030442DE55F2420F582E4355EF5D5
:101AD00083C083C082E0FFE55F2411F582E4355EB8
:101AE000F583E030E1047E1080027E04EF4ED08268
:101AF000D083F0304326E55F2410F582E4355EF5AF
:101B000083E06401F0E55F240AF582E4355EF58345
:101B1000E030E0057412F080037411F0E55F2404F6
:101B2000F582E4355EF583E064016018AF5FAE5E78
:101B30007D01124E0EE55F240EF582E4355EF583DD
:101B4000E04440F0E55F2411F582E4355EF583E082
:101B500054C0FFBF8010E55F2408F582E4355EF5D0
:101B600083740AF0800EE55F2408F582E4355EF5A3
:101B7000837402F00559E559C394085003021A22F0
:101B800022E5612406F582E43560F583E4F0A3F0F4
:101B9000227F09122B388F5975F02CEFA42409F5F8
:101BA00082E5F0344EAF82F5608F61F583E58224E3
:101BB00011F582E43583F583E054C0600302291FE8
:101BC0007F07122B388F59E5612416F582E43560C2
:101BD000F583E0540FFFE5595403C454F04FF0E58A
:101BE000612415F582E43560F583E054F0FFE55992
:101BF000541CFE1313543F4FFFE5612415F582E496
:101C00003560F583EFF0E55930E511E5612413F512
:101C100082E43560F583E04408F0800FE561241329
:101C2000F582E43560F583E054F7F0E55930E611CC
:101C3000E5612413F582E43560F583E04410F0801B
:101C40000FE5612413F582E43560F583E054EFF08D
:101C5000E55930E711E5612413F582E43560F58339
:101C6000E04420F0800FE5612413F582E43560F54F
:101C700083E054DFF07F05122B388F59E559C413E8
:101C8000135403FFE55954304FFFE5612415F582E5
:101C9000E43560F583EFF0E561240EF582E435600C
:101CA000F583E0FF20E61D4440F0754B34754C226F
:101CB000E561240FF582E43560F583E0F54DE4F548
:101CC0004E12519CE5612404F582E43560F583E011
:101CD00064016009AF61AE607D01124E0EE56124C2
:101CE00008F582E43560F5837408F0754B43F54CD4
:101CF000E561240FF582E43560F583E0F54D7F4E14
:101D0000E5612413FDE43560FC7B0712CFA6125178
:101D10009C22E550B40D1B7F09122B388F5975F0AA
:101D20002CEFA42409F582E5F0344EAF82F5608FE4
:101D300061221229208F59E5397003021EAB30064B
:101D4000157F3F1205187F3F1205187F3F120518B7
:101D50007F0D120518227F07122B388F5AE55A542F
:101D60000790A30593F54BE55A30E008E54BC31304
:101D7000F54C8006E54B25E0F54CE5396480705E56
:101D8000535A0F789CE620E10302291FE559D394AA
:101D900050400302291F7895A65AE559C394405034
:101DA0002E78427404F2786AE559F275F005A4249D
:101DB00009F582E5F03490AF82F5648F65E55A301D
:101DC000E30D856483E0454BFFF0E54CF45FF0D212
:101DD000237899A65978837404F2E47892F6E53969
:101DE0006440600302291F789CE620E00302291F5B
:101DF000C22378837404F2E47892F6D206E55A306E
:101E0000E004D2178002C217786AE559F275F00B28
:101E1000A42409F582E5F0347AAF82F5648F65E594
:101E200059543F44807899F6E5591313543F543080
:101E300044807895F6E55A30E71878427401F2E468
:101E40002565F565740B3564F5647895E64440F6D0
:101E50008004E47842F2E55A540F789546F66470AF
:101E6000F6E55A30E335856582856483A3A3E030C7
:101E7000E00B856582856483E0454BF022856582B1
:101E8000856483E0454BFF7850F2E54CF45FF278CF
:101E900036E564F208E565F2D2272285658285641D
:101EA00083E0FFE54BF4FEEF5EF02275F02CE55980
:101EB000A42409F582E5F0344EAF82F5608F61FE0F
:101EC000AD59122979400302291F227F09122B38AC
:101ED0008F597F07122B388F5AE550640D6003022B
:101EE000291FE559D3943F400302291FE559448037
:101EF000F54BE55A30E709754CA1545FF54D800864
:101F0000754CC0780DE559F212519C221229208F90
:101F10005975F02CEFA42409F582E5F0344EAF8218
:101F2000F5608F617F07122B388F59E559C4540F24
:101F30004259E5612419F582E43560F583E559F0ED
:101F4000E5595411600C90918FE560F0A3E561F0C4
:101F5000801390918FE0B5600CA3E0B56107E49029
:101F6000918FF0A3F0E5595422600C909195E560B3
:101F7000F0A3E561F08013909195E0B5600CA3E0CB
:101F8000B56107E4909195F0A3F0E5595444600CD5
:101F900090919BE560F0A3E561F0801390919BE048
:101FA000B5600CA3E0B56107E490919BF0A3F0E568
:101FB000595488600D9091A1E560F0A3E561F002AD
:101FC0001C979091A1E065607004A3E065616003D7
:101FD000021C979091A1F0A3F0021C97E55424BF36
:101FE000602424FC603024F2600302291F301E03A9
:101FF00002291F30140302291FD21E78887441F26F
:10200000C2451297DC22D214C20C1299F912999D82
:10201000C2451297DC22C21EC214C209C20CC203FE
:102020001299E912998AC2451297DC129A2022C2AB
:10203000441229208F5975F02CEFA42409F582E56C
:10204000F0344EAF82F5608F61FEAD5912297950A0
:102050000302291FE539B44015E559D3947F400E9A
:10206000AF61AE60AD59122B52400302291F7F07AA
:10207000122B388F59E55930E00FE5612410F582B5
:10208000E43560F583E06402F0E55930E10FE56185
:102090002410F582E43560F583E06404F0E55930FE
:1020A000E40FE5612413F582E43560F583E0640113
:1020B000F0E55930E511E5612410F582E43560F56D
:1020C00083E06401F0D243E5396440703DE5593066
:1020D000E728E5612410F582E43560F583E06408C3
:1020E000F0E5612411F582E43560F583E030E10A22
:1020F000D244E55930E603435B10E5612408F582DC
:10210000E43560F5837402F0800EE5612408F58201
:10211000E43560F583740AF0E550640D7003022124
:10212000B17F05122B388F59E559603AE561241AC1
:10213000F582E43560F583E0FF30E72AE56124139A
:10214000F582E43560F583E0FEC313F55BEF30E024
:1021500003435B80E561240FF582E43560F583E09D
:10216000FFAD5B129AF5E5612413F582E43560F565
:1021700083E0FFE55925E0FEEF6EF0E55930E70F0B
:10218000E561241AF582E43560F583E06401F07FAF
:1021900003122B388F59E55925E0F559E561241ACA
:1021A000F582E43560F583E0FFE559541EFEEF6EDD
:1021B000F0304317E561240AF582E43560F583E0E9
:1021C00030E0057412F080037411F0E561240EF51F
:1021D00082E43560F583E0FF20E61D4440F0754B56
:1021E00034754C22E561240FF582E43560F583E017
:1021F000F54DE4F54E12519CE5612404F582E43579
:1022000060F583E064016009AF61AE607D01124E4C
:102210000E754B42754C06E561240FF582E435607E
:10222000F583E0F54DE5612410F582E43560F58332
:10223000E0F54EE5612411F582E43560F583E0F5C3
:102240004FE561240BF582E43560F583E0F550E558
:10225000612413F582E43560F583E0F551E56124EE
:102260001AF582E43560F583E0F55212519CE56180
:102270002411F582E43560F583E020E0030223E8D1
:10228000E5612410F582E43560F583E0F55A856058
:102290005E85615FE4F559E55F2406F582E4355E0D
:1022A000F583E0FEA3E08E5EF55F4E700302291F0A
:1022B000E55F65617004E55E6560700302291FE5F6
:1022C0005F2411F582E4355EF583E020E003022906
:1022D0001FE55F2410F582E4355EF583E054D1FFFD
:1022E000F0E55A542E4FF0E561240CF582E4356098
:1022F000F583E0FFE55F240CF582E4355EF583EFBE
:10230000F0E5612417F582E43560F583E0FFE55FD1
:102310002417F582E4355EF583EFF0E55F2420F5C0
:1023200082E4355EF583E04401F030442DE55F241E
:1023300020F582E4355EF583C083C082E0FFE55F6F
:102340002411F582E4355EF583E030E1047E1080EF
:10235000027E04EF4ED082D083F0304326E55F2426
:1023600010F582E4355EF583E06401F0E55F240A50
:10237000F582E4355EF583E030E0057412F0800309
:102380007411F0E55F2404F582E4355EF583E064C2
:10239000016018AF5FAE5E7D01124E0EE55F240E48
:1023A000F582E4355EF583E04440F0E55F2411F505
:1023B00082E4355EF583E054C0FFBF8010E55F2402
:1023C00008F582E4355EF583740AF0800EE55F243B
:1023D00008F582E4355EF5837402F00559E559C3CA
:1023E0009408500302229722E5612406F582E43521
:1023F00060F583E4F0A3F022E554B44510C2183030
:10240000290475320922C22BC202D22622E559B410
:102410005205753721800375373F1229208F59E502
:1024200039700302291FE53964807027855935E525
:10243000376421600302291F75375530290575322D
:102440000F8017D229E4F5327F05122B38786CEF14
:10245000F28007E55914F535D22B7F07122B388F00
:102460003A754B35754C01754D0512519CD21822A9
:102470007885E620E20302291F20430A90ECE874E5
:10248000FFF0A3F0800DE490ECE8F012059490ECDE
:10249000E9EFF01205948F5AE55A704A7F691205E8
:1024A0001890ECE9E0FF12057A7F6312051890ECB2
:1024B000E0E0FFF55A12057AE4F559E559C3955A5B
:1024C00050197F2012051874E02559F582E434EC88
:1024D000F583E0FF12057A055980E07F0D1205189B
:1024E0007F0A12051822855A311205948F3412057D
:1024F000948F3B1205948F3E1205948F3F120594E2
:102500008F40E534653BF53DE531C394044004E577
:102510003E623DE531C394054004E53F623DE5314F
:10252000C394064004E540623D7F6912051890ECB3
:10253000E9E0FF12057A7F201205187F6312051863
:10254000AF3112057A7F201205187F61120518AF8E
:102550003412057A7F201205187F64120518AF3BEC
:1025600012057A7F2012051890ECE0E531F0A37493
:1025700033F0A3E534F0A3E53BF0A3E53DF0E5310E
:10258000C3940440197F44120518AF3E12057A7FA8
:102590002012051890ECE4E53EF0A3E53DF0E531AE
:1025A000C3940540197F44120518AF3F12057A7F86
:1025B0002012051890ECE5E53FF0A3E53DF0E5318C
:1025C000C3940640197F44120518AF4012057A7F64
:1025D0002012051890ECE6E540F0A3E53DF0AF3D94
:1025E00012057A7F0D1205187F0A1205182230197C
:1025F000131205478F5AEF6003B40DF57E9E7F18C6
:102600001203CF221205948F4E7897E66023E538A7
:10261000654E601D1205478F5AEF6003B40DF57EBD
:102620009E7F1D1203CFAF3812057A7F0D12051859
:10263000221205948F4FE54F7019F5387897F612EE
:1026400005478F5AEF700302291F640D700302299A
:102650001F80ECE54F5407F54BD39405401312054A
:10266000478F5AEF6003B40DF57E9E7F211203CF92
:1026700022E4F55AE55AC3954B501512059474A2FD
:10268000255AF8EFF67450255AF8A607055A80E443
:10269000120547EF640D60087E9E7F211203CF2252
:1026A000E54F30E706789776FF8004E47897F67870
:1026B00098A64BE54F131313541F54077890F685D3
:1026C0004E38D219754B45754C08754D1412519CF6
:1026D000227F451205187F09122B388F5A7F071267
:1026E0002B388F59E55A701CE559C3947850157FE3
:1026F0000312057AAF5A12057AAF5912057A7F0D87
:1027000012051822E55A44C0F543855944E4F55BA7
:102710007554FF755C8075F02CE55CA4241DF58272
:10272000E5F0344EF583E0B5432B75F02CE55CA461
:10273000241EF582E5F0344EF583E0B5441775F0BC
:102740002CE55CA42409F582E5F0344EAF82F560F7
:102750008F61022839E554604175F02CE55CA424B2
:102760000DF582E5F0344EF583E0FFF552BF090820
:10277000855C5BE4F5548022E552701E75F02CE513
:102780005CA42427F582E5F0344EF583E0F553C3CD
:1027900095545006855C5B855354055CE55C60038D
:1027A000022716E55B70030228E6F55C75F02CA4A1
:1027B0002409F582E5F0344EAF82F5608F61F58330
:1027C000E582240AF582E43583F583E4F0E56124AB
:1027D0000DF582E43560F583E4F0E5612414F582BB
:1027E000E43560F583E543F0E5612415F582E435D1
:1027F00060F583E544F0E561240CF582E43560F58D
:1028000083E4F0E5612412F582E43560F583E4F0B9
:10281000E561240BF582E43560F583E4F0E561249D
:1028200011F582E43560F5837448F0E5612410F514
:1028300082E43560F5837440F0E5612404F582E4B8
:102840003560F583E064097053788606E5612404F9
:10285000F582E43560F5837404F075629175636503
:10286000AE62AF63AD61AC601250A1E5632405F5C3
:1028700082E43562F583E0FEA3E0B5631FEEB56246
:102880001B856382856283E0FEA3E0FFE563240588
:10289000F582E43562F583EEF0A3EFF0AF5C12054C
:1028A0007AAF5A12057AAF5912057A7F0D120518C0
:1028B000E5612404F582E43560F583E0F55A6401AE
:1028C0006015E55A6402600FE55A64036009AF6160
:1028D000AE607D04124E0EE561241EF582E4356083
:1028E000F58374FFF022E4FF12057AAF5A12057ADD
:1028F000AF5912057A7F0D120518227885E660051A
:10290000AF59120518120575EF60141205478F595B
:10291000EF640D600A7885E660EB12051880E62208
:10292000E554B44E05753940801BE554B44D05752A
:1029300039808011E554B45A05E4F5398007780EE2
:10294000E2F5398020855354855253855152855084
:1029500051854F50854E4F854D4E854C4D854B4C86
:102960007867E2F54BE554541F9005CE93C454F0BC
:10297000FFE553541F932FFF228E668F678F828E41
:1029800083E5822411F582E43583F583E054C0F5B4
:102990006AB53902C322E539B48008EDC3945140C9
:1029A00002D322E539B4400B783DE2FFEDD39F40DE
:1029B00002D322E567240AF582E43566F583E4F064
:1029C000E567240BF582E43566F583E4F0E56724DA
:1029D00012F582E43566F583E4F0E567240DF582AF
:1029E000E43566F583E4F0E567240CF582E43566AA
:1029F000F583E4F07887E630E1267F57120518AFBB
:102A00006A12057AE5672411F582E43566F583E0FC
:102A100054C0FF12057A7F0D1205187F0A1205189F
:102A2000AF67AE661250F8E56AB44023788616E5C3
:102A3000672404F582E43566F583E075F007A42485
:102A400049F582E5F03491AF82F5688F698021788D
:102A50009316E5672404F582E43566F583E075F0A6
:102A600007A4246CF582E5F03491AF82F5688F6994
:102A7000E5692405F582E43568F583E0FEA3E0FF0F
:102A8000B5670BEEB56607AD69AC68124FE3E56755
:102A90002411F582E43566F583E0543FF04539F0C2
:102AA000E5672404F582E43566F5837404F0E539BE
:102AB000B4401D788606E5672411F582E43566F595
:102AC00083E054F3F04408F0756891756965801BE4
:102AD000E5672411F582E43566F583E054F3F044AC
:102AE00008F0756891756988789306AE68AF69AD2E
:102AF00067AC661250A1E5692405F582E43568F5F6
:102B000083E0FEA3E0B5691FEEB5681B8569828589
:102B10006883E0FEA3E0FFE5692405F582E43568FB
:102B2000F583EEF0A3EFF0E567240EF582E4356659
:102B3000F583E054BFF0C322744B2FF8E6541F9086
:102B400005CE93C454F0FE744A2FF8E6541F932E1A
:102B5000FF228E668F678D687F45120518E5672412
:102B600004F582E43566F583E0B409117F051205AA
:102B70007AAF6812057A7F0D120518C322E4FF129E
:102B8000057AAF6812057AE5672414F582E43566A4
:102B9000F583E0543FFF12057AE5672415F582E4DA
:102BA0003566F583E0FF12057A7F0D120518D322F2
:102BB0008E598F5A8F828E83E5822404F582E43504
:102BC00083F583E0640160030231FEE55A2405F5D4
:102BD00082E43559F583E064A560030231DDE55AEE
:102BE0002410F582E43559F583E030E7030231DD46
:102BF0007885E620E103022C91E55A240FF582E462
:102C00003559F583E0FF12057A7F73120518E55AEE
:102C1000240AF582E43559F583E0FF12057A7F6DC9
:102C2000120518E55A2410F582E43559F583E0FFC2
:102C300012057A7F61120518E55A240BF582E435F6
:102C400059F583E0FF12057A7F73120518E55A24BF
:102C500012F582E43559F583E0FF12057A7F63129D
:102C60000518E55A240DF582E43559F583E0FF1285
:102C7000057A7F69120518E55A240CF582E4355966
:102C8000F583E0FF12057A7F0D1205187F0A120501
:102C900018E55A2410F582E43559F583E0FF30E554
:102CA00048E55A240BF582E43559F583E4F0E55AFA
:102CB0002412F582E43559F583E4F0E55A240DF544
:102CC00082E43559F583E4F0E55A240CF582E435C5
:102CD00059F583E054F0F0E55A240AF582E43559B9
:102CE000F583E05407F00231DDE55A2411F582E462
:102CF0003559F583E0FE755D0F54C0FDBD4012EE01
:102D0000540CFDBD0805755D078006BD0C03755D9F
:102D100002E55A240CF582E43559F583E0F55BE5CC
:102D20005A2417F582E43559F583E0FEE55A240B61
:102D3000F582E43559F583E0F55CEF20E1035306B5
:102D40000FEF20E2035306F0E55A240AF582E4353A
:102D500059F583E0540FB410004003023182902DE6
:102D600065F8282873022DA5022E95022F2B022D1F
:102D7000A5022F7E0230320230E6023135022D9557
:102D8000022E95022F2B022D95022F7E0230320249
:102D900030E6023135EE540F7003430601EE54F075
:102DA0007003430610E55A2412F582E43559F58381
:102DB000E0F9C313FFE55CC39F5060E55A240DF5AD
:102DC00082E43559F583E0FD14F0ED6003023182B1
:102DD0007408255CF55CE55A2412F582E43559F552
:102DE00083E0FDC313FDE55CD39D40028D5C535B26
:102DF000F0E55C131313541F425BEEC4540FFDE562
:102E00005B90A0A493FCED8CF0A4FDE55A240DF595
:102E100082E43559F583EDF0023182E55CD39F40C1
:102E200062E55A240DF582E43559F583E0FF14F08C
:102E3000EF600302318274F8255CF55CE55A2412D8
:102E4000F582E43559F583E0FFC313FFE55CC39FCA
:102E50004005E55C30E7028F5C535BF0E55C1313E3
:102E600013541F425BE55B90A0A493FFEE540F8FB9
:102E7000F0A4FFE55A240DF582E43559F583EFF00F
:102E8000023182E55A240AF582E43559F583E0548B
:102E900007F00231DDE55C7037E55A2412F582E473
:102EA0003559F583E0D3955D4006780AE2FF80024C
:102EB0007F00E55A240DF582E43559F583EFF0E5FE
:102EC0005A240AF582E43559F5837415F0023182EB
:102ED000E55A240DF582E43559F583E0FF14F0EF4F
:102EE0006003023182EE540F7003430601EE54F08A
:102EF000700343061074F8255CF55C30E703E4F5D5
:102F00005C535BF0E55C131313541F425BE55B906D
:102F1000A0A493FFEE540F8FF0A4FFE55A240DF503
:102F200082E43559F583EFF0023182E55C7037E5D4
:102F30005A2412F582E43559F583E0D3955D4006B5
:102F4000780AE2FF80027F00E55A240DF582E4351D
:102F500059F583EFF0E55A240AF582E43559F583F3
:102F60007414F0023182E55A240DF582E43559F5E6
:102F700083E0FF14F0EF6003023182022EE5E55A90
:102F8000240DF582E43559F583E0FF14F0EF60037A
:102F9000023182E55A241CF582E43559F583E0605C
:102FA00014E014F0E55A240DF582E43559F58374E4
:102FB0007DF0023182E55A2412F582E43559F58319
:102FC000E0D3955D40067809E2FF80027F00E55A74
:102FD000240DF582E43559F583EFF0E55A240AF51E
:102FE00082E43559F5837416F0E55A240EF582E42F
:102FF0003559F583E054FDF0E55A2410F582E435A7
:1030000059F583E054EEF0754B35754C03754D045E
:10301000E55A240FF582E43559F583E0F54EE55A7B
:103020002410F582E43559F583E0F54F12519C02E6
:103030003182E55A240DF582E43559F583E0FF1419
:10304000F0EF6003023182E55A241CF582E4355921
:10305000F583E06014E014F0E55A240DF582E435C0
:1030600059F583747DF0023182E55A2412F582E429
:103070003559F583E0D3955D40067809E2FF80027B
:103080007F00E55A240DF582E43559F583EFF0E52C
:103090005A240AF582E43559F5837417F0E55A2469
:1030A0000EF582E43559F583E04402F0E55A241028
:1030B000F582E43559F583E04411F0754B35754CD4
:1030C00003754D04E55A240FF582E43559F583E084
:1030D000F54EE55A2410F582E43559F583E0F54FB5
:1030E00012519C023182E55A240DF582E43559F5DE
:1030F00083E07031E55A241DF582E43559F583E00B
:103100006013E014F0E55A240DF582E43559F58397
:10311000747DF0806DE55A240AF582E43559F58313
:103120007418F0805DE55A240DF582E43559F58375
:10313000E014F0804DE55A240DF582E43559F5830D
:10314000E07031E55A241DF582E43559F583E060DD
:1031500013E014F0E55A240DF582E43559F5837433
:103160007DF0801EE55A240AF582E43559F5837412
:103170001BF0800EE55A240DF582E43559F583E005
:1031800014F0E55A240CF582E43559F583E55BF03B
:10319000E55A240BF582E43559F583E55CF0E55AF0
:1031A0002420F582E43559F583E04401F0E55A2402
:1031B00011F582E43559F583E054C0FFBF8010E576
:1031C0005A2408F582E43559F583740AF0800EE537
:1031D0005A2408F582E43559F5837402F0855A8241
:1031E000855983E0FEA3E08E59F55A8E832404F5B9
:1031F00082E43583F583E064017003022BCB222245
:10320000789DE6FF75F02CA42409F582E5F0344E94
:10321000AD82F5598D5AF583E5822411F582E435A6
:1032200083F583E0543070030232A58D82E5822459
:103230001AF582E43559F583E004F054037066759D
:103240004B35754C02754D098F4E12519C80567846
:103250009DE6FF75F02CA42409F582E5F0344EAD0F
:1032600082F5598D5AF583E5822411F582E4358380
:10327000F583E05430602E8D82E582241AF582E4D5
:103280003559F583E0D39402400E754B35754C02E9
:10329000754D0A8F4E12519CE55A241AF582E43579
:1032A00059F583E4F0E4789AF6228E5C8F5DED7038
:1032B00003023405E55D2419F582E4355CF583E00D
:1032C0005D6010E55D2410F582E4355CF583E03047
:1032D000E01322E55D2410F582E4355CF583E020FF
:1032E000E003023405754B35754C03754D04855C60
:1032F0005E855D5FE4F560E55F2410F582E4355E90
:10330000F583E06401F0E55F240AF582E4355EF5BB
:1033100083E030E0057412F080037411F0E55D2461
:103320001CF582E4355CF583E0FFE55F241CF58243
:10333000E4355EF583EFF0E55D241DF582E4355C50
:10334000F583E0FFE55F241DF582E4355EF583EF4C
:10335000F0E55F2404F582E4355EF583E064016006
:1033600048AF5FAE5E7D01124E0EE55F2420F58210
:10337000E4355EF583E04401F0E55F2411F582E475
:10338000355EF583E054C0FFBF8010E55F2408F58B
:1033900082E4355EF583740AF0800EE55F2408F55B
:1033A00082E4355EF5837402F0E55F240FF582E474
:1033B000355EF583E0F54EE55F2410F582E4355E79
:1033C000F583E0F54F12519CE55F2406F582E43564
:1033D0005EF583E0FEA3E08E5EF55F4E6027E55F5D
:1033E000655D7004E55E655C601BE55F2411F58238
:1033F000E4355EF583E030E00C0560E560C39408D9
:1034000050030232F722302103023EFE301B06C277
:103410001B128CA0227885E630E255E4F55274E068
:103420002552F582E434ECF583E0FF74782552F8F8
:10343000EFF20552E552B408E590ECE9E0FF90ECBC
:10344000E8E0FE04F0EEC39F501D787C74FFF27834
:103450007AF2E4787BF278787403F2A3E0B4FF0C9C
:10346000E490ECE8F08005E490ECE8F01287A32209
:103470007887E630E203D38001C3924330064520CB
:103480002942202B3F789206E6C39405403630232C
:10349000117899E6FF7895E6FD128C5C78927603B8
:1034A0008014302702D21F7899E6FF7895E6FD1246
:1034B0008788E47892F67883E214F26003023EFE95
:1034C000129B21227886E67003023B49300B0302EF
:1034D0003B497893E66002D20B20190302355C3039
:1034E000290302355C202B7430206FC2207898E6C7
:1034F000FF047878F27834E27879F278A2E6FE7800
:103500007AF278A3E6FD787BF2EE6D787CF2EFD369
:103510009402403978A4E6FE787CE26E787DF278F9
:103520007CEEF2EFD39403402478A5E6FE787DE2AA
:103530006E787EF2787DEEF2EFD39404400F78A699
:10354000E6FF787EE26F787FF2787EEFF21287A353
:103550007890E67003023EFE1622D22030192878B9
:1035600090E67003D38001C3501DC219754B3575A9
:103570004C03754D1485384E754FFF7897E67004EF
:10358000F54FF53812519CC2447897E6600616E66E
:103590007002F53830431F7E9E7F261203CFE53C34
:1035A00090A28593FF12057A7E9E7F2E1203CF781C
:1035B00094E6FF12057A7843E2700302364B755C9D
:1035C00001E4F55BE55BC39404400302364B7843AA
:1035D000E2FF555C606AE55CF4FEEF5EF274722512
:1035E0005BF8E275F02CA42409F582E5F0344EAFC7
:1035F00082F5598F5AF583E5822413F582E43583E9
:10360000F583E0FF7D80541CFEC3134205E55A2478
:103610001AF582E43559F583E030E603430501EFFE
:1036200030E015E55A2411F582E43559F583E0546C
:103630000C64046003430510AF5AAE591286AA22E7
:10364000055BE55C25E0F55C0235C4E53C90A285B0
:10365000937003023AAC24FE7003023760147003C7
:1036600002388B1470030239B624036003023E9BB8
:103670003043057F21120518909155E0FEA3E08E9E
:1036800059F55A2404F582E43EF583E064016003B1
:1036900002375A30430AAF5AAE597D61FB123EFFE2
:1036A000E55A2405F582E43559F583E064A56017F1
:1036B000AF5AAE597D39125144AF5AAE597C917D03
:1036C00050124FE302375A30041CE55A240FF5829A
:1036D000E43559F583E0FF7894E6B50703D380011C
:1036E000C35003023760E5386010E55A240FF582B5
:1036F000E43559F583E065386066AF5AAE59124734
:10370000AAAF5AAE597C917D50124FE3E55A240876
:10371000F582E43559F583E06006E014F0023E9B43
:10372000E55A240AF582E43559F583E030E40302D2
:103730003E9BAF5AAE597D02124E0EE55A2408F553
:1037400082E43559F5837402F0E55A2409F582E4E0
:103750003559F5837419F0023E9B20440302388BDF
:103760003043057F2212051890915CE0FEA3E08EA5
:1037700059F55A2404F582E43EF583E064026003BF
:1037800002388B30430AAF5AAE597D61FB123EFFBF
:10379000E55A2405F582E43559F583E064A5601700
:1037A000AF5AAE597D41125144AF5AAE597C917D0A
:1037B00057124FE302388B204413E55A2408F58250
:1037C000E43559F583E024FF400302388030041CBF
:1037D000E55A240FF582E43559F583E0FF7894E645
:1037E000B50703D38001C3500302388BE53860135B
:1037F000E55A240FF582E43559F583E06538700306
:1038000002388BAF5AAE591247AAAF5AAE597C91C3
:103810007D57124FE320440EE55A2408F582E43523
:1038200059F583E014F0E55A2409F582E43559F599
:1038300083E06003023E9BAF5AAE597D03124E0EE9
:10384000E55A240FF582E43559F583E0D3947F409F
:103850000EE55A241EF582E43559F58374FFF0E530
:103860005A2411F582E43559F583E054CFF0E55A36
:10387000240EF582E43559F583E054DFF0023E9BD7
:10388000AF5AAE597C917D57124FE33043057F24E8
:10389000120518909163E0FEA3E08E59F55A2404B6
:1038A000F582E43EF583E0640360030239B63043F9
:1038B0000AAF5AAE597D61FB123EFFE55A2405F569
:1038C00082E43559F583E064A56017AF5AAE597D9F
:1038D00042125144AF5AAE597C917D5E124FE302C1
:1038E00039B6204413E55A2408F582E43559F583A6
:1038F000E024FF40030239AB30041CE55A240FF5E5
:1039000082E43559F583E0FF7894E6B50703D38068
:1039100001C350030239B6E5386013E55A240FF5A8
:1039200082E43559F583E0653870030239B6AF5A41
:10393000AE591247AAAF5AAE597C917D5E124FE341
:1039400020440EE55A2408F582E43559F583E01445
:10395000F0E55A240FF582E43559F583E0D3947FDE
:103960005003023E9BE55A241EF582E43559F58347
:10397000E07003023E9B7851E230E003023E9BE59B
:103980005A241EF582E43559F583E014F0600302F1
:103990003E9BAF5AAE59FD124E0EE55A241EF582DB
:1039A000E43559F58374FFF0023E9BAF5AAE597C63
:1039B000917D5E124FE33043057F251205189091EB
:1039C0006AE0FEA3E08E59F55A2404F582E43EF540
:1039D00083E064046003023AAC30430AAF5AAE5944
:1039E0007D61FB123EFFE55A2405F582E43559F569
:1039F00083E064A56017AF5AAE597D43125144AFBE
:103A00005AAE597C917D65124FE3023AAC30041CEA
:103A1000E55A240FF582E43559F583E0FF7894E602
:103A2000B50703D38001C35003023AACE5386010F8
:103A3000E55A240FF582E43559F583E06538606C6A
:103A4000AF5AAE591247AAAF5AAE597C917D651252
:103A50004FE3E55A240FF582E43559F583E0D3941A
:103A60007F5003023E9BE55A241EF582E43559F54A
:103A700083E07003023E9B7851E230E003023E9BFC
:103A8000E55A241EF582E43559F583E014F060030D
:103A9000023E9BAF5AAE59FD124E0EE55A241EF55A
:103AA00082E43559F58374FFF0023E9B3043057F75
:103AB0002612051890914EE0FEA3E08E59F55A2487
:103AC00004F582E43EF583E0706D30430AAF5AAEF0
:103AD000597D61FB123EFFE55A2405F582E4355914
:103AE000F583E064A5600BAF5AAE597D4412514492
:103AF0008037300419E55A240FF582E43559F583EF
:103B0000E0FF7894E6B50703D38001C34029E53888
:103B10006010E55A240FF582E43559F583E06538E5
:103B20006015AF5AAE591247AAAF5AAE597C917D73
:103B300049124FE3023E9B204405D2440236707F77
:103B4000FFE4FD128788023E9BC20B7893E6700368
:103B5000023E9BC24430431F7E9E7F321203CFE55C
:103B60003C90A28593FF12057A7E9E7F2E1203CF92
:103B70007894E6FF12057AE53C90A28593700302E3
:103B80003E3624FE7003023C62147003023D35147D
:103B90007003023DCF24036003023E953043057F4E
:103BA00021120518909178E0FEA3E08E59F55A2471
:103BB00004F582E43EF583E064016003023C523088
:103BC000430AAF5AAE597D61FB123EFFE55A240508
:103BD000F582E43559F583E064A56016AF5AAE5915
:103BE0007D45125144AF5AAE597C917D73124FE31B
:103BF0008060AF5AAE59124BC8AF5AAE597C917D16
:103C000073124FE3E55A2408F582E43559F583E051
:103C10006006E014F0023E95E55A240AF582E43588
:103C200059F583E030E403023E95AF5AAE597D0268
:103C3000124E0EE55A2408F582E43559F5837402D4
:103C4000F0E55A2409F582E43559F5837419F00238
:103C50003E9520440D301D05C21D023D35D21D028A
:103C60003DCF3043057F2212051890917FE0FEA3DF
:103C7000E08E59F55A2404F582E43EF583E06402AF
:103C80006003023D3530430AAF5AAE597D61FB12E5
:103C90003EFFE55A2405F582E43559F583E064A535
:103CA0006017AF5AAE597D46125144AF5AAE597C97
:103CB000917D7A124FE3023D35204410E55A2408E5
:103CC000F582E43559F583E024FF505EAF5AAE59D2
:103CD000124BC8AF5AAE597C917D7A124FE3204403
:103CE0000EE55A2408F582E43559F583E014F0E531
:103CF0005A2409F582E43559F583E06003023E95C4
:103D0000AF5AAE597D03124E0EE55A2411F582E4E6
:103D10003559F583E054CFF0E55A240EF582E435A9
:103D200059F583E054DFF0023E95AF5AAE597C91CD
:103D30007D7A124FE33043057F2412051890918657
:103D4000E0FEA3E08E59F55A2404F582E43EF583A3
:103D5000E06403707A30430AAF5AAE597D61FB12BA
:103D60003EFFE55A2405F582E43559F583E064A564
:103D70006016AF5AAE597D47125144AF5AAE597CC6
:103D8000917D81124FE38047204410E55A2408F5C5
:103D900082E43559F583E024FF5029AF5AAE591219
:103DA0004BC8AF5AAE597C917D81124FE33044032A
:103DB000023E95E55A2408F582E43559F583E0146E
:103DC000F0023E95AF5AAE597C917D81124FE3309F
:103DD00043057F2512051890918DE0FEA3E08E59D2
:103DE000F55A2404F582E43EF583E064047047301C
:103DF000430AAF5AAE597D61FB123EFFE55A2405D6
:103E0000F582E43559F583E064A56016AF5AAE59E2
:103E10007D48125144AF5AAE597C917D88124FE3D0
:103E20008014AF5AAE59124BC8AF5AAE597C917D2F
:103E300088124FE3805F3043057F2612051890916A
:103E400071E0FEA3E08E59F55A2404F582E43EF5B4
:103E500083E0703C30430AAF5AAE597D61FB123E9D
:103E6000FFE55A2405F582E43559F583E064A56041
:103E70000BAF5AAE597D491251448007AF5AAE5923
:103E8000124BC8AF5AAE597C917D6C124FE380053E
:103E9000D244023B9C789CE620E063053C533C7F87
:103EA000E53C704A788306E6C394805002768078B9
:103EB00083E6FF75F02CA4240DF582E5F0344EF571
:103EC00083E0702A75F02CEFA42427F582E5F03406
:103ED0004EF583E060187851E220E01275F02CEF87
:103EE000A42427F582E5F0344EF583E014F07886BB
:103EF000E66003123F677893E66003124042228E29
:103F00005D8F5E8D5F8B607F20120518AF5F12059D
:103F100018E55E240FF582E4355DF583E0FF1205B8
:103F20007AE55E2404F582E4355DF583E0FF120551
:103F30007AE55E2408F582E4355DF583E0FF12053D
:103F40007AE55E2409F582E4355DF583E0FF12052C
:103F50007AE560B40110E55E2411F582E4355DF583
:103F600083E0FF12057A22E53C540F707090915760
:103F7000E0FEA3E08E5DF55E2404F582E43EF58369
:103F8000E064027058E55E2405F582E4355DF58352
:103F9000E064A5600BAF5EAE5D7D4A125144803D8A
:103FA000E55E2408F582E4355DF5837402F0E55E94
:103FB0002409F582E4355DF583E06003E014F085C3
:103FC0005E82855D83E0FEA3E08E5DF55E8E8324D8
:103FD00004F582E43583F583E0640260A8E53C548F
:103FE0001F705E90915EE0FEA3E08E5DF55E24049E
:103FF000F582E43EF583E064037046E55E2405F552
:1040000082E4355DF583E064A5600AAF5EAE5D7D58
:104010004B12514422E55E2408F582E4355DF583B8
:104020007402F0855E82855D83E0FEA3E08E5DF51F
:104030005E8E832404F582E43583F583E0640360B7
:10404000BA22E53C540F707090917AE0FEA3E08EA6
:104050005DF55E2404F582E43EF583E06402705869
:10406000E55E2405F582E4355DF583E064A5600B2B
:10407000AF5EAE5D7D4C125144803DE55E2408F597
:1040800082E4355DF5837402F0E55E2409F582E48F
:10409000355DF583E06003E014F0855E82855D8325
:1040A000E0FEA3E08E5DF55E8E832404F582E435A8
:1040B00083F583E0640260A8E53C541F705E909134
:1040C00081E0FEA3E08E5DF55E2404F582E43EF51A
:1040D00083E064037046E55E2405F582E4355DF512
:1040E00083E064A5600AAF5EAE5D7D4D125144224F
:1040F000E55E2408F582E4355DF5837402F0855EA3
:1041000082855D83E0FEA3E08E5DF55E8E832404F0
:10411000F582E43583F583E0640360BA227880E2B7
:1041200054C0FFBFC00BD226C202C22BE47890F26B
:10413000227885E630E403D38001C392433016042D
:10414000D212D213C244127D74500D7890E26402F0
:104150006006D244127D74221284FA7B057A9E791D
:104160003AE4FD1285AE3043077E9E7F4B1203CFAB
:1041700030130812997F7819742DF2E4FFFD128A2A
:104180003A90F00B740CF0D2BBD2C3E47887F2F50E
:10419000567884F6F532202B030246FC30250AC2FD
:1041A00025C2AFD2AED2BED2AF781BE66043C244C6
:1041B00012527B7885E630E627E54164466005E5E6
:1041C00041B44703204319AF4112057AAF421205AB
:1041D0007AAF4312057A7F0D1205187F0A1205186F
:1041E000E541B4450CE543B4050775320AE478842B
:1041F000F6300C15786E7402F23043077E9E7F56BF
:104200001203CF753205024669E532B40E005086BE
:10421000904217F82828730242410242750242CCAC
:1042200002463A02451C0246690243A30241960235
:10423000448A0246940246C40245C802419602429C
:10424000E6129A0930132B7884E6C3940A40F8E406
:104250007884F630430C7887E270077E9E7F641284
:1042600003CF7881E2FF7887E204F2C39F50030214
:1042700041967532013043077E9E7F6E1203CFE474
:10428000F556786E74FFF2E53764527026FF7D01B3
:10429000128A3A7819747CF27B057A9E797C7D10BB
:1042A0001285AE3043077E9E7F861203CF753203A0
:1042B0000241961299697819747CF23043077E9E08
:1042C0007F951203CFE47884F6753202784DE2FFD1
:1042D000E556C39F50030241963043077E9E7F9F61
:1042E0001203CF75320D7F06C244127E5D789BA605
:1042F000073043137E9E7FAA1203CF789BE6FF12FE
:10430000057A7F0A120518789BE6D39499402A789B
:104310006E7402F23043077E9E7FB41203CF789B07
:10432000E6C394FE5005E537B43F0E12997F781925
:10433000742DF2753205024669789B741E26F67B51
:10434000057A9E79C67D101285AEE5352401FFE41D
:1043500033FEE4FD1285EE7B057A9E79C97D161247
:1043600085AEE537B43F137829743FF2753EE07FA0
:1043700078AD357BE0128A55801178297421F28559
:104380003A3E7F7CAD35AB3A128A553043077E9E6C
:104390007FCE1203CFE4F5567896F67889F6D208E8
:1043A000753206E556C3940A403AE537B43F1CE53A
:1043B0003E20E317433E087F78AD35AB3E128A5569
:1043C000E4F5567896F6D2080241963043077E9E71
:1043D0007FDF1203CFE4FFFD128A3AE4F55675320F
:1043E000080241967896E6C3940450030241963041
:1043F00043197F49120518AF5612057A7F2012051E
:1044000018AFD912057A7F20120518E537643F707E
:1044100054E53E30E3125407FF7401A807088002F8
:10442000C333D8FC788946F6533EF7754B35754C47
:1044300002754D067889E6F54E12519C78917617F3
:10444000AF357E00E4FD1285EEE53E64E7601605BB
:104450003E7F78AD35AB3E128A55E4F5567896F638
:10446000D208024196E537B42105853A4F80057898
:1044700089E6F54F754C03754D0785354E12472279
:10448000E47884F6753209024694E556C3940750E1
:1044900003024196E535D394074005E535B41C0683
:1044A000E53564047037E537643F7022F53EF55614
:1044B0007896F6D2087F74AD35AB3E128A553043FC
:1044C000077E9E7FFF1203CF75320B024196786EF6
:1044D000E2B4FF037409F2753205024669E535B4AA
:1044E0001C057534748006E5354470F534E537B441
:1044F0003F05E4F53B8006433478853A3B3043077B
:104500007E9F7F151203CFE4F5567896F6D208AF5A
:1045100034AD3B128A3A753204024196E556B40135
:10452000047888A63BE537B43F047F0980027F0BFF
:10453000EF65567045E537643F7030053BE53B60FD
:104540002A78917617FF7E00E4FD1285EE754B35D3
:10455000754C02754D06853B4E12519CE4F556D2C2
:1045600008AF34AD3B128A3A024196786EE2B4FF4E
:10457000037404F27532050246697896E6C3940422
:10458000500302419630431B7E9F7F271203CFAF1B
:104590005612057A7F49120518AFD912057A7F0A9B
:1045A000120518754C03754D0785354EE537B42156
:1045B00005853A4F80057888E6F54F124722E47862
:1045C00084F6753209024694E556B401047888A64B
:1045D0003EE556C39406403D053EE53E602C78918D
:1045E0007611FF7E00E4FD1285EE754B35754C02A9
:1045F000754D06853E4E12519CE4F556D208AF34F7
:10460000AD3BAB3E128A55024196786E7404F2754A
:1046100032050241967896E6C3940450030241960F
:10462000754C03754D0785354E7888E6F54F124772
:1046300022E47884F6753209805AE556D394014015
:1046400003129969E556C394505003024196754B85
:1046500035754C03754D07E4F54EF54F12519CE44A
:104660007884F67532090241963043137E9F7F2D80
:104670001203CF786EE2FF12057A7F0A12051875D1
:104680004C02754D08786EE2F54E124722E47884AC
:10469000F67532091299AD500F7819742DF278849D
:1046A000E6C394C8500F80F67819742DF27884E62A
:1046B000C3941E40F83043077E9F7F351203CFC25C
:1046C0002B0241961299AD500F7819742DF278840F
:1046D000E6C394C8500F80F67819742DF27884E6FA
:1046E000C3941E40F83043077E9F7F3F1203CFC222
:1046F0002BD226C202E47890F202419630160512BF
:10470000997F8003129969129A1478447414F230D4
:1047100043077E9F7F4C1203CF90F00B7404F0C2CE
:10472000BB22754B353018307F511205187F4E1261
:104730000518E54DB40809786EE2FF12057A800588
:10474000E4FF12057AE53504FF12057AAF4F120532
:104750007A7F0A120518800312519C7885E630E4AE
:104760001D7E9F7F551203CFE53504FF12057A7F2A
:104770002C120518AF4F12057A7F0A120518E54D65
:10478000B408197B057A9F795E7D101285AE789109
:104790007616AF4E7E00E4FD1285EE2278917617F4
:1047A000AF4F7E00E4FD1285EE228E5D8F5E8F821C
:1047B0008E83E582240FF582E43583F583E0F55F8F
:1047C0003029030249DE302B030249DEE55E240571
:1047D000F582E4355DF583E064A5600AAF5EAE5D09
:1047E0007D4F12514422E55E2411F582E4355DF5DA
:1047F00083E054C0FFBF800AAF5EAE5D7D501251B2
:1048000044227887E630E20C7E9F7F691203CFAFA7
:104810005F12057A301E0AE4FF7888E2FD1287886D
:1048200022E55E2410F582E4355DF583E030E7088B
:104830007FFFE4FD128788227894A65FE55F70030E
:104840000249DE7859E2655F7039E55E240EF58233
:10485000E4355DF583E0A2E19241E55E240BF5824B
:10486000E4355DF583E0547FF560C4540FF518E539
:1048700060C454F0F51974252519F519740135181B
:10488000F51822E55E2404F582E4355DF583E064E5
:10489000016003024966E55E2408F582E4355DF5B2
:1048A00083E0F561E55E2420F582E4355DF583E083
:1048B000F56230E016AF5EAE5D124AA3E561D394B7
:1048C0000140030249DE5362FE8073E56230E11667
:1048D000AF5EAE5D1249F6E561D394014003024933
:1048E000DE5362FD8058E56230E216AF5EAE5D12C7
:1048F0004A46E561D3940140030249DE5362FB80DE
:104900003DE56230E316AF5EAE5D124A8CE561D3E1
:10491000940140030249DE5362F78022E56230E4ED
:1049200016AF5EAE5D1249DFE561D394014003022C
:1049300049DE5362EF8007AF5EAE5D124AA3E562C7
:10494000541F60047F0380027F00E55E2408F58227
:10495000E4355DF583EFF0E55E2420F582E4355D16
:10496000F583E562F022E55E241FF582E4355DF50E
:1049700083E014601914602214603F14604824041A
:10498000704EAF5EAE5D124AA37560018042AF5EAD
:10499000AE5D1249F67560028036AF5EAE5D124ABA
:1049A00046E55E2411F582E4355DF583E030E104EF
:1049B0007F0380027F008F608016AF5EAE5D124A7B
:1049C0008C756004800AAF5EAE5D1249DFE4F5606D
:1049D000E55E241FF582E4355DF583E560F0227D18
:1049E0003EE4FBEF2410F582E43EF583E030E30281
:1049F0007B8012870D22EF241AF582E43EF583E0D6
:104A0000FCEF2413F582E43EF583E0FB7D80EC307F
:104A1000E711EB541CFAC3134205EC30E60D4305D5
:104A2000018008EB541EFCC3134205EB30E013EF8A
:104A30002411F582E43EF583E0540C6404600343E2
:104A400005101286AA22EF2413F582E43EF583E0D6
:104A50007DA054E0FCC41354074205EF241AF582EC
:104A6000E43EF583E030E003430508EF2411F582CE
:104A7000E43EF583E020E10DEF2410F582E43EF5FD
:104A800083E030E3034305101286AA22EF241AF5CF
:104A900082E43EF583E07DA0541EFCC31342051260
:104AA00086AA228E638F648F828E83E5822411F51D
:104AB00082E43583F583E0F5678F828E83E5822477
:104AC0000BF582E43583F583E0F5688F828E83E50C
:104AD00082240EF582E43583F583E0F5698F828EBA
:104AE00083E5822413F582E43583F583E0F56AE5F6
:104AF00067540C640C704375653F8F828E83E5822A
:104B00002410F582E43583F583E030E50575660110
:104B10008014E568547FF566D394004009E566C3C8
:104B2000947F50020566E56920E103436680AF6427
:104B3000AE63AD65AB6612870D22756540E56920F1
:104B4000E103436520E5642410F582E43563F583D1
:104B5000E030E515436501E567540C6408605FE5E6
:104B60006A13505A4365108055E567540C64087009
:104B70002FE5681313543FF566D3941C4003756604
:104B80001FE566600BC3941D500674032566F56629
:104B9000E56630E003436510E566C3134265801E99
:104BA000E568131313541FF5666007C3940F500292
:104BB0000566E5664265E56A30E003436510AF646B
:104BC000AE63AD651286AA228E5D8F5E3029030228
:104BD0004E0D302B03024E0DE55E2405F582E435C3
:104BE0005DF583E064A5600AAF5EAE5D7D51125154
:104BF0004422E55E2411F582E4355DF583E054C07E
:104C00006480600AAF5EAE5D7D5212514422E55E63
:104C1000240FF582E4355DF583E0F55FC3945140E0
:104C200003024E0DE55E240EF582E4355DF583E06A
:104C3000FFF561E55E2416F582E4355DF583E05409
:104C400030FEBE10035361EFE56130E422E55E24DF
:104C50000EF582E4355DF583EF54EFF0AF5FE55E6E
:104C60002413F582E4355DF583E0FD128C2F2230AC
:104C70001E1AE56130E00FE55E240EF582E4355D35
:104C8000F583E054FEF0E4F560024D1AE56130E092
:104C900011E55E240EF582E4355DF583E054FEF007
:104CA000804BE561A2E292F7A2E130F701B3503DFB
:104CB000436101D21BE56130E10543610480035388
:104CC00061FBE55E240EF582E4355DF583E561F078
:104CD0007560807560C0AF5FAD60E55E2413F582DE
:104CE000E4355DF583E0139245128C8022E55E2465
:104CF0000BF582E4355DF583E0FF131313541F5465
:104D00000FF5606006640F60020560856062E56013
:104D1000540F90A1F59354AAF560E55E241BF5822B
:104D2000E4355DF583E0540714601624FE603224F8
:104D3000FE604E240524F94003024DC16063024D1C
:104D4000D6E55E2413F582E4355DF583E030E104B9
:104D50007F1080027F00E5622F90A2059342608061
:104D600075E55E2413F582E4355DF583E030E204F9
:104D70007F3080027F20E5622F90A2059342608001
:104D800055E55E2413F582E4355DF583E030E304F8
:104D90007F5080027F40E5622F90A20593426080A1
:104DA00035E55E2413F582E4355DF583E030E404F7
:104DB0007F7080027F60E5622F90A2059342608041
:104DC00015E56130E1054360448003436010E56010
:104DD00020E103436001E55E241BF582E4355DF5C7
:104DE00083E004F05403700FE55E240EF582E43591
:104DF0005DF583E04410F0AF5FAD60E55E2413F530
:104E000082E4355DF583E0139245128C80228E7129
:104E10008F728D738F828E83E5822405F582E4354F
:104E200083F583E064A560067D5312514422E57248
:104E30002404F582E43571F583E0F57664097003A6
:104E4000024FE2E57365767003024FE27887E63041
:104E5000E177E509D3947350F97F55120518E5728F
:104E6000240FF582E43571F583E0FF12057AE572CF
:104E70002411F582E43571F583E054C0FFBF80074B
:104E80007F6D120518801EE5722411F582E43571DC
:104E9000F583E054C0FFBF40077F6E120518800500
:104EA0007F7A120518E5722404F582E43571F583E2
:104EB000E04430FF120518E5732430FF1205187F17
:104EC0000D1205187F0A120518AF72AE711250F854
:104ED000E5722411F582E43571F583E054C0F5766E
:104EE00064407062E5722404F582E43571F583E074
:104EF00075F007A42449F582E5F03491AF82F5748A
:104F00008F75F583E5822405F582E43583F583E02A
:104F1000FEA3E0FFB5720BEEB57107AD75AC741270
:104F20004FE3E5722404F582E43571F583E573F00F
:104F300075F007E573A42449F582E5F03491AF825A
:104F4000F5748F758060E5722404F582E43571F59F
:104F500083E075F007A4246CF582E5F03491AF820C
:104F6000F5748F75F583E5822405F582E43583F5C4
:104F700083E0FEA3E0FFB5720BEEB57107AD75AC33
:104F800074124FE3E5722404F582E43571F583E58C
:104F900073F075F007E573A4246CF582E5F03491A5
:104FA000AF82F5748F75AE74AF75AD72AC7112507F
:104FB000A1E5752405F582E43574F583E0FEA3E0F0
:104FC000B5751FEEB5741B857582857483E0FEA3ED
:104FD000E0FFE5752405F582E43574F583EEF0A372
:104FE000EFF0228E778F788C798D7A7887E630E4AF
:104FF000407E9F7F6C1203CFE5782404F582E43570
:1050000077F583E0FF12057A857882857783E0FE65
:10501000A3E0AA06F97B02126D0F8578828577835B
:10502000E0FEA3E02404F582E43EF583E0FF1205F0
:105030007AE5782404F582E43577F583E0D39405A6
:10504000502A857882857783E0FEA3E0FFE57A2405
:1050500005F582E43579F583EEF0A3EFF0EF240453
:10506000F582E43EF583E0D39405401B857A828582
:105070007983E0FEA3E0FFE57A2405F582E4357943
:10508000F583EEF0A3EFF0E5782405F582E43577BB
:10509000F583E064A56009AF78AE777D5412514482
:1050A000228E778F78AF05AE04EF2405F582E43EBB
:1050B000F583E064A5703B857882857783E0FCA367
:1050C000E0FD4C600B8D828C83A3A3EEF0A3EFF088
:1050D000857882857783EEF0A3EFF0F5828E83A347
:1050E000A3E577F0A3E578F08F828E83ECF0A3ED53
:1050F000F0227D55125144228F828E83E0FCA3E082
:105100008C77F5788F828E83A3A3E0FCA3E0FDEF7C
:105110002405F582E43EF583E0B4A522ED4C60233E
:10512000AA77AB788D828C83EAF0A3EBF04A601308
:10513000857882857783A3A3ECF0A3EDF0227D56DA
:10514000125144228E7B8F7C8D7D8F828E83E582EF
:10515000240FF582E43583F583E090FE01F090FEA4
:1051600000E57DF07887E630E5317F2A120518AF3B
:105170007D120518AE7BAF7C12057AE57BFF120528
:105180007AE57C240FF582E4357BF583E0FF120598
:105190007A7F0D1205187F0A12051822E4F5759022
:1051A000F711E0543064207042900001E0FF90005D
:1051B00000E02FFF900002E02FF5760575E575D32E
:1051C00094FA40DB303C0302527AD23C90F70074F0
:1051D00003F0740AF0781A74FFF67885E620E50388
:1051E00002527A7E9F7F701203CF2290F712E54B16
:1051F000F0E54C54E0A3F0E54CC454F0440890F7BB
:1052000016F0E54C540FF576E4F575E575C3957623
:105210005018744D2575F8E6FF74172575F582E46E
:1052200034F7F583EFF0057580E190F7117465F0C0
:10523000781CE6C394FF5001067885E630E53B7F95
:1052400053120518AF4B12057A7F20120518AF4C88
:1052500012057A7F3A120518E4F575E575C395765F
:10526000500E744D2575F8E6FF12057A057580EB32
:105270007F0D1205187F0A12051822C245302A0F29
:10528000C22A7F417CEC7DE07B0A12CFA680547855
:105290001DE6FE2412F582E434F7F583E0F541744F
:1052A000162EF582E434F7F583E0FFC4540FFF7443
:1052B000132EF582E434F7F583E04FF5427F43EE99
:1052C0002417FDE434F7FCE542540FFB12CFA67817
:1052D0001D741026F6B4F0027610781B16204403D5
:1052E0000264FE7885E6FF30E650E54164466005DD
:1052F000E541B44704EF20E441AF4112057A7F2035
:10530000120518AF4212057A7F3A120518E5425489
:105310000FF567E4F566E566C3956750137443259A
:1053200066F8E6FF12057A7F20120518056680E60A
:105330007F0D1205187F0A12051830210FE5416410
:10534000356009E541644560030264FEE54154C0EF
:10535000FFBFC00412A7D722E54154C06480600398
:10536000025403E54254E0FFBFA00412BBAB227815
:105370009FE67058E54254E064407050E541543F68
:10538000FF780DE26F7045E542540FF5677F4E12CE
:105390000518780DE2FF12057AE56724FCFF120577
:1053A0007A756606E5672402FFE433FEC3E5669F6F
:1053B000EE6480F8748098500E74412566F8E6FF1C
:1053C00012057A056680DD789F763222789FE6D3D3
:1053D000940050030264FEE54254E064206003023E
:1053E00064FEE541543FFF780DE26F60030264FE06
:1053F000E54320E5030264FE541FFF12057A789FFF
:10540000763222E54124E7B4360040030264FE9080
:105410005416F82828730264F70264FE0264FE0240
:1054200064F70264FE0264FB0264FE0255F4025B50
:1054300016025BCC025E2D0264FE025F920261E9FD
:105440000261FD0262540262CC025538026312020C
:10545000631602631A0264720264FE0264FE02644E
:10546000FE0264FE0264FE0254B80254DE0264FED0
:105470000264FE0264FE0264FE0264FE0264FE0236
:1054800064FE0264FE0264FE0264FE0255F4025BE6
:1054900016025BCC025E2D0264FE025F920261E99D
:1054A0000261FD0262540262CC02553802631202AC
:1054B000631602631A02647275F02CE543A4240992
:1054C000F582E5F0344EAF82F5648F65F583E582B1
:1054D000240EF582E43583F583E054BFF022E543E2
:1054E000146021146031146039240360030264FEE7
:1054F0001299E912998A129A20C21EC214C209C2D4
:105500000CC203223014061299E912998AD21EC2E3
:105510001478887441F2221299F912999DC20CD222
:1055200014221299F912999DC20CE542B40204D2D8
:10553000038002D209D2142275F02CE543A4240979
:10554000F582E5F0344EAF82F5648F65F583E58230
:105550002410F582E43583F583E054C02480605D37
:105560008000754B307F4DE565240FFDE43564FC0C
:105570007B0712CFA67859E2B54D06534FF3434F40
:105580000C754C27E543D3947F4065E54F54C064C8
:1055900040705DE5652404F582E43564F583E064DC
:1055A000096008E55254C064C06045754C05E4F5D7
:1055B00050F54FF54E85434D7551058033754B328F
:1055C000754C2485434DE5652410F582E43564F57A
:1055D00083E0F54EE565241AF582E43564F583E051
:1055E000F54FE565241BF582E43564F583E0F5505D
:1055F00012519C22754B30754C0585434D85444EA8
:1056000085454F854650E542540F640460030258B7
:1056100076E54354C064C0600775510212519C2264
:10562000E543543F700EE544C39478500775510329
:1056300012519C22E4F5667554FF75678075F02C55
:10564000E567A42409F582E5F0344EAF82F5648F56
:1056500065F583E5822414F582E43583F583E0B5AE
:1056600043158F82E5822415F582E43564F583E0E5
:10567000654470030257C5E5546037E5652404F5B9
:1056800082E43564F583E0FFF552BF09088567665B
:10569000E4F554801DE5527019E565241EF582E499
:1056A0003564F583E0F553C39554500685676685E8
:1056B00053540567E5677085E566700302586F759A
:1056C000F02CA42409F582E5F0344EAF82F5648F06
:1056D00065F583E582240AF582E43583F583E4F0F9
:1056E000E565240BF582E43564F583E4F0E5652493
:1056F0000CF582E43564F583E4F0E565240DF5826C
:10570000E43564F583E4F0E565240EF582E4356460
:10571000F583E4F0E5652410F582E43564F58374DF
:1057200040F07F1A1291CBEF60047F0280027F006D
:10573000EF4448FFE5652411F582E43564F583EF15
:10574000F0E5652412F582E43564F583E4F0E5655F
:105750002413F582E43564F583E4F0E5652414F55B
:1057600082E43564F583E543F0E5652415F582E4CC
:105770003564F583E544F0E5652416F582E4356487
:10578000F583E4F0E5652417F582E43564F583E4F8
:10579000F0E5652418F582E43564F583E4F0E56509
:1057A0002419F582E43564F583E4F0E565241AF5FF
:1057B00082E43564F583E4F0E565241BF582E43585
:1057C00064F583E4F0E5652404F582E43564F5834B
:1057D000E0F56764097055788606E5652404F5826E
:1057E000E43564F5837404F0F567756991756A654D
:1057F000AE69AF6AAD65AC641250A1E56A2405F5E7
:1058000082E43569F583E0FEA3E0B56A1FEEB56971
:105810001B856A82856983E0FEA3E0FFE56A2405B3
:10582000F582E43569F583EEF0A3EFF0E5676401F6
:105830006015E5676402600FE56764036009AF65A2
:10584000AE647D04124E0E754B30754C27E5652411
:105850001EF582E43564F58374FFF07F4DE5652421
:105860000FFDE43564FC7B0712CFA612519C22E4A5
:10587000F55112519C22E543D3947F4007755104A2
:1058800012519C2275F02CE543A42409F582E5F021
:10589000344EAF82F5648F65F583E5822411F5827D
:1058A000E43583F583E054C0F567E54754C0656788
:1058B0007003025A518F82E582240AF582E435642E
:1058C000F583E4F0E565240BF582E43564F583E4C3
:1058D000F0E5652412F582E43564F583E4F0E565CE
:1058E000240DF582E43564F583E4F0E565240CF5D8
:1058F00082E43564F583E4F07887E630E1247F576D
:10590000120518E565240FF582E43564F583E0FFA0
:1059100012057AAF6712057A7F0D1205187F0A12F9
:105920000518AF65AE641250F8E567B4802378932C
:1059300016E5652404F582E43564F583E075F00727
:10594000A4246CF582E5F03491AF82F5698F6A800A
:1059500021788616E5652404F582E43564F583E054
:1059600075F007A42449F582E5F03491AF82F5691A
:105970008F6AE56A2405F582E43569F583E0FEA3C4
:10598000E0FFB5650BEEB56407AD6AAC69124FE395
:10599000E5652411F582E43564F583E0543FFFF0BA
:1059A000E54754C0FE4FF0E5652404F582E4356414
:1059B000F5837404F0EE64407040788606E5652453
:1059C00011F582E43564F583E054F3F07859E2B5DB
:1059D0004311E5652411F582E43564F583E0440C58
:1059E000F0800FE5652411F582E43564F583E04429
:1059F00008F0756991756A65801BE5652411F5826B
:105A0000E43564F583E054F3F04408F0756991756A
:105A10006A88789306AE69AF6AAD65AC641250A12E
:105A2000E56A2405F582E43569F583E0FEA3E0B577
:105A30006A1FEEB5691B856A82856983E0FEA3E073
:105A4000FFE56A2405F582E43569F583EEF0A3EFFE
:105A5000F0E54454C0248060558000E5652410F5CD
:105A600082E43564F583E030E71AE565240BF582BE
:105A7000E43564F583E4F0E5652412F582E43564E9
:105A8000F583E4F0E5652410F582E43564F583E000
:105A9000547FF04440F0754B30754C277F4DE565E1
:105AA000240FFDE43564FC7B0712CFA68064E56516
:105AB0002410F582E43564F583E030E61CE56524C6
:105AC0001AF582E43564F583E4F0E5652411F58286
:105AD000E43564F583E054CFF0E5652410F582E405
:105AE0003564F583E054BFF04480F0754B32754C5B
:105AF0002485434DF54EE565241AF582E43564F5B9
:105B000083E0F54FE565241BF582E43564F583E019
:105B1000F55012519C2275F02CE543A42409F5821E
:105B2000E5F0344EAF82F5648F65F583E582240E8F
:105B3000F582E43583F583E030E605754B36800366
:105B4000754B31754C0685434D7F4E75F02CE54302
:105B5000A4241FF582E5F0344EAD82FC7B0512CF04
:105B6000A612519CE5652404F582E43564F583E0D2
:105B700064016018AF65AE647D01124E0EE56524C8
:105B80000EF582E43564F583E04420F0E5652411E8
:105B9000F582E43564F583E054C0FFBF8010E5650D
:105BA0002408F582E43564F583740AF0800EE56517
:105BB0002408F582E43564F5837402F0E565242059
:105BC000F582E43564F583E04403F02275F02CE5BA
:105BD00043A42409F582E5F0344EAF82F5648F6565
:105BE000754B33754C0185434DF583E5822404F5EF
:105BF00082E43583F583E0B4090A754C04E4F5507A
:105C000012519C22E543D3947F401AE54454C0FFCF
:105C1000BF4008E54554C06440600A754C047550A7
:105C20000212519C22E565241AF582E43564F5835D
:105C3000E0F567E5652413F582E43564F583E0F566
:105C400066F568E54830E73AE5675401FFE54854F2
:105C5000016F700CE56654FEFEE54754FE6E60224F
:105C6000E566C313F566EF6003436680AF43AD6638
:105C7000129AF5E5652420F582E43564F583E04465
:105C800002F0E4F566E5652412F582E43564F583F7
:105C9000E065466003436601E545540CFFBF040F11
:105CA000E5475401FFE56854016F6003436601E571
:105CB00047541FFFE568541F6F6003436602E547C2
:105CC00054E0FFE56854E06F6003436604E5485420
:105CD00001FFE56754016F6003436604E548541E05
:105CE000FFE567541E6F6003436608E5652410F501
:105CF00082E43564F583E05408FFE54454086F609E
:105D000011D246E54530E10543661080074366043D
:105D10008002C246E5652420F582E43564F583E01F
:105D20004566F0E565240FFFE43564FE7D437B05A1
:105D300012CF96E54854BFFFE56754404FFFE56535
:105D4000241AF582E43564F583EFF012519C7885CE
:105D5000E630E013E54730E00EE5435401FFE54649
:105D600054FE4FFF120518E5652410F582E43564F2
:105D7000F583E030E014E565240AF582E43564F546
:105D800083E020E0057411F0D245E5652410F5822A
:105D9000E43564F583E020E014E565240AF582E447
:105DA0003564F583E030E0057412F0D245E56524F2
:105DB00016F582E43564F583E0540FC454F0FFE532
:105DC00065240CF582E43564F583E0540F2FF0E58B
:105DD000652404F582E43564F583E064016018AF5E
:105DE00065AE647D01124E0EE565240EF582E43544
:105DF00064F583E04420F0E54554C0FFBF8010E522
:105E0000652408F582E43564F583740AF0800EE5B4
:105E1000652408F582E43564F5837402F0AF65AE5D
:105E200064A2469247A24592481264FF2275F02C64
:105E3000E543A42409F582E5F0344EAF82F5648F82
:105E400065F583E5822404F582E43583F583E0B4C7
:105E50000910754B33754C0485434DE4F5501251D0
:105E60009C22E543D3947F4037E5652414F582E412
:105E70003564F583E0F54EE5652415F582E4356477
:105E8000F583E0F54FE545B54E06E546654F6010F4
:105E9000754B33754C0485434D75500112519C224E
:105EA000E5652413FFE43564FE7D447B0712CF963D
:105EB000E54A30E00C90918FE564F0A3E565F08051
:105EC0001390918FE0B5640CA3E0B56507E4909161
:105ED0008FF0A3F0E54A30E10C909195E564F0A3D2
:105EE000E565F08013909195E0B5640CA3E0B5658D
:105EF00007E4909195F0A3F0E54A30E20C90919B75
:105F0000E564F0A3E565F0801390919BE0B5640C27
:105F1000A3E0B56507E490919BF0A3F0E54A30E378
:105F20000C9091A1E564F0A3E565F080139091A138
:105F3000E0B5640CA3E0B56507E49091A1F0A3F08F
:105F4000754B33754C0185434D12519CE565240416
:105F5000F582E43564F583E064016018AF65AE64F2
:105F60007D01124E0EE565240EF582E43564F5835D
:105F7000E04420F0E5652420F582E43564F583E013
:105F80004403F0E5652408F582E43564F583740282
:105F9000F022302109E543641860030264FEE54302
:105FA000B4190040030264FE905FAFF82828730222
:105FB0005FFA0260170260360264FE0264FE02604D
:105FC0004F0260610264FE0264FE0264FE0264FE2F
:105FD0000260970264FE0264FE0264FE0264FE0236
:105FE00064FE0264FE0264FE0264FE0260B80261A6
:105FF0002B0264FE0264FE0261481299E912998A3A
:10600000C21EC214C209C20CC203754B35754C01C5
:10601000E4F54D12519C223014061299E912998A26
:10602000D21EC21478887441F2754B35754C0175D7
:106030004D0112519C221299F912999DD214C20C51
:10604000C203754B35754C01754D0212519C2230BF
:10605000290475320922C22BD226C202E47890F2BA
:1060600022854437E537B4551430290575320F8041
:1060700013D229E4F532786CE547F28007D22BD2AF
:10608000021299AD85453585463A754B35754C01FB
:10609000754D0512519C22754B35754C02754D0B93
:1060A000E4F54E789CE6FF30E003434E02EF30E12A
:1060B00003434E0412519C22301910754B35754C18
:1060C00002754D1585384E12519C227897E6601660
:1060D000E53865446010754B35754C02754D168575
:1060E000384E12519C22E54530E706789776FF80BE
:1060F00004E47897F6E54554077898F6700302644F
:10610000FED3940540030264FEE545131313541FA8
:1061100054077890F685443878A2A64608A6470822
:10612000A64808A64908A64AD21922E543B415187C
:10613000E544B53813754B35754C01754D17125143
:106140009CE4F5387897F622E542540F6407600323
:106150000264FEE54760030264FE780FE265446076
:10616000030264FEE5451460260460030264FE75C4
:106170004B35754C07754D18E4F54EF54FF550F558
:1061800051854852AF481291CB8F5312519C2275C2
:106190004B35754C07754D18E4F54E754F01F550AC
:1061A000F551854852E54890A60D9330E030AF4850
:1061B000AD491292438F5312928512519CE54620AD
:1061C000E00CE54890A60D9320E1030264FE754BB8
:1061D00035754C01754D0D12519CC2AF80FCAF4816
:1061E0001291CB8F5312519C2275F02CE543A424BD
:1061F00012F582E5F0344EF5837419F022756602CB
:1062000074412566F8E6FF604175F02CA42409F579
:1062100082E5F0344EAF82F5648F65F583E5822424
:1062200004F582E43583F583E0F5676401601BE5DE
:106230006764026015AE647D02124E0EE5652409A6
:10624000F582E43564F583740FF00566E566C39462
:106250000740AD2275660274412566F8E6FF60339B
:1062600074422566F8E6FE602A75F02CA42409F530
:1062700082E5F0344EAD82FC75F02CEFA4240FF5CE
:1062800082E5F0344EF583ECF0A3EDF00566E566AB
:10629000B409C4E54370030264FE74412566F8E660
:1062A000FF70030264FE75F02CE543A42409F58217
:1062B000E5F0344EAD82FC75F02CEFA4240FF5828E
:1062C000E5F0344EF583ECF0A3EDF0227566027430
:1062D000412566F8E6FF603275F02CA42409F582AA
:1062E000E5F0344EAF82F5648F65F583E5822411C5
:1062F000F582E43583F583E054FEF0E5652406F588
:1063000082E43564F583E4F0A3F00566E566B40A3B
:10631000BE2212B82B2212B83422E542540F640276
:106320007079754B3385434D85444EE54330E22803
:10633000754C03E544C3944040030264FE75F005C8
:10634000E544A42409F582E5F03490AF82F5698F25
:106350006AF583E0F54F803F754C0575F00BE54419
:10636000A42409F582E5F0347AAF82F5698F6AE5F5
:106370004330E00BE4256AF56A740B3569F56985ED
:106380006A82856983E0F54FA3E0F550856A8285CE
:106390006983A3A3E0F55112519C22E542540FFFFB
:1063A000BF031D53450F300610754B33754C0285E6
:1063B000434D85444E12519C2212BC8B1266BD2265
:1063C000E542540F6404705A754B3385434D854440
:1063D0004EE54330E2030264FE754C0575F00BE5B3
:1063E00044A42409F582E5F0347AAF82F5698F6A16
:1063F000E54330E00BE4256AF56A740B3569F5690D
:10640000856A82856983E0F54FAF458F50A3EFF031
:10641000AF468F51856A82856983A3A3EFF012513D
:106420009C227885E620E3030264FE7858E254C09B
:10643000FFF2E54254E0FE1313543F4FFFF2120502
:106440007A7F3A1205187858E22408F275660274C9
:10645000412566F8E6FF12057A7F201205180566C9
:10646000E566C3940A40E87F0D1205187F0A1205FD
:106470001822E54370030264FE754B38754C08F52D
:106480004D75F02CA42409F582E5F0344EAF82F569
:10649000648F65F56985656A756603E56A2406F5A6
:1064A00082E43569F583E0FEA3E08E69F56A6565EF
:1064B0007003EE6564602AE56A2411F582E43569AB
:1064C000F583E030E01BE56A240FF582E43569F5D9
:1064D00083E0FF744B2566F8A6070566E566B40AF7
:1064E000BAE566C3940A500B744B2566F8E4F605CA
:1064F0006680EE12519C2212B06B2212B0BA228E2C
:106500006B8F6C8F828E83E5822411F582E4358354
:10651000F583E020E0030266AD8F828E83E582245E
:1065200010F582E43583F583E0F56F856B6D856C3E
:106530006EE4F570E56E2406F582E4356DF583E0D2
:10654000FEA3E08E6DF56E4E70030266BCE56E65CF
:106550006C7004E56D656B70030266BCE56E24111A
:10656000F582E4356DF583E020E0030266BCE56E5C
:106570002410F582E4356DF583E054D1FFF0E56F2A
:10658000542E4FF0E56C240CF582E4356BF583E076
:10659000FFE56E240CF582E4356DF583EFF0E56CD4
:1065A0002417F582E4356BF583E0FFE56E2417F5DB
:1065B00082E4356DF583EFF030472DE56E2420F54C
:1065C00082E4356DF583C083C082E0FFE56E24115F
:1065D000F582E4356DF583E030E1047E1080027EC3
:1065E00004EF4ED082D083F0304826E56E2410F5BB
:1065F00082E4356DF583E06401F0E56E240AF582EE
:10660000E4356DF583E030E0057412F08003741119
:10661000F0E56C2412F582E4356BF583E0FFE56E5E
:106620002412F582E4356DF583EFF0E56E2420F554
:1066300082E4356DF583E04401F0E56E2411F582C6
:10664000E4356DF583E054C0FFBF8010E56E24088B
:10665000F582E4356DF583740AF0800EE56E24084A
:10666000F582E4356DF5837402F0E56E2404F5825D
:10667000E4356DF583E064016026E56E2420F58243
:10668000E4356DF583E06018AF6EAE6D7D01124E9E
:106690000EE56E240EF582E4356DF583E04420F0BE
:1066A0000570E570C39408500302653422E56C243C
:1066B00006F582E4356BF583E4F0A3F022E545545A
:1066C0000790A30593FCE54530E006ECC313FD807D
:1066D00004EC25E0FD786AE544F27842E543F230C7
:1066E000E249789CE620E1030267CDE544C394408B
:1066F00040030267CD75F005E544A42409F582E561
:10670000F03490FEAF827899A6447895A645E54589
:1067100030E30A8E83E04CFBF0EDF45BF0D223D241
:106720000678837404F27892760322789CE620E05F
:10673000030267CDC223D20678837404F2E4789210
:10674000F675F00BE544A42409F582E5F0347AFEF1
:10675000AF82E54530E004D2178002C217E5445409
:106760003F44807899F6E5441313543F54304480F5
:106770007895F6E54330E00BE42FFF740B3EFEE620
:106780004440F67895E64545F66470F6E54530E315
:10679000308F828E83A3A3E030E00E8F828E83E061
:1067A0004CF0E47836F208F2228F828E83E04CFBC4
:1067B0007850F2EDF45BF27836EEF208EFF2D22781
:1067C000228F828E83E0FBECF4FCEB5CF022C0E0D5
:1067D000C0F0C083C082C0D0C000C004C005C006E5
:1067E000C007C28C758CF5758A95D28C788406307A
:1067F00024030268BC300826E556602275DC46E4B6
:10680000F5DA20DCFDE5D9C3789B96400D78960635
:10681000E6C394044008C2088004E47896F6A228EF
:10682000B39228504575DC44E4F5DA30DC0890F08A
:1068300002E0422B80F5E5D9D3788C96401C786D28
:10684000E2FF7839E204F2C39F40715357F090F0B1
:106850000DE557F0D209E4F28062789EE66402709A
:106860005B7839E2605614F2805275DC45E4F5DA63
:1068700030DC0890F002E0422B80F5E5D9D3788F28
:1068800096402C786FE2FF783BE204F2C39F402CE5
:10689000E55754F7F55790F00DF0300F0A5357F8BD
:1068A000E557F0D2098002D20CE4783BF2800D78F3
:1068B0009EE6B40207783BE2600214F2A201B392B2
:1068C000015070200D03026CD6152AE52A7020783D
:1068D000A0E6FF441890F00CF0EF4408F0EF4410ED
:1068E000F0EFF0752A2275361454C0F6026CD6E526
:1068F0002AB4111778A0E6FF441C90F00CF0EF4486
:106900000CF0EF4410F0EFF0026CD6A836E2FFC4B2
:10691000540FFE78A0E6FD4430FC4E90F00CF0EDF4
:106920004420FD4EF0EF540FFF4CF0ED4FF00536D4
:10693000026CD6302403026CD6789EE6FF4440F504
:10694000DCE4F5DA90F002E0422BEFB408004003FB
:10695000026CD290695AF82828730269720269CCD5
:10696000026A26026A9F026B1B026B93026C0B0287
:106970006C6DE52B30E0177845E2C394105004E2CB
:106980002408F27845E230E712748FF2800D7845E2
:10699000E2600814F2E2B48002E4F2E52B30E4177E
:1069A0007849E2C394105004E22408F27849E230B6
:1069B000E713748FF2800E7849E26009E214F2E284
:1069C000B48002E4F2789E7601026CD6E52B30E1C9
:1069D000177846E2C394105004E22408F27846E2A5
:1069E00030E712748FF2800D7846E2600814F2E20C
:1069F000B48002E4F2E52B30E517784AE2C3941044
:106A00005004E22408F2784AE230E713748FF280EF
:106A10000E784AE26009E214F2E2B48002E4F2780D
:106A20009E7602026CD6E52B30E2177847E2C394DB
:106A3000105004E22408F27847E230E713748FF232
:106A4000800E7847E26009E214F2E2B48002E4F2D8
:106A5000E52B30E617784BE2C394105004E224088B
:106A6000F2784BE230E713748FF2800E784BE260DD
:106A700009E214F2E2B48002E4F220DCFDAFDAEFC6
:106A800075F004A4E5F0FDAFD9EF75F004A4FFE5BF
:106A9000F0788AF6ED4F08F6789E7603026CD6E51C
:106AA0002B30E3177848E2C394105004E22408F234
:106AB0007848E230E713748FF2800E7848E260097C
:106AC000E214F2E2B48002E4F2E52B30E717784CEE
:106AD000E2C394105004E22408F2784CE230E71349
:106AE000748FF2800E784CE26009E214F2E2B48016
:106AF00002E4F2E4F52B20DCFDAFDAEF75F004A43C
:106B0000E5F0FDAFD9EF75F004A4FFE5F0788DF660
:106B1000ED4F08F6789E7604026CD6E52B30E01730
:106B20007845E2C394105004E22408F27845E2303C
:106B3000E712748FF2800D7845E2600814F2E2B437
:106B40008002E4F2E52B30E4177849E2C394105058
:106B500004E22408F27849E230E713748FF2800EE1
:106B60007849E26009E214F2E2B48002E4F220DC47
:106B7000FDAFDAEF75F004A4E5F0FDAFD9EF75F0E5
:106B800004A4FFE5F0787FF6ED4F08F6789E7605D1
:106B9000026CD6E52B30E1177846E2C3941050041E
:106BA000E22408F27846E230E712748FF2800D7822
:106BB00046E2600814F2E2B48002E4F2E52B30E52C
:106BC00017784AE2C394105004E22408F2784AE2AB
:106BD00030E713748FF2800E784AE26009E214F213
:106BE000E2B48002E4F220DCFDAFDAEF75F004A439
:106BF000E5F0FDAFD9EF75F004A4FFE5F07881F67C
:106C0000ED4F08F6789E7606026CD6E52B30E2173B
:106C10007847E2C394105004E22408F27847E23047
:106C2000E713748FF2800E7847E26009E214F2E213
:106C3000B48002E4F2E52B30E617784BE2C39410FF
:106C40005004E22408F2784BE230E713748FF280AC
:106C50000E784BE26009E214F2E2B48002E4F22022
:106C6000DCFD785AE5D9F2789E76078069E52B300D
:106C7000E3177848E2C394105004E22408F27848FD
:106C8000E230E713748FF2800E7848E26009E21474
:106C9000F2E2B48002E4F2E52B30E717784CE2C36D
:106CA00094105004E22408F2784CE230E713748F19
:106CB000F2800E784CE26009E214F2E2B48002E461
:106CC000F2E4F52B20DCFD785EE5D9F2E4789EF65F
:106CD0008004E4789EF6D22530071F780B08E22462
:106CE00001FFF218E23400FEF2C3EF9460EE940468
:106CF0005008C2AFD2AED2BED2AFD007D006D005B8
:106D0000D004D000D0D0D082D083D0F0D0E0328B6D
:106D10007B8A7C897DAE02AF01EF4E70087E9F7F3B
:106D20007C1203CF22E4F57EE57E75F02CA42409C5
:106D3000F9744E35F0FAE57B857C83857D826402AB
:106D40007008E965827003EA658370127E9F7F8216
:106D50001203CFAF7E12057A7F2012051822057E1E
:106D6000E57E70C4F57EE57E75F007A42449F974CC
:106D70009135F0FAE57B857C83857D82640270081D
:106D8000E965827003EA658370157E9F7F85120333
:106D9000CFE57E4430FF1205187F2012051822052A
:106DA0007EE57EC3940540BEE4F57EE57E75F00782
:106DB000A4246CF9749135F0FAE57B857C83857D9C
:106DC0008264027008E965827003EA658370157E4B
:106DD0009F7F891203CFE57E4430FF1205187F2084
:106DE00012051822057EE57EC3940540BE7F3F1242
:106DF0000518E57CFF12057AAF7DE57D12057A2244
:106E0000E4F562F563C243C244783AE2FF54037882
:106E10009CF6EF30E402D243789CE6540324FFB39F
:106E200092217F161291CBBF01097F16E4FD1292C9
:106E300043D2437F1A1291CB8F5BC0077F1B129105
:106E4000CBAE07D007EE6F601AE55B600C7F1B7D51
:106E500001129243436201800A7F1BE4FD129243B8
:106E60004363019091C0E0FF540B64087028EF3039
:106E7000E2134362017F1A7D011292437F1B7D0161
:106E800012924380114363017F1AE4FD1292437F03
:106E90001BE4FD129243E49091C0F030430B755E09
:106EA00004755F0475600480157F501291CB8F5E6E
:106EB0007F511291CB8F5F7F521291CB8F601292D4
:106EC00085E4F55B75F007E55BA42449F582E5F000
:106ED0003491F583AF82FEF0A3EFF075F007E55B28
:106EE000A4244BF582E5F03491F583EEF0A3EFF0A6
:106EF00075F007E55BA4244EF582E5F03491F58347
:106F0000EEF0A3EFF075F007E55BA4244DF582E504
:106F1000F03491F58374AAF075F007E55BA4246C56
:106F2000F582E5F03491F583AF82FEF0A3EFF075C2
:106F3000F007E55BA4246EF582E5F03491F583EE6D
:106F4000F0A3EFF075F007E55BA42471F582E5F09E
:106F50003491F583EEF0A3EFF075F007E55BA42420
:106F600070F582E5F03491F58374AAF0055BE55B7A
:106F700064056003026EC4302103D21522D204D20C
:106F8000AED2BE789CE630E007780E7440F2800501
:106F9000780E7480F2783D7480F2E4F55B7886F6C2
:106FA0007893F63044077E9F7F8D1203CF204403F1
:106FB0000271A075F02CE55BA424DDF582E5F034C8
:106FC0004DAF82F5598F5AE55B14FF12057A7F2089
:106FD000120518E55A2404F582E43559F583E0FFDB
:106FE00012057A7F20120518E55A2405F582E4354A
:106FF00059F583E0FF12057A7F20120518E55A241F
:1070000008F582E43559F583E0FF12057A7F2012F6
:107010000518E55A2409F582E43559F583E0FF1295
:10702000057A7F20120518E55A240AF582E43559BD
:10703000F583E0FF12057A7F20120518E55A240B2C
:10704000F582E43559F583E0FF12057A7F201205B9
:1070500018E55A240CF582E43559F583E0FF120552
:107060007A7F20120518E55A240DF582E43559F58A
:1070700083E0FF12057A7F20120518E55A240EF5E9
:1070800082E43559F583E0FF12057A7F2012051856
:10709000E55A240FF582E43559F583E0FF12057AAD
:1070A0007F20120518E55A2411F582E43559F5833D
:1070B000E0FF12057A7F20120518E55A2411F582A7
:1070C000E43559F583E0FF12057A7F20120518E5B3
:1070D0005A2412F582E43559F583E0FF12057A7FD0
:1070E00020120518E55A2413F582E43559F583E09A
:1070F000FF12057A7F20120518E55A2414F582E460
:107100003559F583E0FF12057AE55A2415F582E436
:107110003559F583E0FF12057A7F20120518E55AEC
:107120002416F582E43559F583E0FF12057A7F20B5
:10713000120518E55A2417F582E43559F583E0FF66
:1071400012057A7F20120518E55A2418F582E435D5
:1071500059F583E0FF12057A7F20120518E55A24BD
:1071600019F582E43559F583E0FF12057A7F201284
:107170000518E55A241AF582E43559F583E0FF1223
:10718000057A7F20120518E55A241BF582E435594B
:10719000F583E0FF12057A7F0A120518D2AED2BE3F
:1071A00075F02CE55BA42409F582E5F0344EAF823E
:1071B000F5598F5AF583E582240FF582E43583F57E
:1071C00083E55BF0855A82855983E4F0A3F0855A04
:1071D00082855983A3A3F0A3F0E55A2411F582E434
:1071E0003559F583E054CFF030220EE55A2411F5DD
:1071F00082E43559F5837408F0E55A2405F582E4F4
:107200003559F58374A5F0E55A240EF582E4355915
:10721000F583E0549FF0E55A2411F582E43559F5E1
:1072200083E0F55D54C0FF6440702F789CE6540302
:1072300064026003027303535D3F435D80E55A249B
:1072400014F582E43559F583E4F0E55A2404F58217
:10725000E43559F583E4F0027303EF6480704778F6
:107260009CE6FF30E10AE55BD394515003027303BF
:10727000EF20E003027303535D33435D48E55A2476
:1072800014F582E43559F583E4F0E55A2415F582C6
:10729000E43559F583E4F0E55A2404F582E43559E0
:1072A000F583E4F0805D789CE6FF5403FEBE022285
:1072B000535D3F435D80E55A2414F582E43559F56A
:1072C00083E4F0E55A2404F582E43559F583E4F0CB
:1072D0008031EF30E02D535D33435D48E55A24148F
:1072E000F582E43559F583E4F0E55A2415F582E496
:1072F0003559F583E4F0E55A2404F582E43559F56F
:1073000083E4F0E55A2411F582E43559F583E55D0F
:10731000F0E55D54C06440600302760A789CE62084
:10732000E00302760AE55A2410F582E43559F58324
:10733000E0547FF04440F0E56230E00FE55A24115C
:10734000F582E43559F583E04402F0E56330E00F5F
:10735000E55A2411F582E43559F583E054FDF0E552
:107360005A2410F582E43559F583E0FF30E02244D9
:1073700010F0E55A240AF582E43559F5837403F0D8
:10738000E55A240EF582E43559F583E04402F08095
:107390002FEF20E02BE55A2410F582E43559F583D0
:1073A000EF54EFF0E55A240AF582E43559F583E409
:1073B000F0E55A240EF582E43559F583E054FDF0EA
:1073C000E55B7011E55A2404F582E43559F58374C0
:1073D00009F002776C783DE2FFE55BC39F40030252
:1073E00074BB788606E55A2404F582E43559F583A2
:1073F000E0F5616069E55E24FD60151460171460B6
:107400001914602E14604224057053756103804E78
:107410007561048049E4F5618044E55A2412F582DF
:10742000E43559F583E070047F0480027F038F61A7
:10743000802CE55A2412F582E43559F583E0700377
:10744000FF80027F048F618015E55A2412F582E4E3
:107450003559F583E07003FF80027F038F61E5619A
:10746000D39405400302776C75F007E561A42449C5
:10747000F582E5F03491AF82FEAD5AAC591250A1BD
:1074800075F007E561A42449F582E5F03491F583B0
:10749000E0FEA3E0FF75F007E561A4244EF582E568
:1074A000F03491F583EEF0A3EFF0E55A2404F58271
:1074B000E43559F583E561F002776CE55BD3947FA1
:1074C000500302776CE55A2414F582E43559F583AC
:1074D000E054C064C07029E55A2404F582E43559AB
:1074E000F583E0FF64096018E55FB4080EE55A24EF
:1074F00012F582E43559F583E06005E55FB4092BA8
:10750000E55A2404F582E43559F5837409F0E55A07
:107510002414F582E43559F583E4F0E55A2415F591
:1075200082E43559F583E4F002776C8F61EF60698E
:10753000E55F24FD601514601714601914602E14A3
:10754000604224057053756103804E756104804963
:10755000E4F5618044E55A2412F582E43559F58357
:10756000E070047F0480027F038F61802CE55A2441
:1075700012F582E43559F583E07003FF80027F0441
:107580008F618015E55A2412F582E43559F583E0C0
:107590007003FF80027F038F61E561C39405505043
:1075A00075F007E561A42449F582E5F03491AF82D6
:1075B000FEAD5AAC591250A175F007E561A42449FB
:1075C000F582E5F03491F583E0FEA3E0FF75F00766
:1075D000E561A4244EF582E5F03491F583EEF0A345
:1075E000EFF0E55A2404F582E43559F583E561F0BE
:1075F000788606E55A241EF582E43559F583E07055
:107600000302776CE014F002776CE55D54C064808F
:10761000600302776C789CE620E10302776CE55BFF
:10762000C39451400302776CD20A789306E55A243A
:1076300010F582E43559F583E0547FF030E02EE513
:107640005A2410F582E43559F583E04410F0E55AE8
:10765000240AF582E43559F5837403F0E55A240EC3
:10766000F582E43559F583E04402F0802FE55A2491
:1076700010F582E43559F583E0FF20E01F54EFF068
:10768000E55A240AF582E43559F583E4F0E55A24F5
:107690000EF582E43559F583E054FDF0E55A2404F3
:1076A000F582E43559F583E0F5616069E56024FD14
:1076B000601514601714601914602E1460422405BC
:1076C0007053756103804E7561048049E4F56180F3
:1076D00044E55A2412F582E43559F583E070047FBD
:1076E0000480027F038F61802CE55A2412F582E426
:1076F0003559F583E07003FF80027F048F618015A8
:10770000E55A2412F582E43559F583E07003FF80D1
:10771000027F038F61E561C39405505075F007E562
:1077200061A4246CF582E5F03491AF82FEAD5AACD1
:10773000591250A175F007E561A4246CF582E5F0BB
:107740003491F583E0FEA3E0FF75F007E561A42422
:1077500071F582E5F03491F583EEF0A3EFF0E55A90
:107760002404F582E43559F583E561F0AF5B055BF0
:10777000EFC394FF5003026FAD30441C7E9F7F9C8B
:107780001203CF7886E6FF12057A7E9F7FA7120349
:10779000CF7893E6FF12057A22D2077885E620E3B8
:1077A000030278487F6C1205187F621205187F610A
:1077B00012051878B4E6FF12057A78B5E6FF1205CF
:1077C0007A7F641205187F651205187F6612051806
:1077D00078B2E6FF12057A78B2E6FE08E6FF1205F7
:1077E0007A7F701205187F701205187F70120518C5
:1077F00078B0E6FF12057A78B0E6FE08E6FF1205DB
:107800007A7F6C1205187F651205187F6E120518B5
:1078100078B0E6FE08E6FFC3901C1AE09F901C19A2
:10782000E09EFF3395E012057A78B0E6FE08E6FFA9
:10783000901C19E0FCA3E0FDC39FFF12057A7F0DA9
:107840001205187F0A120518901C19E0FEA3E078B3
:10785000B166700318E66E7003027971E4F559E5BC
:107860005925E0246DF582E4341CF583E0FEA3E0A5
:10787000D378B396EE18964024E55925E0246EF5AA
:1078800082E4341CF58378B4E6FE08E6FFC3E09F8B
:10789000F00582D5820215831582E09EF00559E538
:1078A00059B414BB78AB761C0876A1E4FFFEC3EF95
:1078B0009484EE9403400302793778ABE6FC08E643
:1078C000F5828C83E0FDA3E07894CDF208EDF2E23E
:1078D000700218E2604F7894E230E708E2547FF2D9
:1078E000D2398002C23978B2E6FC08E6FDD3789539
:1078F000E29D18E29C402E78B4E6FC08E6FDC378D1
:1079000095E29DF218E29CF2303904E24480F2786C
:1079100094E2FC08E2FD78ABE6FA08E6F5828A8399
:10792000ECF0A3EDF00FBF00010E78AC740226F668
:1079300018E436F60278AE78B0E6FE08E6FFC390AB
:107940001C1AE09FFD901C19E09EFCC004C005AA13
:1079500006A9077B02C003C00278B2E6FE08E6AAC9
:1079600006F8AC02AD03D002D003D007D00612D582
:10797000A978B4E6FE08E6FFC3901C1AE09FFD90CC
:107980001C19E09EFCF0A3EDF0C3901C1CE09FF0DE
:10799000901C1BE09EF08D828C83E4F0C239C235CE
:1079A000C20778847601223002097844E260041428
:1079B000F2705EE47891F6788DE6FE08E6FF7D12BF
:1079C0007B0212992E7C007D2112D3637838E2FD70
:1079D00012D3777D021285EE78187456F2781974F6
:1079E00020F278917606788AE6FE08E6FF7D107B25
:1079F0000212992E7C007D2112D3637835E2FD12AC
:107A0000D3777D021285EE781E7456F2781F7420AB
:107A1000F23002087844E26003027B9D30160E7B50
:107A2000057A9F79B27D101285AE027AE5300C0E90
:107A30007B057A9F79B97D101285AE027AE530090F
:107A40000E7B057A9F79C07D101285AE027AE530F3
:107A5000140E7B057A9F79C77D101285AE027AE5F8
:107A6000301E0D7B057A9F79CE7D101285AE807514
:107A700030150D7B057A9F79D57D101285AE806516
:107A8000789176107881E6FE08E6FF7D8C7B021205
:107A9000992E8E648F657855E2FF3395E0FE783F2E
:107AA000E22FFFE43EFEC3E5659FF565E5649EF5C4
:107AB00064D3E56594FFE564947F40067E007F0013
:107AC0008004AE64AF657892E2FD7C0012D36378E7
:107AD00041E2FD12D3777D011285EE78287441F2E0
:107AE00078297420F230090E7B057A9F79C07D16C3
:107AF0001285AE027B9D30030E7B057A9F79DC7D7B
:107B0000161285AE027B9D30140E7B057A9F79C7D5
:107B10007D161285AE027B9D301E0D7B057A9F7906
:107B2000CE7D161285AE807530150D7B057A9F7956
:107B3000E37D161285AE806578917616787FE6FE35
:107B400008E6FF7D8A7B0212992E8E648F65785439
:107B5000E2FF3395E0FE783EE22FFFE43EFEC3E510
:107B6000659FF565E5649EF564D3E56594FFE5647E
:107B7000947F40067E007F008004AE64AF657891FC
:107B8000E2FD7C0012D3637840E2FD12D3777D01E1
:107B90001285EE782E7441F2782F7420F230210392
:107BA000027C697887E6B4801678207454F27821D4
:107BB0007445F278227453F2782304F2027C6378DD
:107BC0001AE6FD706B781CE6FF700A7821742EF2BD
:107BD0007822F2804BEFC3940350117821742EF277
:107BE000EF25E025E024307822F28034EF75F06450
:107BF000A4E5F0F566C394644003756663E56675B5
:107C0000F00A84FF700778217420F28006EF243098
:107C10007821F2E56675F00A84E5F024307822F2E6
:107C200078207443F278237425F2E4781CF68033CC
:107C300078207443F278217445F27822743AF2ED98
:107C4000540724307823F27885E630E5167F431216
:107C500005187F45120518781AE6FF12057A7F0A83
:107C6000120518E4781AF6802378207453F27821EC
:107C7000744CF2780FE2FF75F00A8424307822F217
:107C8000EF75F00A84E5F024307823F290F002E0FA
:107C9000F566C4540F9005BD937832F2E566540F33
:107CA000937833F222E4F55B7445255BF8E220E437
:107CB00003027D67748FF2E55B75F006A4248FF5EF
:107CC00082E43491AF82F5598F5AF583A3A3E0245F
:107CD000FE605814605A14605C14605924046003F8
:107CE000027D67855A82855983E0FEA3E0FF4E60DE
:107CF00076855A82855983A3A3A3E0FDEF241CF562
:107D000082E43EF583EDF0E55A2404F582E435592A
:107D1000F583E0FDEF241DF582E43EF583EDF0E50B
:107D20005B90A71B93FD1232AA803C127E0B80371A
:107D3000127E188032E55A2405F582E43559F58320
:107D4000E0FF601375F00A84F543EF75F00A84E5EF
:107D5000F014F54412B834855A82855983A3A3E000
:107D600064057003027CE3055BE55BC39408500384
:107D7000027CA822C245204435E4F564E56475F030
:107D800006A42491F582E43491F583E0B4060E78DC
:107D900089E2FFE56490A30593FEEF4EF20564E5EA
:107DA00064B408D87889E26003D38001C322E4F583
:107DB0006474452564F8E254906011E56490A3056D
:107DC00093FF7889E25F6004D24580070564E5642B
:107DD000B408DE7890E2701630450C7B057A9F7906
:107DE000EAFD1285AE802278907401F2801B7890B3
:107DF000E2B4011520450D7B057AA0790BE4FD1254
:107E000085AE800578907402F2C322D21E78887401
:107E100041F2C2451297DC22D214C20CC20312995D
:107E2000F912999DC2451297DC22D224EF4440F505
:107E3000DCE4F5DA20DCFD204507AFD9C2247E0062
:107E400022AFDAEF75F004A4E5F0FDAFD9EF75F0DD
:107E500004A4FFAEF0E5F0ED4FFFC22422AC077999
:107E600010E4FBFAAF04A2449245127E2AEF2BFBEA
:107E7000EE3AFAD9EFEAC4F854F0C868FEEBC454FD
:107E80000F48FF22E4F5597557F090F00D74F0F0AB
:107E90001284FA90F001E020E003028211C2AFD216
:107EA000AED2BED2AF90F000E0FFC4540F9005BD3B
:107EB000937824F290F000E0540F9005BD9378255C
:107EC000F290F001E0FFC4540F9005BD937827F2C3
:107ED00090F001E0540F9005BD937828F290F002E5
:107EE000E0FFC4540F9005BD93782AF290F002E0B1
:107EF000540F9005BD93782BF2E55924FD601514BD
:107F0000601714601914601B14601D2405701E7521
:107F10005C15801E755C198019755C1D8014755C7C
:107F200021800F755C2D800A755C318005755901C3
:107F3000802DAF59D244127E5D8E5A8F5BE55A90E8
:107F400005BD93AE5C055CA806F2AF5BEFC4540FB1
:107F500093AD5C055CA805F2EF540F93A85CF205A5
:107F60005990F000E020E003027E93C2AFD2AED27F
:107F7000BED2AFA3E0F55E5442FFBF020A1299BD24
:107F80007FA87E611203C0E55E5484FFBF040A121D
:107F900099C87FA87E611203C043570390F00DE596
:107FA00057F0C2AFD2AED2BED2AF7F507EC3120363
:107FB000C07F04D244127E5D783EEFF27F05D2444A
:107FC000127E5D783FEFF218E2D39414500708E276
:107FD000D3941440111284FA7B057AA0792CE4FD25
:107FE0001285AE027F6112998A90F000E020E003D2
:107FF000027F617F04C244127E5DD3EF9432EE941F
:108000000050030280F17F02D244127E5D8E5A8FAF
:108010005BE47891F6FC7D2112D3637D6612D37701
:108020007D021285EE78187455F2AE5AAF5B7C0073
:108030007D2812D3637DC612D3777891EFF27891C1
:1080400076067E007D011285EE781E7443F27F0471
:10805000D244127E5D8E5A8F5BEF7803CEC313CE6F
:1080600013D8F9FF7840F27891760C7E00E4FD1287
:1080700085EE78237448F278917610783EE2FF7EA0
:1080800000E4FD1285EE7827744CF278917615782D
:108090003EE2FFC3E55B9FFFE55A9400FED3EF94F9
:1080A000FFEE947F400A7C007D00AE04AF058000A7
:1080B0007891E2FD7C0012D3637840E2FD12D37721
:1080C0007D011285EE782D7441F27891761BAF5BBD
:1080D000AE5A7D011285EE78337449F2E4FF7840A0
:1080E000E2FD1292437F027891E2FD1292430281F7
:1080F000FC7F05C244127E5DD3EF9432EE940050B3
:10810000030281EE7F03D244127E5D8E5A8F5BE4C0
:108110007891F6FC7D2112D3637D6612D3777D02C0
:108120001285EE78187455F2AE5AAF5B7C007D284C
:1081300012D3637DC212D3777892EFF278917606EC
:108140007E007D011285EE781E7443F27F05D244D5
:10815000127E5D8E5A8F5BEF7803CEC313CE13D899
:10816000F9FF7841F27891760C7E00E4FD1285EEFD
:1081700078237448F278917610783FE2FF7E00E42D
:10818000FD1285EE7827744CF278917615783FE2EF
:10819000FFC3E55B9FFFE55A9400FED3EF94FFEE2B
:1081A000947F400A7C007D00AE04AF058000789289
:1081B000E2FD7C0012D3637841E2FD12D3777D01AA
:1081C0001285EE782D7441F27891761BAF5BAE5A32
:1081D0007D011285EE78337449F27F017841E2FD2A
:1081E0001292437F037892E2FD129243800E128432
:1081F000FA7B057AA07944E4FD1285AEC2AFD2AE17
:10820000D2BED2AF7FA87E611203C01284FA027F71
:10821000E9E4F55790F00DF0754B35754C01754D4F
:108220000D12519C12519C12519CD2AED2BEC2AFC3
:1082300080FC22E4F559F55AD2437EA77F2312032E
:10824000CF7B057AA7792D7D101285AEE4F55D7E92
:10825000A77F2D1203CFAF5D12057A7F0A12051892
:1082600090F008E55DF0FF7401A807088002C333B1
:10827000D8FCF55FE4F559F55AF55BF55CD2AED262
:10828000BEB290E4F55E055AE55AAE597002055942
:1082900014F5828E83E55FF0055EE55EB480E70548
:1082A0005CE55C7002055BE4B55CD2E55BB401CDD6
:1082B000055DE55DC3940840967B057AA779387D16
:1082C000101285AEE4F55D7EA77F381203CFAF5D57
:1082D00012057A7F0A12051890F008E55DF0FF7428
:1082E00001A807088002C333D8FCF55FE4F559F50F
:1082F0005AF55BF55CD2AED2BEB291E4F55E855A1A
:1083000082855983E0655F60467EA77F431203CF75
:10831000AF5D12057A7F20120518E55CAE5B780729
:10832000C333CE33CED8F97C00255EEC3EFF120578
:108330007AE55CAE5B7807C333CE33CED8F97C00E8
:10834000255EFFEC3E12057A7F0A120518C243052E
:108350005AE55AAE597002055914F5828E83E4F03D
:10836000055EE55EC394804095055CE55C700205A2
:108370005BC3E55B940150030282F5055DE55DC3D7
:10838000940850030282C790F008E4F03043137E53
:10839000A77F501203CF7B057AA779507D101285F5
:1083A000AE227EA77F5B1203CF7B057AA7795B7D28
:1083B000101285AE22E4F55B7F171291CBBF6F09D7
:1083C0007F17E4FD1292438027783AE2F46021E5BA
:1083D0005BC39418501AE55B90A08C93FF74002542
:1083E0005BF582E43400F583E0B50704055B80DFCC
:1083F000E55BC39418400302847BC2AFD2AED2BE09
:108400007EF07F007D007B027A00790012D40E7E20
:10841000037FFF7D007B027AFC790012D40E780086
:108420007C007D027B057AA0798C7E007F1812D3B8
:1084300016D2AED2BED2AFD2227F1A7D01129243A3
:108440007F1BE4FD1292437EA07F541203CF12845F
:10845000FA7B057AA07964E4FD1285AEE4F55BC28F
:10846000AFD2AED2BED2AF7FA87E611203C0055B91
:10847000E55BC3940740E8C2AF80FC22E4F559F500
:108480005AFDFCFE7F80855A82855983E493FA74F5
:1084900001932DFDEA3CFC7402255AF55AE4355946
:1084A000F559DFE27F80855A82855983E493FA7417
:1084B00001932DFDEA3CFC7402255AF55AE4355926
:1084C000F559DFE2D2AED2BE0EBE80B87557F0EDE0
:1084D0004C602690F00DE557F06357F0E4FCFDC3C7
:1084E000EC948050EAEFF5F0A4FF7C007D01D2AE61
:1084F000D2BE0DBD00010C80E6227E007F207D20D3
:108500007B037AFC791412D40EE47891F62212845B
:10851000FA7F887E131203C090F00C7413F074037A
:10852000F07FE27E041203C090F00C7413F0740329
:10853000F07F327E001203C090F00C7413F07403CD
:10854000F07F0C7E001203C090F00C7412F07402E5
:10855000F07F0C7E001203C090F00C7412F07402D5
:10856000F07418F07408F07F0C7E001203C090F0D5
:108570000C7410F0E4F0741CF0740CF0FF7E001228
:1085800003C090F00C7410F0E4F07411F07401F07A
:108590007FF4FE1203C090F00C7410F0E4F0741637
:1085A000F07406F07F0C7E001203C0D20D228B67A0
:1085B0008A688969EDF4600AEDC3942050047891CB
:1085C000A605AB67AA68A96912D348FF601F789116
:1085D000E6FEC39420501674142EF8EFF2740125B1
:1085E00069F569E43568F56878910680D5228D676C
:1085F000AB07AA06E56760047F0180027F007891DF
:10860000E624022FF568C3648094A040030286A983
:10861000E56804F6AE02AF037C007D0A12D377ED65
:108620002430FFAE68156874142EF8EFF2AE02AF76
:10863000037C007D0A12D377AA06AB07E567B40274
:108640000BAF68156874142FF8742EF2AE02AF03E6
:108650007C007D0A12D377ED2430FFAE6815687474
:10866000142EF8EFF2AE02AF037C007D0A12D3772E
:10867000AA06AB07E567B4010BAF68156874142F41
:10868000F8742EF2AE02AF037C007D0A12D377EDB0
:108690002430FF74142568F8EFF2AE02AF037C00BB
:1086A0007D0A12D377AA06AB0722EF240FF582E4E6
:1086B0003EF583E0FCC39480501A78787403F27816
:1086C00034E27879F2787AECF2787BEDF2EC6D783E
:1086D0007CF2803578787404F27834E27879F2EFBD
:1086E0002414F582E43EF583E0787AF2EF2415F560
:1086F00082E43EF583E0787BF2787CEDF2787BE2F1
:10870000FF787AE26F6D787DF21287A3228E6B8FED
:108710006C8F828E83E582240FF582E43583F583A6
:10872000E0FFC39480501F78787404F27834E278C4
:1087300079F2787AEFF2787BEDF2787CEBF2EF6DFC
:108740006B787DF2803E78787405F27834E278793F
:10875000F2E56C2414F582E4356BF583E0787AF267
:10876000E56C2415F582E4356BF583E0787BF278CF
:108770007CEDF2787DEBF2787BE2FF787AE26F6D48
:108780006B787EF21287A32278787403F27834E251
:108790007879F2787AEFF2787BEDF26F787CF212EA
:1087A00087A3227887E630E003D38001C392457522
:1087B0006F78AF6F056FA807E2F5717003028893B9
:1087C000D394064003028893203F13756DEC756EB9
:1087D00000E490EEE0F0A3F0A3F0A3F08011756D3B
:1087E000ED756E00E490EEE4F0A3F0A3F0A3F0E5E5
:1087F0007175F012A42404FF056EE56EAC6D700275
:10880000056D14F5828C83EFF0AF6F056FA807E25A
:10881000FF056EE56EAC6D7002056D14F5828C83FC
:10882000EFF03045057F441205181571E4F570E549
:1088300070C39571503DAF6F056FA807E2F57230B8
:108840004504FF12057AE570C394025013203F09D6
:10885000742D2570F8A6728007742F2570F8A67203
:10886000AF6EAE6DAD72C2461288948E6D8F6E057E
:108870007080BC30450CA86FE2FF12057A7F0A12A7
:108880000518AF6EAE6DA86FE2FDD246128894D285
:108890003DB23F227C803041328F828E83E519F0D9
:1088A0000FBF00010E8F828E83E518F00FBF00010D
:1088B0000E8F828E837425F00FBF00010E8F828E83
:1088C000837401F00FBF00010E80308F828E83749D
:1088D00025F00FBF00010E8F828E837401F00FBF51
:1088E00000010E8F828E83E519F00FBF00010E8FFD
:1088F000828E83E518F00FBF00010EEC7003028931
:10890000A05D60308F828E83E533F00FBF00010ED3
:108910008F828E83E4F00FBF00010E8F828E83E57D
:1089200033F00FBF00010E8F828E83E4F00FBF0083
:10893000010E80653041328F828E83E519F00FBFC2
:1089400000010E8F828E83E518F00FBF00010E8F9D
:10895000828E837425F00FBF00010E8F828E837488
:1089600001F00FBF00010E80308F828E837425F0DE
:108970000FBF00010E8F828E837401F00FBF0001C4
:108980000E8F828E83E519F00FBF00010E8F828E4D
:1089900083E518F00FBF00010EECC313FC0288FB47
:1089A000204603028A398F828E83E533F00FBF00A1
:1089B000010E8F828E83E4F00FBF00010E8F828E36
:1089C00083E533F00FBF00010E8F828E83E4F00F3A
:1089D000BF00010E3041328F828E83E519F00FBF48
:1089E00000010E8F828E83E518F00FBF00010E8FFD
:1089F000828E837425F00FBF00010E8F828E8374E8
:108A000001F00FBF00010E80308F828E837425F03D
:108A10000FBF00010E8F828E837401F00FBF000123
:108A20000E8F828E83E519F00FBF00010E8F828EAC
:108A300083E518F00FBF00010E2278787403F278F6
:108A40004FE27879F2787AEFF2787BEDF26F787C0A
:108A5000F2128A762278787404F2784FE27879F20A
:108A6000787AEFF2787BEDF2787CEBF2EF6D6B7851
:108A70007DF2128A76227887E630E003D38001C344
:108A80009244756678AF660566A807E2F5677003DD
:108A9000028B2ED394064003028B2E20400875646F
:108AA000EE75650080067564EF756500E56775F025
:108AB00012A42404FF0565E565AC64700205641426
:108AC000F5828C83EFF0AF660566A807E2FF0565C7
:108AD000E565AC647002056414F5828C83EFF030B8
:108AE00044057F501205181567E56760213044077B
:108AF000A866E2FF12057AAF65AE64AD660566A8AA
:108B000005E2FDC245128B2F8E648F6580D93044FB
:108B10000CA866E2FF12057A7F0A120518AF65AE4F
:108B200064A866E2FDD245128B2FD23EB240227C71
:108B3000808F828E837425F00FBF00010E8F828E8E
:108B4000837401F00FBF00010E8F828E837425F0B5
:108B50000FBF00010E8F828E837401F00FBF0001E2
:108B60000EEC60695D60308F828E83E533F00FBF5D
:108B700000010E8F828E83E4F00FBF00010E8F8202
:108B80008E83E533F00FBF00010E8F828E83E4F0F9
:108B90000FBF00010E80308F828E837425F00FBFCF
:108BA00000010E8F828E837401F00FBF00010E8FC3
:108BB000828E837425F00FBF00010E8F828E837426
:108BC00001F00FBF00010EECC313FC809430455E32
:108BD0008F828E83E533F00FBF00010E8F828E836C
:108BE000E4F00FBF00010E8F828E83E533F00FBFDC
:108BF00000010E8F828E83E4F00FBF00010E8F8282
:108C00008E837425F00FBF00010E8F828E83740156
:108C1000F00FBF00010E8F828E837425F00FBF000E
:108C2000010E8F828E837401F00FBF00010E227837
:108C3000787403F208741EF2EF90A1A493787AF28C
:108C4000EDC313540F24F5F582E434A1F583E493C6
:108C5000787BF2787C7403F2128CA022787874030B
:108C6000F208741EF2EF90A1A493787AF2ED540FFB
:108C700090A1F593787BF2787C7402F2128CA0229A
:108C800078787403F208741EF2EF90A1A493787AB6
:108C9000F2787BEDF2A245E433787CF2128CA022CC
:108CA000787AE2F566787BE2F567787CE2FF1392EA
:108CB00047EFA2E192487887E630E003D38001C312
:108CC0009246756578203F087563EC7564008006F0
:108CD0007563ED7564000564E564AE637002056359
:108CE00014F5828E837449F0780EE2B480047F001C
:108CF00080047879E2FF0564E564AC637002056383
:108D000014F5828C83EFF0AF64AE63AD66A248E4E5
:108D1000334402FB128DA88E638F64A2479249A24E
:108D200048924A1290FE8E638F64A2479249A248ED
:108D3000924A1290FE8E638F64AD67A248E433447A
:108D400004FB128DA88E638F64AD66A248E433FBEA
:108D5000128DA88E638F64A2479249A248924A124C
:108D600090FE8E638F64A2479249A248924A129065
:108D7000FE8E638F64AD67A248E433440CFB128D12
:108D8000A88E638F64D23DB23F30461B7F4D1205E3
:108D900018AF6612057AAF6712057A787CE2FF1287
:108DA000057A7F0A120518228E688F698D6A7F8086
:108DB000EB30E12285698285688374ACF00569E552
:108DC0006970020568856982856883740AF005699F
:108DD000E56970020568EB30E003028F6B791130B2
:108DE000E3034301407E10EB30E303430640EF64AE
:108DF000017003028E8AE56A5F6045856982856835
:108E00008374E5F00569E569700205688569828506
:108E100068837401F00569E56970020568856982F7
:108E20008568837445F00569E569700205688569A0
:108E300082856883E4F00569E5697002056880430E
:108E40008569828568837445F00569E56970020566
:108E500068856982856883E4F00569E569700205C3
:108E60006885698285688374E5F00569E569700243
:108E700005688569828568837401F00569E5697014
:108E8000020568EFC313FF028DEEE56A5F606E8531
:108E9000698285688374E5F00569E5697002056893
:108EA0008569828568837401F00569E5697002054A
:108EB00068EB30E2248569828568837426F0056951
:108EC000E56970020568856982856883EEF0056949
:108ED000E569700205680290F5856982856883748A
:108EE00045F00569E56970020568856982856883D2
:108EF000E4F00569E569700205680290F58569820C
:108F00008568837445F00569E569700205688569BF
:108F100082856883E4F00569E56970020568EB30D5
:108F2000E22485698285688374C6F00569E5697005
:108F3000020568856982856883E9F00569E56970DD
:108F40000205680290F585698285688374E5F005FD
:108F500069E569700205688569828568837401F036
:108F60000569E569700205680290F57908EB30E360
:108F7000034301407E08EB30E303430640EF640106
:108F80007003029019E56A5F604585698285688390
:108F900074F2F00569E56970020568856982856883
:108FA00083E4F00569E56970020568856982856872
:108FB000837422F00569E569700205688569828518
:108FC00068837480F00569E56970020568804385EF
:108FD00069828568837422F00569E5697002056815
:108FE0008569828568837480F00569E5697002058A
:108FF0006885698285688374F2F00569E5697002A5
:109000000568856982856883E4F00569E569700211
:109010000568EFC313FF028F7DE56A5F606D8569A8
:109020008285688374F2F00569E5697002056885D8
:109030006982856883E4F00569E56970020568EB7B
:1090400030E2248569828568837411F00569E569D9
:1090500070020568856982856883EEF00569E569B7
:10906000700205680290F58569828568837422F034
:109070000569E56970020568856982856883748081
:10908000F00569E56970020568806A85698285680E
:10909000837422F00569E569700205688569828537
:1090A00068837480F00569E56970020568EB30E259
:1090B0002385698285688374E1F00569E56970023A
:1090C0000568856982856883E9F00569E56970024C
:1090D0000568802185698285688374F2F00569E5F9
:1090E0006970020568856982856883E4F00569E531
:1090F0006970020568AC68AD69AF05AE0422204A0C
:10910000663049328F828E8374E5F00FBF00010E06
:109110008F828E837401F00FBF00010E8F828E83C9
:109120007445F00FBF00010E8F828E83E4F00FBFF5
:1091300000010E0291CA8F828E837445F00FBF002A
:10914000010E8F828E83E4F00FBF00010E8F828E9E
:109150008374E5F00FBF00010E8F828E837401F0DF
:109160000FBF00010E80633049318F828E8374F20D
:10917000F00FBF00010E8F828E83E4F00FBF00015D
:109180000E8F828E837422F00FBF00010E8F828EAD
:10919000837480F00FBF00010E802F8F828E837446
:1091A00022F00FBF00010E8F828E837480F00FBFFC
:1091B00000010E8F828E8374F2F00FBF00010E8FBC
:1091C000828E83E4F00FBF00010E2290F008740736
:1091D000F075F003EFA4FDACF0F5828C83E0FEA304
:1091E000E0F98D828C83A3A3E0F56BEEB50103F06B
:1091F000802CEEB56B088D828C83A3F08020E9B5BE
:109200006B08FE8D828C83F08014EF90A40D93FE8A
:109210008D828C83F0A3F08D828C83A3A3F090F0D9
:1092200008E4F0EF90A30D93FDEEC39D400BEF908B
:10923000A50D93FDEED39D4007EF90A40D93FF2263
:10924000AF06228D6BAE0790F0087407F075F0033F
:10925000EEA485F06CF56DAF6BEE90A30D93FDEE73
:1092600090A50D93FB1299198F6B856D82856C8388
:10927000EFF0A3F0856D82856C83A3A3F090F008D6
:10928000E4F0AF6B22E4FF1291CB7840EFF27F0164
:109290001291CB08EFF27F021291CB7891EFF27F1F
:1092A000031291CB08EFF27F041291CB788CA607C2
:1092B000E6FB24F6FFE434FFFE7C017DF412D36369
:1092C0001C7D4912D377788EEEF208EFF27840E2F7
:1092D000FFEB8FF0A4FFAEF07891E2FD7C0012D39B
:1092E00077EF2B788CF67F061291CB786DEFF27FBB
:1092F000081291CB7835EFF27F091291CB7838EFD5
:10930000F27F0A1291CB8F337F0D1291CBEF25E0C4
:10931000147834F27F0E1291CBEF25E014784FF2DF
:109320007F101291CB7853EFF27F111291CB784ED0
:10933000EFF27F121291CB7859EFF27F131291CB9B
:10934000780AEFF27F141291CB18EFF27F15129189
:10935000CB9091BFEFF07F181291CB7854EFF27F52
:10936000191291CB08EFF27F1E1291CB909191EFE1
:10937000F07F1F1291CB909197EFF07F201291CB4D
:1093800090919DEFF07F211291CB9091A3EFF07F10
:10939000221291CB9091A9EFF07F231291CB909163
:1093A000AFEFF07F241291CB9091B5EFF07F2512B3
:1093B00091CB9091BBEFF07F281291CB909192EFDF
:1093C000F07F291291CB909193EFF07F2A1291CBED
:1093D000909198EFF07F2B1291CB909199EFF07FC5
:1093E0002C1291CB90919EEFF07F2D1291CB90910A
:1093F0009FEFF07F2E1291CB9091A4EFF07F2F1270
:1094000091CB9091A5EFF07F301291CB9091AAEF84
:10941000F07F311291CB9091ABEFF07F321291CB74
:109420009091B0EFF07F331291CB9091B1EFF07F3C
:10943000341291CB9091B6EFF07F351291CB909191
:10944000B7EFF07F361291CB9091BCEFF07F3712DF
:1094500091CB9091BDEFF07F381291CB909194EF2A
:10946000F07F391291CB90919AEFF07F3A1291CB25
:109470009091A0EFF07F3B1291CB9091A6EFF07FFF
:109480003C1291CB9091ACEFF07F3D1291CB90913B
:10949000B2EFF07F3E1291CB9091B8EFF07F3F1288
:1094A00091CB9091BEEFF07F531291CB7851EFF2B8
:1094B0007F5A1291CBEF30E003D38001C39213EFB8
:1094C00030E103D38001C392127F0B1291CB129A29
:1094D0003C129A5E2290F001E0F56490F000E0FF0B
:1094E000540BFEBE08107882E26007EF540F909193
:1094F000C0F0EF783AF2783AE26F6021E4F55790E5
:10950000F00DF0754B35754C01754D0D12519C12D7
:10951000519C12519CD2AED2BEC2AF80FC300E1014
:10952000E56420E10BC20EE47870F21299BD80125E
:10953000200E0FE56430E10AD20E78707423F21227
:1095400099BD300F10E56420E20BC20FE47871F290
:109550001299C88012200F0FE56430E20AD20F780A
:10956000717423F21299C87870E26058E56430E1B2
:1095700053E214F2641470311299741299D3E4789E
:109580003EF27F041291CB788CA6077840E2FF78F8
:109590008CE6FB8FF0A4FFAEF07891E2FD7C001228
:1095A000D377EF2B788CF6801B7870E270167F04EF
:1095B000D244127E5D783EEFF21313543F788C262E
:1095C000F612995E7871E26035E56430E230E214BB
:1095D000F2B4140F12997F1299DEE4783FF2129AD6
:1095E0005E801B7871E270167F05D244127E5D7832
:1095F0003FEFF21313543F788F26F6129969E56412
:1096000054846404701A201417200C142015117847
:1096100071E2700CD20CD2141299C8C2451297DCB8
:10962000E56454426402701A2014172009142015AE
:10963000117870E2700CD209D2141299BDC2451291
:1096400097DC202132E56430E3252003227853E2C1
:10965000D39401401A7856E2FF14F2EF7047D20318
:10966000D2141299F912999DC2451297DC8036786E
:109670004EE27856F2802EE56430E31E301526C2A5
:109680001EC214C209C20CC2031299E97F507EC3E4
:109690001203C012998AC215800BD2151299F912C1
:1096A000999D129A20C3788BE6943518E694014070
:1096B00005E55720E20CE5574480F55790F00DF092
:1096C000800AE557547FF55790F00DF0C3788EE689
:1096D000943518E694014005E55720E30CE557441E
:1096E00020F55790F00DF0800AE55754DFF55790BC
:1096F000F00DF020210A302607C2451297DCC22661
:1097000090F700E030E01012CE727885E630E50781
:109710007EA07F731203CF7F0A227E01E4FDEDC39A
:10972000940440030297DB74722DF8E2FC7003028C
:1097300097D375F02CECA42409F582E5F0344EABF8
:1097400082F5598B5A74622DF8E2F47065E5822433
:1097500013F582E43559F583E0FCC313F98B82E5F8
:1097600082241AF582E43559F583E030E0034301A1
:10977000807C01E4FFEC603274052DF8E25CFBE9CB
:109780005C6B601FE26CF274622DF8EFF2E55A2414
:109790001AF582E43559F583E06440F07843E24EEF
:1097A000F2802EEC25E0FC0F80CB74722DF8E4F2F1
:1097B000801F74622DF8E2FC14F2EC6014E55A2468
:1097C0001AF582E43559F583E06440F07843E24EBF
:1097D000F2E4FF0DEE25E0FE02971E22754B357573
:1097E0004C01300911754D03302131201531754C74
:1097F00002129A2E8026300C05754D0C801E300307
:1098000005754D038016301405754D02800E301E0F
:1098100005754D018006204506E4F54D12519C2248
:1098200090F001E0FF20E104C20E8002D20EEF2092
:10983000E204C20F8002D20F30210F783AE254F0D6
:10984000FFC4540F04780FF28008783AE254C078CD
:1098500080F230210790F00BE4F0800690F00B745A
:1098600004F0129A5E300E031299D3300F0312994E
:10987000DEC2AFD2AED2BED2AF7F507EC31203C023
:109880007F04D244127E5D783EEFF27F05D244120F
:109890007E5D783FEFF218E22403F208E22403F23F
:1098A00018E2FF1313543F788C26F6783FE2FF133B
:1098B00013543F788F26F6302109C2AFD2AED2BE04
:1098C000D2AF227FFFE4FD12878812998A129A1F75
:1098D000E4F559203DFD7FFFE4FD128788C2AFD239
:1098E000AED2BED2AF0559E559C3940A40E5E4FFB4
:1098F0007888E2FD12878812999DE4F5597FE27E0F
:10990000041203C0C2AFD2AED2BED2AF0559E559E0
:10991000C3940A40E812998A22AE07EEC39D500311
:10992000AF0522EED39B4003AF0322AF06228E6722
:109930008F68AA05A802E2FE08E2FFC3E5689FFF60
:10994000E5679EFEAD037C0012D3CCA80208E22F8F
:10995000FF18E23EFEAD02A805F208EFF222E5573D
:109960004404F55790F00DF022E5574408F5579060
:10997000F00DF022E55754FBF55790F00DF022E57D
:109980005754F7F55790F00DF022E5574404F5577A
:1099900090F00DF02016054408F557F022E55754D5
:1099A000FBF55790F00DF054F7F557F02230120AFE
:1099B000E55754F7F55790F00DF0A21222E55754F1
:1099C000FEF55790F00DF022E55754FDF55790F055
:1099D0000DF022E5574401F55790F00DF022E557C0
:1099E0004402F55790F00DF022E5574401F55790E9
:1099F000F00DF04402F557F022E55754FEF557906C
:109A0000F00DF054FDF557F02278A0E64480F69072
:109A1000F00CF02278A0E6547FF690F00CF02222B1
:109A200030210A78A0E654BFF690F00CF0223021E5
:109A30000A78A0E64440F690F00CF0227598524364
:109A4000D880EF25E0240DF582E434A7F583E49374
:109A5000FC740193F5AAEC5403F5BAC2B2227F0755
:109A60001291CB786FEFF27F051291CB788FA6071A
:109A70007841E2FF788FE6FB8FF0A4FFAEF078929A
:109A8000E2FAFD7C0012D377EF2B788FF67880E234
:109A900024C0600624C0702DD216788FE6D3940AB5
:109AA00040177841E275F00AA4FFAEF0EAFD7C00B1
:109AB00012D377EF240A788FF6786FE2D3940540BB
:109AC000337405F222200F2C788FE6D3941E4019B0
:109AD0007841E275F01EA4FFAEF07892E2FD7C00C2
:109AE00012D377EF241E788FF6786FE2D39432404A
:109AF000037432F222E4FE74722EF8E26F60210EDB
:109B0000BE04F4E4FE74722EF8E27010EFF27405F5
:109B10002EF8EDF274622EF874FFF2220EBE04E508
:109B200022C206754B33786AE2F54E7842E2F54D73
:109B3000E54DF4607730231E75F005E54EA4240949
:109B4000F582E5F03490AF82F55D8F5E754C03F5DC
:109B500083E0F54F80537836E2FE08E2FF4E60085E
:109B60007850E28F828E83F0754C0575F00BE54ED0
:109B7000A42409F582E5F0347AAF82F55D8F5EE5C5
:109B80004D30E00BE4255EF55E740B355DF55D85CB
:109B90005E82855D83E0F54FA3E0F550855E8285AA
:109BA0005D83A3A3E0F551C22712519C22E4F5592D
:109BB000F5607561FF75620AF5347834E2F53B753E
:109BC0003F04754004203D6CE53460041534806129
:109BD000E559603E7F3F1205187878E559F208E5AF
:109BE0003BF2856034E5607004D21C8004C21C1511
:109BF00034E4F563E563C395595012745A2563F84C
:109C0000E6FF747A2563F8EFF2056380E7E4F5591F
:109C1000801F201C1C78787403F208E53BF2787AE8
:109C200074FFF2E4787BF2787C74FFF27F691205AE
:109C3000181287A3E5087003029CD3E5596003025C
:109C40009CD312038E8F55E555B4F00812038E8F06
:109C50003B029CD3E555B4F10712038E8F3F80730E
:109C6000E555B4F21B753752D22B1299AD7F7212A3
:109C7000051812411D7F52120518E47884F68053AE
:109C8000E555B4F30280FEE55564F4704612038E88
:109C90008F6012038E8F59E5597008755903129918
:109CA0009D800312998AE4F563E563C39559501EBC
:109CB000E5632475FF12051812038E745A2563F8A4
:109CC000A607E5632455FF120518056380DB7F2195
:109CD0001205187884E67003029BC5788416E54067
:109CE000600ED5400B853F4090F002E0FF12057AF0
:109CF000E561600ED5610B7561FF7F731205181267
:109D000079A7E562600DD5620A7F6F12051812947B
:109D1000D58F62202503029BC5C22575A0FCC2AF6A
:109D2000D2AED2BED2AF029BC522301062C210E4C6
:109D3000FF3017020F0FC205303F1E74E42FF5826B
:109D4000E434EEF583E0602D74E52FF582E434EE23
:109D5000F583E06020D205801C74E02FF582E434A6
:109D6000EEF583E0600F74E12FF582E434EEF583C5
:109D7000E06002D2053005177850E2FF7836E2FC49
:109D800008E2F5828C83EFF0E47883F2129B2130B5
:109D90001F04C21FD210224D5831206D6F64656CB4
:109DA00020323030300020202053573A4D58314D6A
:109DB0003200446F776E6C6F616400466C6173684B
:109DC0002E2E2E00446F776E6C6F61642E2E2E0047
:109DD000456D7066546573740D0A0045210D0A20A7
:109DE000202000206D3D0020653D0020733D0020B7
:109DF0007A3D0020613D0020643D0020703D002040
:109E0000773D000D0A004E3A20004F3A20003F3FB8
:109E10003F3F3F3F3F3F0D003F3F620D003F3F6CE4
:109E2000003F3F690D000D0A442D70633D006C61D9
:109E30003D000D0A4D2D70633D0050726F673A2052
:109E40002020202020202020202000505247205376
:109E5000746172740A0049524546203E20302E3209
:109E600035410A0050524720494E49540A00505289
:109E700047204C4545524C4155460A0048617264A2
:109E800072657365740050524720484152445245F0
:109E90005345540A0050524720502D55500A005047
:109EA000524720502D5550320A00505247204952F7
:109EB000454620005052472049524546203E20301A
:109EC0002E3235410A004356003D202020005052DA
:109ED0004720574F524B494E475F4449520A004E64
:109EE0004F2041434B202D3E2050524720574F5288
:109EF0004B494E475F4449525F454E44450A005026
:109F0000524720574F524B494E475F4449525F4298
:109F10005954450A0050524720574F524B494E471B
:109F20005F504859530A005052472043005052474F
:109F3000204552520050524720502D444E0A0050A6
:109F4000524720414242525543480A00505247204E
:109F5000456E640A000A5052472043563A00457243
:109F6000726F723A20202020006873000D0A57009B
:109F700043414E5F496E697420210A004E554C4C96
:109F8000200020410020506E0020506D004C4F47B3
:109F90003A20496E69745072696F0A000A4443435B
:109FA000757365643A20000A4D4F54757365643AC1
:109FB0002000204F464620200020554550202000FC
:109FC0002055455320200020415553202000205388
:109FD0005350202000204E6F20536900534C2055D1
:109FE000455300676E616C202000536574204175F5
:109FF00078496E203C2D204F6666202020202020AE
:10A000002020202020202020202000536574204183
:10A010007578496E203C2D204F6E20202020202076
:10A020002020202020202020202020004552523AAD
:10A030002049204C6565726C617566207A752068D0
:10A040006F636800204C61737420616E7374656384
:10A050006B656E00446174656E7665726C757374C1
:10A06000210D0A002020446174656E7665726C755E
:10A070007374004255534F46463A43414E5F496E12
:10A08000697420210A0020322E303300312E303105
:10A090002E3030302052414D20696E204F72646E58
:10A0A000756E6700090909090909090909090909FA
:10A0B000090909090A0A0A0A09090909090908080E
:10A0C000080808080A0A0A0A0A0A09090908080801
:10A0D000070707070C0C0B0B0B0A090908080808EF
:10A0E000070707070D0D0C0B0B0A090908080707DE
:10A0F000070606060E0E0E0C0A0A090908080707CD
:10A10000060606060F0F0E0E0B0A090808070707BA
:10A110000606060610100F0D0C0A090807060606AB
:10A120000505050510100E0C0B0A090807060505A4
:10A13000060707070F0F0E0C0B0A0908070605058F
:10A14000050608080E0E0D0B0A0908070605060786
:10A15000080809090D0D0C0A090807070606070873
:10A16000080909090C0C0B0A090807070707070863
:10A1700009090A0A0B0B0A09080707070707080954
:10A18000090A0A0A0A0A0909080807070708080944
:10A19000090A0B0B09090808080707080809090A32
:10A1A0000A0B0B0BAAC08030F0B020E0A00CCC8CC6
:10A1B0003CFCBC2CECAC08C88838F8B828E8A803EC
:10A1C000C38333F3B323E3A30FCF8F3FFFBF2FEF3F
:10A1D000AF0BCB8B3BFBBB2BEBAB02C28232F2B2A1
:10A1E00022E2A20ECE8E3EFEBE2EEEAE0ACA8A3A03
:10A1F000FABA2AEA0000C030F00CCC3CFC03C333AE
:10A20000F30FCF3FFF5050504450505050505050DB
:10A210005050505050515151515151515151515133
:10A22000115151515104040404440404040404046D
:10A2300004040404040505050505050505050505D3
:10A2400005110505051414141414144414141414DD
:10A2500014141414141515151515151515151515B3
:10A2600015151511155454545454545444545454FD
:10A270005454545454555555555555555555555593
:10A280005555555511010201030102010401020156
:10A2900003010201040102010301020104010201A0
:10A2A0000301020100010201030102010401020194
:10A2B0000301020104010201030102010401020180
:10A2C0000301020104010201030102010401020170
:10A2D0000301020100010201030102010401020164
:10A2E0000301020104010201030102010401020150
:10A2F0000301020104010201030102010401020140
:10A300000301020100010204081020408001010144
:10A3100001010101015A5A9201000A1400010100D1
:10A32000010101000000000000000000000000002A
:10A33000000000000000000000000000000000001D
:10A3400000000000000B0B0B0B0B0B0B0B000000B5
:10A3500000000000000000000000000000010101FA
:10A3600000000000000000000000000000000000ED
:10A3700000000000000000000000000000000000DD
:10A3800000000000000000000000000000000000CD
:10A3900000000000000000000000000000000000BD
:10A3A00000000000000000000000000000000000AD
:10A3B000000000000000000000000000000000009D
:10A3C000000000000000000000000000000000008D
:10A3D000000000000000000000000000000000007D
:10A3E000000000000000000000000000000000006D
:10A3F000000000000000000000000000000000005D
:10A400000000000000000000000000000044486759
:10A41000655050FAFA6666A204001A1700020A0094
:10A42000FF64460000000001000000000000000082
:10A43000000000000000000000000000000000001C
:10A44000000000000000000000000000000000000C
:10A4500000000000000000000000000000070707E7
:10A4600000000000000000000000000000000000EC
:10A4700000000000000000000000000000000000DC
:10A4800000000000000000000000000000000000CC
:10A4900000000000000000000000000000000000BC
:10A4A00000000000000000000000000000000000AC
:10A4B000000000000000000000000000000000009C
:10A4C000000000000000000000000000000000008C
:10A4D000000000000000000000000000000000007C
:10A4E000000000000000000000000000000000006C
:10A4F000000000000000000000000000000000005C
:10A5000000000000000000000000000000787878E3
:10A51000789650FEFE6E6EA206001E1E0005FE7F9F
:10A52000FFFFFFFFFFFFFF01010000060606060612
:10A530000606060000FFFFFFFFFFFFFFFFFFFFFF14
:10A54000FFFFFFFFFF6363636363636363000000F8
:10A5500000000000000000000000000000070907E4
:10A56000FF000000000000030000000000000000E9
:10A5700000000000000000000000000000000000DB
:10A5800000000000000000000000000000000000CB
:10A5900000000000000000000000000000000000BB
:10A5A00000000000000000000000000000000000AB
:10A5B000000000000000000000000000000000009B
:10A5C000000000000000000000000000000000008B
:10A5D000000000000000000000000000000000007B
:10A5E000000000000000000000000000000000006B
:10A5F000000000000000000000000000000000005B
:10A60000000000000000000000000000000000004A
:10A61000000101010101010101010101010101012B
:10A620000101010303010103000101010101010115
:10A63000010101010101010101010101010101010A
:10A6400001010101010101010101010101010101FA
:10A6500001010101010101010101010101010101EA
:10A6600001010101010101010101010101010101DA
:10A6700001010101010101010101010101010101CA
:10A6800001010101010000000000000000000000C5
:10A6900000000000000000000000000000000000BA
:10A6A00000000000000000000000000000000000AA
:10A6B000000000000000000000000000000000009A
:10A6C000000000000000000000000000000000008A
:10A6D000000000000000000000000000000000007A
:10A6E000000000000000000000000000000000006A
:10A6F000000000000000000000000000000000005A
:10A700000000000000000000000000000003CC0278
:10A71000600330039803CC03E603F310204080006D
:10A72000000000546573742052616D0A0046696C24
:10A730006C2042616E6B2000546573742042616E20
:10A740006B20004665686C65722042616E6B20006C
:10A7500052616D204F4B2120200A0052616D20462E
:10A7600065686C657268616674210A00018C9601E7
:10A770008F96816DFA816FFA81600A810DFF815297
:10A7800000818841813D64013400013B41013D412C
:10A79000019400013103013800C122A020142020BF
:10A7A00020202020202020202020202020202020A9
:10A7B00020202020202020202020202020200136A2
:10A7C00014818164814D1E012A22012B00C10101E7
:10A7D0002C00C1BDC1BE00E541543FF56DC394409E
:10A7E000400302ABDB85436E74C4256DF582E4340F
:10A7F00091F5837418F0E54254E0FF700A754B1828
:10A80000754C01856D4D22EF6420600302ABDBE5E2
:10A8100043C39408400302ABDBE542540F14F56FC9
:10A8200064026009E56F6406600302ABDB754B1AD6
:10A83000E543C43354E04401F54C856D4D12519C01
:10A8400075F070E56DA42418F582E5F03400F58309
:10A8500075F00EE54312D402AF8285836B8F6C8551
:10A86000436EE0F54AAE6B7D44AB6F12CF96202D60
:10A870000302AB4020300302AB40E5455430700387
:10A8800002ABDBE4F551E5434480F54AE54530E4AD
:10A8900003434A08E5455403FFC454F0424A303BA1
:10A8A00045755180C23B78B2E6FE08E6FFF5828E20
:10A8B00083E54AF0A3E56DF020380302AAD9C23837
:10A8C00078ADA60608A6077885E620E40302AAD993
:10A8D000754B63754C0278ADE608E6F54DEEF54E26
:10A8E00012519C02AAD920370302A9AD78B7E6FE1F
:10A8F00008E6FFF5828E83A3E0656D70548F828E2B
:10A9000083E054CFFFE54A54CF6F7045E54AF0E449
:10A91000F5517885E620E40302ABDB754B65754C99
:10A920000778B7E6FC08E6FDECF54DAF05EFF54E10
:10A93000F5828C83E0F54FA3E0F55075510178ADB9
:10A94000E6FC08E6FDECF552AF05EFF55312519C1D
:10A950002278B8740226F618E436F6FE08E6F58288
:10A960008E83E0700D78AEE6240279B8F718E436ED
:10A9700019F778B7E6FE08E6F5828E83E0FF54C04B
:10A98000FEBE80CDA3E0B56D1EEF54CFFFE54A5467
:10A99000CFB5071378B7E6FE08E6F5828E83E54A61
:10A9A000F075510102A91275511002AA4E78B2E653
:10A9B000FE08E6FFF5828E83A3E0B56D188F828EC8
:10A9C00083E054CFFFE54A54CFB50709755140E500
:10A9D0004AF002AAD978B3740226F618E436F69043
:10A9E0001C1CE02402F0901C1BE03400F030384DB9
:10A9F000C238E6FE08E678ADA60608F67885E630A9
:10AA0000E414754B64754C0278ADE6FE08E6F54D2E
:10AA1000EEF54E12519CC3901C1CE09454901C1BEC
:10AA2000E0942A4004D22C802578B2E6FE08E6F5B0
:10AA3000828E83E54AF0A3E56DF002AAD9C3901C8B
:10AA40001CE09454901C1BE0942A4041D22CC22D4F
:10AA5000D231901C95E0FFA3E0901C1BCFF0A3EF38
:10AA6000F0E4901C95F0A3F0901C19E0FEA3E0F533
:10AA7000828E83E4F0A3F0201E5F20145CD21E754A
:10AA80004B35754C01754D0112519C804C78B2E6E6
:10AA9000FE08E6FFF5828E83E54AF0A3E56DF0201F
:10AAA000383778ADE6FC08E6FDF5828C83A3E0B587
:10AAB0006D03D38001C350218D828C83E054CFFD80
:10AAC000E54A54CFB50503D38001C3500C75510836
:10AAD000D23778B7A60608A60778B2E6FE08E6FFE2
:10AAE000F5828E83A3A3E4F08F828E83A3A3A3F0C9
:10AAF0007885E620E40302ABDB754B62754C087881
:10AB0000B2E6FC08E6FDECF54DAF05EFF54EF5823B
:10AB10008C83E0F54FA3E0F550302D034351013015
:10AB2000370343510278B7E6FC08E6FDECF552AF77
:10AB300005EFF55378ADE6FE08E6F55412519C2278
:10AB4000303A0CAF6CAE6BAD6DAB4312BD8F2220B3
:10AB5000360302ABDBE56C2408F582E4356BF58344
:10AB6000E030E63AE5445498FFE54A54986F606B4C
:10AB7000E54AA2E3500FE544A2E34009AF6CAE6B97
:10AB8000D24712ABDCE54AA2E34013E544A2E3500E
:10AB90000DAF6CAE6BAD6DAB6ED24712ADD9E56C3F
:10ABA000240CF582E4356BF583E030E62EE54AA20D
:10ABB000E4500FE544A2E44009AF6CAE6BC247120B
:10ABC000ABDCE54AA2E44013E544A2E4500DAF6CCF
:10ABD000AE6BAD6DAB6EC24712ADD9228E708F7168
:10ABE00030470512CE2A8007AF71AE7012CE4B30BF
:10ABF0004714E51054BFFFE5712406F582E4357073
:10AC0000F583EFF08012E51054BFFFE571240AF5DB
:10AC100082E43570F583EFF075740A3047047F08DD
:10AC200080027F10E50E5F600302ADD8E51320E7D8
:10AC300056E51020E70302ADD8AF741574EF70032A
:10AC400002ADD8E510543FF572E5115407F5737560
:10AC5000F070E572A42418F582E5F03400F58375F0
:10AC6000F00EE57312D402AF828583708F71E51107
:10AC7000A2E39247304707AE7012CE2A809DAF7193
:10AC8000AE7012CE4B809475740AE51220E7030271
:10AC9000ADD8E512543FF572E5135407F57375F01E
:10ACA00070E572A42418F582E5F03400F58375F0A0
:10ACB0000EE57312D402AF828583708F71E513A203
:10ACC000E39247304707AE7012CE2A8007AF71AECD
:10ACD0007012CE4BE51320E7193047047F0880023D
:10ACE0007F10E50E5F600302ADD8AF741574EF708E
:10ACF0009922C248C249754B1BE573C43354E044E2
:10AD000003F54C85724D754E03E5734408F54F30DD
:10AD100047047F0880027F10E50E5F6002D249750C
:10AD2000740A30492C204829304714E51054BFFFDD
:10AD3000E5712406F582E43570F583EFF08012E5C5
:10AD40001054BFFFE571240AF582E43570F583EFF6
:10AD5000F012519CAF741574EF700302ADD8E51278
:10AD600030E775E512543FF572E5135407F5737536
:10AD7000F070E572A42418F582E5F03400F58375CF
:10AD8000F00EE57312D402AF828583708F71E513E4
:10AD9000A2E39247304707AE7012CE2A8007AF7108
:10ADA000AE7012CE4BE51330E702D2483048133074
:10ADB00047047F0880027F10E50E5F601BE51030BE
:10ADC000E616754B1BE573C43354E04402F54C851D
:10ADD000724D754E0302AD22228E708F718D728B73
:10ADE0007330470512CE2A8007AF71AE7012CE4B7A
:10ADF000E511C4540F5407F54EC249E51230E74B34
:10AE0000E51330E324E512543F75F070A42421F5D6
:10AE100082E5F03400F583E513540775F00E12D483
:10AE200002E030E726D2498022E512543F75F070E7
:10AE3000A42425F582E5F03400F583E51354077565
:10AE4000F00E12D402E030E702D24975740AE5131D
:10AE500020E763E51020E70302B06AE510543FF5F0
:10AE600072E5115407F57375F070E572A42418F5B6
:10AE700082E5F03400F58375F00EE57312D402AF6D
:10AE8000828583708F71E511A2E39247304707AE48
:10AE90007012CE2A8007AF71AE7012CE4BAF741510
:10AEA00074EF700302B06A3047047F0880027F109D
:10AEB000E50E5F609922851254851353754B1BE58F
:10AEC00073C43354E0F54C85724D85734FE511C45E
:10AED000540F54076006434C0202AF60E51020E7B0
:10AEE00005434C03807A75740AE510543FF572E50A
:10AEF000115407F57375F070E572A42418F582E516
:10AF0000F03400F58375F00EE57312D402AF82853C
:10AF100083708F71E511A2E39247304707AE70123C
:10AF2000CE2A8007AF71AE7012CE4B3047047F0837
:10AF300080027F10E50E5F6005434C038022E5131D
:10AF400030E70B434C03754E03434F088012E51066
:10AF500020E705434C038008AF741574EF708A2214
:10AF600012519CE55420E70302B06AE554543FF5C2
:10AF700072E5535407F573E553A2E39247C248C202
:10AF80004A75740A75F070E572A42418F582E5F02C
:10AF90003400F58375F00EE57312D402AF82858319
:10AFA000708F71304707AE7012CE2A8007AF71AE36
:10AFB0007012CE4B85724D85734FE51330E721300B
:10AFC0004A0EC249E573C43354E04402F54C800C88
:10AFD000E573C43354E04403F54CD24AD248800AA6
:10AFE000E573C43354E04402F54C30480E30470456
:10AFF0007F0880027F10E50E5F606F304927304880
:10B0000024431040304710E5712406F582E4357082
:10B01000F583E510F0800EE571240AF582E43570C1
:10B02000F583E510F0304805E51030E63DE50F54B6
:10B0300007B54E08E54C5407FFBF030D12519C8520
:10B040007182857083A3E54EF0AF741574EF601ABA
:10B05000E51230E715E512543FF572E5135407F594
:10B0600073E513A2E3924702AF8422E541B41912BB
:10B07000E543B4630DD230202D3F202E3CD23AD28E
:10B080002F22E541641C7031E5436463702BC230AC
:10B090007E007F18C3EE941C50178F828E83741825
:10B0A000F0740E2FFFE43EFE740E2FFFE43EFE8090
:10B0B000E3303A05C23A12C25C22202D0302B19A53
:10B0C000303B0302B19A5344074344C07885E630CD
:10B0D000E429754B66754C0678B2E6FC08E6FDEC93
:10B0E000F54DAF05EFF54EF5828C83E0F54FA3E00B
:10B0F000F55085445185435212519C78B2E6FE08C2
:10B10000E6F5828E83E0B5441EA3E0B5431918E648
:10B1100008E6FFF5828E83E544F0A3A3E4F08F8276
:10B120008E83A3A3A3F02278B3740226F618E43624
:10B13000F6901C1CE02402F0901C1BE03400F0C3CD
:10B14000A3E09454901C1BE0942A402CD22CC22DD6
:10B15000D231901C95E0FFA3E0901C1BCFF0A3EF31
:10B16000F0E4901C95F0A3F0901C19E0FEA3E0F52C
:10B17000828E83E4F0A3F02278B2E6FE08E6FFF5C3
:10B18000828E83E544F0A3E543F08F828E83A3A3F0
:10B19000E4F08F828E83A3A3A3F02220310302B2B6
:10B1A000B1754B37754C0578AFE6F54D302D077806
:10B1B000A7E6F54E8003854D4E75F012E54EA424AA
:10B1C000A1F582E5F0341CAF8278ABF608A607E45F
:10B1D000F551F550F54FF55FE54F1313543FF54F1B
:10B1E000302D0B78AAE6B55F05434FC0802278ABBF
:10B1F000E6FE08E6FFF5828E83E0FCA3E04C6010DB
:10B200008F828E83E030E705434F808003434F40B9
:10B2100078AC740226F618E436F6055FE55FB404F0
:10B22000B7E55FC394085046E5501313543FF550FB
:10B23000302D0B78AAE6B55F054350C0802278AB6D
:10B24000E6FE08E6FFF5828E83E0FCA3E04C60108A
:10B250008F828E83E030E705435080800343504067
:10B2600078AC740226F618E436F6055F80B3E55F25
:10B27000C394095030302D0B78AAE6B55F054351D1
:10B2800003802278ABE6FE08E6FFF5828E83E0FCC1
:10B29000A3E04C60108F828E83E030E705435102BB
:10B2A0008003435101302C0343518012519CC23121
:10B2B000227896E2F56024C4F582E43491F583E0C7
:10B2C000700302B3C774C42560F582E43491F5833A
:10B2D000E014F0704175F070E560A42418F582E583
:10B2E000F03400AF82F55B8F5CE4F55F855C8285AE
:10B2F0005B837418F0740E255CF55CE4355BF55BDC
:10B30000055FE55FB408E5754B19754C0185604D27
:10B3100012519C02B3C7303A0302B3C7302E030266
:10B32000B3C77893E26560600302B3C775F070E558
:10B3300060A42418F582E5F03400AF82F55B8F5CE1
:10B34000F583E030E775E582240EF582E43583F578
:10B3500083E030E7668F82E582241CF582E4355B6A
:10B36000F583E030E7558F82E582242AF582E435C3
:10B370005BF583E030E7448F82E5822438F582E490
:10B38000355BF583E030E7338F82E5822446F58232
:10B39000E4355BF583E030E7228F82E5822454F5C3
:10B3A00082E4355BF583E030E7118F82E582246229
:10B3B000F582E4355BF583E020E70C754B19754C9D
:10B3C0000185604D12519C7896E204F2C39440408E
:10B3D00026E4F2F55F7893E204F2C394404002E47D
:10B3E000F27893E224C4F582E43491F583E07007A7
:10B3F000055FE55FB40ADE30350302B6AC20391BC9
:10B400009091BFE0FF901C18E0FE04F0EEC39F5047
:10B410000302B6ACD239E4F078B6F678B6E6FFC3EC
:10B420009414400302B6AA74452FF582E4341CF547
:10B4300083E06401600302B6A4EF25E0246DF58289
:10B44000E4341CF583E0FEA3E08E5DF55E055EE569
:10B450005EAE5D7002055D14F5828E83E0F54F05EA
:10B460005EE55EAE5D7002055D14F5828E83E0F5EB
:10B470004D7885E630E413754B60754C0478B6E67C
:10B48000F54E7897E2F55012519CE54F700302B5E6
:10B49000FEE54F20E70302B555303A0302B6A47823
:10B4A00097E2FFF46009EF78B666600302B6A4780D
:10B4B000B6E67897F2202E04D22ED22FE54D543FD7
:10B4C000F560E54F30E61C754B1B534F07E54FC445
:10B4D0003354E04403F54C434F08E4F54E12519CBD
:10B4E00002B44DE56044C0F541754223E54F540771
:10B4F000F5437544C0E54F5430FFC4540FF545E59E
:10B500004F30E3084344084345108006434410434A
:10B51000452075F070E560A42418F582E5F034004C
:10B52000F58375F00EE54312D402AF8285835B8FFD
:10B530005C754B1B534F07E54FC43354E04403F590
:10B540004CE4F54E12519CAF5CAE5BAD60AB431268
:10B55000BD8F02B44DE54F30E549E54D30E72E3063
:10B56000060302B6A4754B4D75414D754C037542EB
:10B5700003E54D547FF54EF544534F0F854F457508
:10B580004D0475430412519C1266BD8051E54D5423
:10B590003F4480F54B754CA1E54F545FF54D12517A
:10B5A0009C803BE54F30E63630060302B6A4754B6F
:10B5B0004D75414D754C03754203AF4D8F4E8F4411
:10B5C000E54F30E408754D017543018005E4F54D04
:10B5D000F543534F0F854F4512519C1266BD855E52
:10B5E00082855D83E0601778B6E625E0246DF582FC
:10B5F000E4341CF583E55DF0A3E55EF00622789760
:10B60000E278B666702C789774FFF212C25CC22E94
:10B6100078B6E6FF25E0246DF582E4341CF583E47A
:10B62000F0A3F074452FF582E4341CF5837402F026
:10B63000806E78B6E6FD25E0241DF582E4341CF525
:10B6400083A3E025E0FF0582D5820215831582E001
:10B6500033FE74A12FF582EE341CAF82F55D8F5E50
:10B66000F583E0547FF074452DF582E4341CF583B6
:10B67000E4F0ED25E0246DF582E4341CF583E4F07C
:10B68000A3F0ED25E0241DF582E4341CF583E0FEF3
:10B69000A3E0FF7C007D0912D37778AFA607D231F3
:10B6A00078B6062278B60602B41BC23922D20778D1
:10B6B0009774FFF220220D901C19E07002A3E06045
:10B6C0000302B7497E077F087D007B027A1C79A1BF
:10B6D00012D40E7E007F147D007B027A1C79451205
:10B6E000D40E7E007F287D007B027A1C796D12D4F7
:10B6F0000E7E007F287D007B027A1C791D12D40EFD
:10B70000E49023A9F0A3F0A3F0A3F0901C197423F4
:10B71000F0A374ABF0901C1BE4F0A37402F0E4906F
:10B720001C95F0A3F0909209F0A3F0909206F0A37C
:10B73000F09091C3F09091C1F0909204F090920833
:10B74000F0909205F09091C2F0901C95E0FEA3E07D
:10B75000FF4E601D901C1BEEF0A3EFF0901C19E053
:10B76000FEA3E0F5828E83E4F0A3F0901C95F0A395
:10B77000F07E007F18E4FDE4FC8F828E837418F065
:10B78000A3E4F0EF2406F582E43EF583E054BFF035
:10B79000EF240AF582E43EF583E054BFF0EF24077E
:10B7A000F582E43EF583E030E72CEF2406F582E4F1
:10B7B0003EF583E4F0EF2407F582E43EF583E4F000
:10B7C000EF2408F582E43EF583E4F0EF2409F582E6
:10B7D000E43EF583E4F0EF240BF582E43EF583E0EC
:10B7E00030E72CEF240AF582E43EF583E4F0EF2401
:10B7F0000BF582E43EF583E4F0EF240CF582E43EA1
:10B80000F583E4F0EF240DF582E43EF583E4F07473
:10B810000E2FFFE43EFE0CEC6408600302B7790DC6
:10B82000ED6440600302B777C2072278AFA643C237
:10B830002CD2312230350302BBAAC22CD23178AFD0
:10B84000A643E54375F009A4FFAEF0E544540FFDAF
:10B850007A002FF56CEA3EF56BE56C25E0FFE56BB1
:10B8600033FE74A12FF582EE341CAF8278ABF6085C
:10B87000A607302D73E54378A766600302BBAAEDE7
:10B8800078AA66600302BBAAC22D303B0302BBAAA2
:10B89000901C19E0FEA3E0FF08E6FC08E6F5828CA8
:10B8A00083EEF0A3EFF078B2E6FE08E6FFF5828EB5
:10B8B00083A3A3E4F08F828E83A3A3A3F0901C1C28
:10B8C000E02404F0901C1BE03400F0EF2404FFE4BB
:10B8D0003EFE901C19F0A3EFF0F5828E83E4F0A3F6
:10B8E000F0901C95F0A3F02278ABE6FE08E6FFF599
:10B8F000828E83E0FCA3E078B0A60408F6E5445409
:10B90000C06480706530330302BBAA30320302BBCF
:10B91000AA78B1E61846600302BBAA303A0302BB1C
:10B92000AA78A7A643E544540F78AAF6901C1BE01A
:10B93000FCA3E0FDC39448EC942A502B901C19E022
:10B94000FAA3E078B0A60208F608A60208F6D22DFF
:10B95000D23BD238C237F5828A83E4F0A3F0901C40
:10B9600095ECF0A3EDF022D22C2278B0E6FC08E6AC
:10B97000FD4C700302BBAAE54430E64BEC30E70314
:10B9800002BBAA8F828E83E4F0A3F078B2A60408EB
:10B99000A60508F608760278B0E6FE08E6F5828E7F
:10B9A00083E0601678B5740226F618E436F678B1AE
:10B9B000740226F618E436F680DD78B1740226F6B5
:10B9C00018E436F6D2352278B0E60820E70302BB49
:10B9D0004378ABE6FE08E6F5828E83E0547FF0E420
:10B9E000F56DE56D25E0241DF582E4341CF583E05A
:10B9F000FEA3E0656C7003EE656B6007056DE56D99
:10BA0000B414DFE56D6414700302BBAA7445256DA0
:10BA1000F582E4341CF583E4F0E56D25E0246DF552
:10BA200082E4341CF583E4F0A3F07897E2B56D0767
:10BA3000C22EC22F74FFF278ABE6FE08E6F5828EC6
:10BA400083E0FEA3E078B0A60608F678B00806E624
:10BA500018860670010614F5828E83E0F54F78B0E3
:10BA60000806E618860670010614F5828E83E0F556
:10BA70004D7885E630E40C754B61754C02854F4E70
:10BA800012519CE54F700302BBAAE54F54C0FFBFA3
:10BA900080B9E54D543FF56E75F070A42418F58219
:10BAA000E5F03400F583E54F540775F00E12D4022B
:10BAB000AF82AE83E54F30E342E5822406F582E4AF
:10BAC0003583F583E4F08F828E83E5822407F58247
:10BAD000E43583F583E4F08F828E83E5822408F5D4
:10BAE00082E43583F583E4F08F828E83E582240936
:10BAF000F582E43583F583E4F0802CEF240AF582A7
:10BB0000E43EF583E4F0EF240BF582E43EF583E4B4
:10BB1000F0EF240CF582E43EF583E4F0EF240DF51C
:10BB200082E43EF583E4F0754B1B534F07E54FC4A9
:10BB30003354E04403F54C856E4DE4F54E12519CB0
:10BB400002BA4BE4F56D7445256DF582E4341CF5BD
:10BB500083E06007056DE56DB414EBE56D6414607A
:10BB600049E56D25E0241DF582E4341CF583E56B81
:10BB7000F0A3E56CF07445256DF582E4341CF58383
:10BB80007401F078B0E6FE08E6FFE56D25E0246D6F
:10BB9000F582E4341CF583EEF0A3EFF078ABE6FE1B
:10BBA00008E6F5828E83E04480F022202D0302BC5B
:10BBB0008A53435F43432053413F303B25C23B7888
:10BBC000B2E6FE08E6FFF5828E83E543F0A3E54189
:10BBD000F08F828E83A3A3E4F08F828E83A3A3A32E
:10BBE000F02278B2E6FE08E6FFF5828E83A3E065D8
:10BBF0004170248F828E83E0541FFFE543541FB5AC
:10BC0000071518E608E6FFE543F0A3A3E4F08F82EA
:10BC10008E83A3A3A3F02278B3740226F618E43629
:10BC2000F6901C1CE02402F0901C1BE03400F0C3D2
:10BC3000A3E09452901C1BE0942A402CD22CC22DDD
:10BC4000D231901C95E0FFA3E0901C1BCFF0A3EF36
:10BC5000F0E4901C95F0A3F0901C19E0FEA3E0F531
:10BC6000828E83E4F0A3F02278B2E6FE08E6FFF5C8
:10BC7000828E83E543F0A3E541F08F828E83A3A3F8
:10BC8000E4F08F828E83A3A3A3F022202D0302BDB4
:10BC90008EE54330E210E545540F4420F549E54474
:10BCA0004480F54A8013E545540F4440F549E54387
:10BCB00030E00343491085444A303B25C23B78B20B
:10BCC000E6FE08E6FFF5828E83E549F0A3E54AF03B
:10BCD0008F828E83A3A3E4F08F828E83A3A3A3F02D
:10BCE00022E54320E23578B2E6FE08E6FFF5828ED3
:10BCF00083A3E0654A70248F828E83E05417FFE5AA
:10BD0000495417B5071518E608E6FFE549F0A3A35F
:10BD1000E4F08F828E83A3A3A3F02278B37402266B
:10BD2000F618E436F6901C1CE02402F0901C1BE090
:10BD30003400F0C3A3E09452901C1BE0942A402CE2
:10BD4000D22CC22DD231901C95E0FFA3E0901C1B99
:10BD5000CFF0A3EFF0E4901C95F0A3F0901C19E055
:10BD6000FEA3E0F5828E83E4F0A3F02278B2E6FE33
:10BD700008E6FFF5828E83E549F0A3E54AF08F825D
:10BD80008E83A3A3E4F08F828E83A3A3A3F0228EDD
:10BD9000708F718D728B73E5455430700302C25BF6
:10BDA000E545A2E49247304709AF71AE7012CE2A42
:10BDB0008007AF71AE7012CE4B302F3D909206E5EA
:10BDC00070F0A3E571F0909204E572F0909208E5AE
:10BDD00073F0A247E433FF9091C1F0909209E570AF
:10BDE000F0A3E571F0909205E572F09091C2E573D1
:10BDF000F0A3EFF0C22F02BE9F909205E0B572143F
:10BE00009091C2E0B5730DA247E433FFA3E06F70D9
:10BE10000302C21B304708E5734488F5748006E5C9
:10BE2000734480F5749091C3E06029E5724480FF0B
:10BE3000909209E0FCA3E0FD2406F582E43CF58342
:10BE4000EFF0ED2407F582E43CF583E054F0F04593
:10BE500074F08027E5724480FF909209E0FCA3E033
:10BE6000FD240AF582E43CF583EFF0ED240BF58226
:10BE7000E43CF583E054F0F04574F0909209E570ED
:10BE8000F0A3E571F0909205E572F09091C2E57330
:10BE9000F0A247E433A3F0E51130E70302C21B3000
:10BEA0004714E5114480FFE5712407F582E43570FD
:10BEB000F583EFF08012E5114480FFE571240BF566
:10BEC00082E43570F583EFF0E51020E70302C03B14
:10BED000E510543FF57285117330471DE571240656
:10BEE000F582E43570F583E4F0E5712407F582E42A
:10BEF0003570F5837480F0801BE571240AF582E4C7
:10BF00003570F583E4F0E571240BF582E43570F5C6
:10BF1000837480F0E573A2E3924753730775F07062
:10BF2000E572A42418F582E5F03400F58375F00E6F
:10BF3000E57312D402AF828583708F7130473CE580
:10BF4000822407F582E43583F583E030E70302C0FD
:10BF50001EE5712408F582E43570F583E4F0E5719F
:10BF60002409F582E43570F583E4F0E5712406F5E3
:10BF700082E43570F583E0F572803AE571240BF5C3
:10BF800082E43570F583E030E70302C01EE57124DA
:10BF90000CF582E43570F583E4F0E571240DF5824B
:10BFA000E43570F583E4F0E571240AF582E4357038
:10BFB000F583E0F572E57230E76430472AE57124D5
:10BFC00007F582E43570F583E0F573E5712406F535
:10BFD00082E43570F583E4F0E5712407F582E435F9
:10BFE00070F583E4F08028E571240BF582E4357068
:10BFF000F583E0F573E571240AF582E43570F58385
:10C00000E4F0E571240BF582E43570F583E4F0E5A6
:10C0100073A2E3924753730753723F02BF1D90927E
:10C0200009E0FEA3E08E70F571909205E0F5729044
:10C0300091C2E0F573A3E024FF9247E51220E703E5
:10C0400002C1ACE512543FF57285137330471CE50D
:10C05000712408F582E43570F583E4F0E571240974
:10C06000F582E43570F583E4F0801AE571240CF56F
:10C0700082E43570F583E4F0E571240DF582E43552
:10C0800070F583E4F0E573A2E3924753730775F00C
:10C0900070E572A42418F582E5F03400F58375F09C
:10C0A0000EE57312D402AF828583708F7130474AD8
:10C0B000E5822407F582E43583F583E030E7030267
:10C0C000C18FE5712406F582E43570F583E4F0E56F
:10C0D000712407F582E43570F583E4F0E5712408F6
:10C0E000F582E43570F583E0F572E5712409F58297
:10C0F000E43570F583E0F5738048E571240BF58233
:10C10000E43570F583E030E70302C18FE571240A5E
:10C11000F582E43570F583E4F0E571240BF582E4F3
:10C120003570F583E4F0E571240CF582E43570F5A3
:10C1300083E0F572E571240DF582E43570F583E056
:10C14000F57330471CE5712408F582E43570F583FA
:10C15000E4F0E5712409F582E43570F583E4F080BC
:10C160001AE571240CF582E43570F583E4F0E5718D
:10C17000240DF582E43570F583E4F0E57230E70FC5
:10C18000E573A2E3924753730753723F02C08E9048
:10C190009209E0FEA3E08E70F571909205E0F572D1
:10C1A0009091C2E0F573A3E024FF9247304737E552
:10C1B000712406F582E43570F583E4F0E571240717
:10C1C000F582E43570F5837480F0E5712408F5821A
:10C1D000E43570F583E4F0E5712409F582E4357007
:10C1E000F583E4F08035E571240AF582E43570F5D5
:10C1F00083E4F0E571240BF582E43570F5837480F7
:10C20000F0E571240CF582E43570F583E4F0E57116
:10C21000240DF582E43570F583E4F030471FE545E1
:10C220005407FFC454F0FFE511548F44804FFFE5DD
:10C23000712407F582E43570F583EFF022E545546B
:10C2400007FFC454F0FFE511548F44804FFFE571A0
:10C25000240BF582E43570F583EFF022302F0302D2
:10C26000C546909206E0FEA3E08E6DF56E909204B6
:10C27000E0F573909208E0F5719091C1E024FF928F
:10C2800047856E82856D837418F0304723AF6EAE9C
:10C290006D12CE2AE51120E70302C546E511547F51
:10C2A000FFE56E2407F582E4356DF583EFF080211C
:10C2B000AF6EAE6D12CE4BE51120E70302C546E529
:10C2C00011547FFFE56E240BF582E4356DF583EFA5
:10C2D000F0E510543FFF6573600302C35CE5115441
:10C2E0000765717077E511A2E3304701B3406D3007
:10C2F0004735E56E2406F582E4356DF583E4F0E517
:10C300006E2407F582E4356DF583E4F0E56E2408CC
:10C31000F582E4356DF583E4F0E56E2409F582E4F9
:10C32000356DF583E4F022E56E240AF582E4356D7F
:10C33000F583E4F0E56E240BF582E4356DF583E4D6
:10C34000F0E56E240CF582E4356DF583E4F0E56EDE
:10C35000240DF582E4356DF583E4F02220470302D5
:10C36000C41CE56E2408F582E4356DF583E0444095
:10C37000F0E51020E725E51220E710E56E2408F52A
:10C3800082E4356DF583E054BFF022E56E2409F5B3
:10C3900082E4356DF583E04480F0228F74E511541A
:10C3A00007F572E511A2E3924875F070E574A424D4
:10C3B00018F582E5F03400F58375F00EE57212D4BD
:10C3C00002AD8285836F8D70304816E5822407F5B3
:10C3D00082E43583F583E0FEC4540F5407F554809E
:10C3E00014E570240BF582E4356FF583E0FEC45448
:10C3F0000F5407F554E511C4540F5407F553600367
:10C4000002C4CCE554700302C4CCE56E2409F58265
:10C41000E4356DF583E04480F002C4CCE56E240C75
:10C42000F582E4356DF583E04440F0E51020E72522
:10C43000E51220E710E56E240CF582E4356DF583F6
:10C44000E054BFF022E56E240DF582E4356DF583EE
:10C45000E04480F0228F74E5115407F572E511A2D3
:10C46000E3924875F070EFA42418F582E5F03400EB
:10C47000F58375F00EE57212D402AF8285836F8F5B
:10C4800070304816E5822407F582E43583F583E0B1
:10C49000FFC4540F5407F5548014E570240BF58243
:10C4A000E4356FF583E0FFC4540F5407F554E511EC
:10C4B000C4540F5407F5537013E554600FE56E2410
:10C4C0000DF582E4356DF583E04480F03047034399
:10C4D0007108304823E57344C0FFE5702408F582F5
:10C4E000E4356FF583EFF0E5702409F582E4356FEC
:10C4F000F583E04571F08021E57344C0FFE57024C9
:10C500000CF582E4356FF583EFF0E570240DF582CC
:10C51000E4356FF583E04571F0909204E0B5741353
:10C52000909208E0B5720CA248E433FF9091C1E00C
:10C530006F6013856F6D85706E857473857271A2DF
:10C5400048924702C28122E4F566F567E56725E077
:10C55000FFE56633FE74A12FF582EE341CAF8278BE
:10C56000A8F608A607F583E0FEA3E0FF4E700302DD
:10C57000C605EE547F78B0F608A6077F5712051857
:10C580007F49120518E566FF12057AAF67E5671265
:10C59000057A7F0D1205187F0A12051878B0E6FE9D
:10C5A00008E6F5828E83E06048E509D3943F400BAE
:10C5B0003025F6C225D2AED2BE80EE78B00806E6AF
:10C5C00018860670010614F5828E83E0FF12057A44
:10C5D00078B00806E618860670010614F5828E8388
:10C5E000E0FF12057A7F0D1205187F0A12051880E8
:10C5F000ABE4FF12057AE4FF12057A7F0D120518ED
:10C600007F0A1205180567E56770020566C3E567CE
:10C610009484E5669403500302C54C22120594EFFE
:10C62000756700F566120594EF2567F567E43566D2
:10C63000F566C3E5679484E566940340087ECD7F84
:10C64000AB1203CF22E56725E0FFE56633FE74A158
:10C650002FF582EE341CAF8278A8F608A607F58382
:10C66000E0FEA3E04E60087ECD7FC51203CF2230EE
:10C670002D087ECD7FE01203CF22C3901C1CE094D6
:10C6800048901C1BE0942A40087ECD7FFB1203CF0C
:10C6900022901C1BE0FFA3E0901C95CFF0A3EFF0CD
:10C6A000901C19E0FEA3E078ADA60608F67F3F12C5
:10C6B00005187F0D1205187F0A120518D2332212B1
:10C6C00005948F661205948F6712054778AD0806AA
:10C6D000E618860670010614F5828E83E566F0E59D
:10C6E00066706B901C19E0FEA3E0FF78A8E6FC08DA
:10C6F000E6F5828C83EEF0A3EFF078AD0806E6183D
:10C70000860670010614F5828E83E4F078ADE6FEAD
:10C7100008E6FF901C19EEF0A3EFF0F5828E83E49B
:10C72000F0A3F0901C95F0A3F0901C1CE02402F004
:10C73000901C1BE03400F0C2337F6F1205187F6B32
:10C740001205187F0D1205187F0A1205182278AD00
:10C750000806E618860670010614F5828E83E567E2
:10C76000F0901C1CE02402F0901C1BE03400F0C38D
:10C77000A3E09452901C1BE0942A403D7ECD7FFBA9
:10C780001203CF78A8E6FE08E6F5828E83E4F0A3D4
:10C79000F0901C95E0FFA3E0901C1BCFF0A3EFF0FE
:10C7A000E4901C95F0A3F0901C19E0FEA3E0F58244
:10C7B0008E83E4F0A3F0C233227F3F1205187F0D71
:10C7C0001205187F0A120518227F6E1205187F665F
:10C7D000120518901C19E0FF12057A901C19E0FE52
:10C7E000A3E0FF12057A7F201205187F7512051845
:10C7F0007F63120518901C1BE0FF12057A901C1C29
:10C80000E0FF12057A7F0D1205187F0A12051878CD
:10C81000AB761C0876A1E4F566F567C3E5679484FA
:10C82000E5669403400302C8FB78ABE6FE08E6F534
:10C83000828E83E0FEA3E04E700302C8E67F4612BC
:10C840000518E566FF12057AAF67E56712057A7F7E
:10C850003A1205187F2012051878ABE6FE08E6F5B7
:10C86000828E83E0FF12057A78ABE6FE08E6F58259
:10C870008E83E0A3E0FF12057A7F2012051878ABC3
:10C88000E6FE08E6F5828E83E0547FFEA3E08E6824
:10C89000F569856982856883E06041E509D3943F45
:10C8A000400B3025F6C225D2AED2BE80EE0569E53A
:10C8B00069AE687002056814F5828E83E0FF120588
:10C8C0007A0569E569AE687002056814F5828E83A1
:10C8D000E0FF12057A7F2012051880B67F0D120541
:10C8E000187F0A1205180567E5677002056678ACBF
:10C8F000740226F618E436F602C81B7F41120518AA
:10C900007F0D1205187F0A120518E4F566F56774A5
:10C91000452567F582E4341CF583E0700302C9E124
:10C920007F41120518E566FF12057AAF67E56712C9
:10C93000057A7F201205187F4E1205187F721205A6
:10C94000187F3D120518E56725E0FFE56633FE74A4
:10C950001D2FF582EE341CF583E0FF12057AE567A2
:10C9600025E0FFE56633FE741D2FF582EE341CF5DD
:10C9700083E0A3E0FF12057A7F2012051874452595
:10C9800067F582E4341CF583E0FF12057A7F2012FC
:10C990000518E56725E0FFE56633FE746D2FF58227
:10C9A000EE341CF583E0FF12057AE56725E0FFE52C
:10C9B0006633FE746D2FF582EE341CF583E0FEA322
:10C9C000E0FF12057A7F0D1205187F0A120518E59F
:10C9D00009D3943F400B3025F6C225D2AED2BE809B
:10C9E000EE0567E56770020566C3E5679414E566C2
:10C9F0009400500302C90F22120547EF24BD7003B3
:10CA000002CC1624FA700302CB2724FA600302CC6E
:10CA100056E4F569E4F56875F070E569A42418F545
:10CA200082E5F03400F58375F00EE56812D402AFAC
:10CA3000828583668F67E5822408F582E43583F575
:10CA400083E020E6148F82E582240CF582E43566CB
:10CA5000F583E020E60302CB0E7F4F1205187F49D5
:10CA6000120518AF6912057AAF6812057A7F3A127B
:10CA70000518E5672406F582E43566F583E0FF12C4
:10CA8000057AE5672407F582E43566F583E0FF1251
:10CA9000057AE5672408F582E43566F583E0FF1240
:10CAA000057AE5672409F582E43566F583E0FF122F
:10CAB000057AE567240AF582E43566F583E0FF121E
:10CAC000057AE567240BF582E43566F583E0FF120D
:10CAD000057AE567240CF582E43566F583E0FF12FC
:10CAE000057AE567240DF582E43566F583E0FF12EB
:10CAF000057A7F0D1205187F0A120518E509D394EF
:10CB00003F400B3025F6C225D2AED2BE80EE05687E
:10CB1000E568C39408500302CA170569E569C39420
:10CB200040500302CA14221205948F691205948F93
:10CB300068120547BF3A0EE569C394405007E5689F
:10CB4000C3940840127ECE7F141203CF120547EF24
:10CB5000700302CC5680F575F070E569A42418F5D1
:10CB600082E5F03400F58375F00EE56812D402AF6B
:10CB7000828583668F67120594E5672406F582E453
:10CB80003566F583EFF0120594E5672407F582E436
:10CB90003566F583EFF0120594E5672408F582E425
:10CBA0003566F583EFF0120594E5672409F582E414
:10CBB0003566F583EFF0120594E567240AF582E403
:10CBC0003566F583EFF0120594E567240BF582E4F2
:10CBD0003566F583EFF0120594E567240CF582E4E1
:10CBE0003566F583EFF0120594E567240DF582E4D0
:10CBF0003566F583EFF0120547EF640D600302CB55
:10CC0000457F6F1205187F6B1205187F0D120518EE
:10CC10007F0A12051822120547EF644C703812057E
:10CC200047EF64457030120547EF644170281205E4
:10CC300047EF64527020D2077E1C7F007D007B028C
:10CC40007A00791812D40EC22212B6AD7F2A1205CC
:10CC5000187F0D12051822909209E0FEA3E08E596C
:10CC6000F55A909205E0F55B9091C2E0F55CA3E087
:10CC700024FF9243755DFF20430302CD05855A8250
:10CC8000855983E05488FFBF880FAF5AAE59AD5B1A
:10CC9000AB5CA243924712ADD9E55A2408F582E471
:10CCA0003559F583E0FF20E70302CDAAEF543FF5A5
:10CCB0005BE55A2409F582E43559F583E05407F51C
:10CCC0005C75F070E55BA42418F582E5F03400F59E
:10CCD0008375F00EE55C12D402AF828583598F5ABA
:10CCE000E5822409F582E43583F583E0A2E39243EB
:10CCF0008F82E5822408F582E43559F583E030E639
:10CD00000302CD8622855A82855983E05490FFBF65
:10CD1000900FAF5AAE59AD5BAB5CA243924712ADD8
:10CD2000D9E55A240CF582E43559F583E0FF30E764
:10CD300079EF543FF55BE55A240DF582E43559F55A
:10CD400083E05407F55C75F070E55BA42418F58268
:10CD5000E5F03400F58375F00EE55C12D402AF8285
:10CD60008583598F5AE582240DF582E43583F58356
:10CD7000E0A2E392438F82E582240CF582E43559E8
:10CD8000F583E030E624909206E0FEA3E0B55A1168
:10CD9000E559B5060CA243E433FF9091C1E06F6002
:10CDA00009155DE55D600302CC77224552523A20B9
:10CDB0007A7520686F6865204673742D4E756D6DA9
:10CDC00065720D0A004552523A204673742062651E
:10CDD00072656974732062656E75747A740D0A00E9
:10CDE0004552523A20446566696E6974696F6E20D7
:10CDF000696D2047616E67210D0A004552523A2045
:10CE00004673742D537065696368657220766F6C24
:10CE10006C0D0A004552523A20496E76616C696485
:10CE200020466F726D61740D0A008E838F82790EB9
:10CE3000E0F709A3E0F709A3A3A3A3A3E0F709A3DD
:10CE4000E0F709A3E0F709A3E0F7228E838F827948
:10CE50000EE0F709A3E0F709EF240AFF50010E8E58
:10CE6000838F82E0F709A3E0F709A3E0F709A3E0C5
:10CE7000F72290F7007443F090F70474C3F0A374A2
:10CE80001CF0A3E4F0A3F090F70CF0A3F090F716D9
:10CE90007408F090F7117455F090F7107495F090B5
:10CEA000F7207440F090F730F090F740F090F75092
:10CEB000F090F760F090F770F090F780F090F790B6
:10CEC000F090F7A0F090F7B0F090F7C0F090F7D0A6
:10CED000F090F7E0F090F7F07499F0A37455F090AB
:10CEE000F7F67480F090F700740AF0781D76E0226F
:10CEF000C0E0C083C082C0D0C000C00790F701E08E
:10CF0000FF30E715203C12D23C90F7007403F07418
:10CF10000AF0781A74FFF68070C23C781AE6700442
:10CF2000EF5487F690F702E0FFC39402405BEFD323
:10CF300094105055BF02047F0F80021F1FEFC4548E
:10CF4000F0FFE42FF582E434F7F5837441F0781BA9
:10CF50000674112FFFBF01027F21E42FF582E43414
:10CF6000F7F5837455F01F74062FF582E434F7F556
:10CF7000837480F0E42FF582E434F7F5837499F03C
:10CF8000781CE6C394FF500106D007D000D0D0D063
:10CF900082D083D0E0328E838F828D01E709F0A3A7
:10CFA000EB603DDBF7228C838D828F01E0F709A3D4
:10CFB000EB602DDBF7228F008D01E3F60809EB60B3
:10CFC0001FDBF7228F008D01E7F20809EB6011DB10
:10CFD000F7228F008D01E7F60809EB6003DBF722EB
:10CFE0002275B12078FFE4F6D8FD75A0FC78007FAB
:10CFF00000E4F208DFFC7581B802D0370205E8E4EE
:10D0000093A3F8E493A34003F68001F208DFF480D1
:10D0100029E493A3F85407240CC8C333C4540F4421
:10D0200020C8834004F456800146F6DFE4800B01FB
:10D030000204081020408090A76CE47E019360BC3D
:10D04000A3FF543F30E509541FFEE493A360010E93
:10D05000CF54C025E060A840B8E493A3FAE493A3BA
:10D06000F8E493A3C8C582C8CAC583CAF0A3C8C5DB
:10D0700082C8CAC583CADFE9DEE780BE35CBF5CBFF
:10D08000C2C20582151475920490F00DE55754FB49
:10D09000F0D092D0D0D0E03235CBF5CBC2C20582F1
:10D0A0001514B29075920490F00DE557F0D092D01F
:10D0B000D0D0E03235CBF5CBC2C205821514D09268
:10D0C000D0D0D0E03235CBF5CB0582B290151475B7
:10D0D000E00A10C213D5E0FAD092D0D0D0E032C02E
:10D0E000E0C0D0C092759201E5146024B40300E062
:10D0F000058225CAF5CAE010E7CB10E6B735CBF5B7
:10D10000CBB290C2C205821514D092D0D0D0E032FA
:10D11000E516603CE53325CAF5CAE435CBF5CBB25C
:10D1200090C2C2151680E2E55860DE15587592036C
:10D13000A310C2B1759204E0543060F5759203E01B
:10D1400005E0F010C29F759204E0543070F580E164
:10D15000C23D20BB020556E53325CAF5CAE435CBEE
:10D16000F5CBC290C2C2303F2090EC00E00582F5C2
:10D1700014E00582F516202B0975920390EEDF75F9
:10D180005804D092D0D0D0E03290ED00E00582F586
:10D1900014E00582F516D092D0D0D0E032C0E0C0C5
:10D1A000D0C092759202E515604CE0058225C2F56B
:10D1B000C2E010E72710E61335C3F5C3B291C2C32E
:10D1C00005821515D092D0D0D0E03235CBF5CBC248
:10D1D000C305821515D092D0D0D0E03235C3F5C347
:10D1E000B2910582151575E00A10C3BAD5E0FAD0E0
:10D1F00092D0D0D0E032E5176018E53325C2F5C2F1
:10D20000E435C3F5C3B291C2C31517D092D0D0D0C4
:10D21000E032C23E0556E53325C2F5C2E435C3F51A
:10D22000C3C291C2C330401490EE00E00582F515F0
:10D23000E00582F517D092D0D0D0E03290EF00E038
:10D240000582F515E00582F517D092D0D0D0E032F6
:10D25000E709F608DFFA8046E709F208DFFA803EC0
:10D2600088828C83E709F0A3DFFA8076E309F60869
:10D27000DFFA806EE309F208DFFA806688828C8329
:10D28000E309F0A3DFFA805A89828A83E0A3F608D3
:10D29000DFFA804E89828A83E0A3F208DFFA8042B7
:10D2A00080AE80B480BA80C480CA80D080DA80E446
:10D2B00080378023805389828A83ECFAE493A3C861
:10D2C000C582C8CCC583CCF0A3C8C582C8CCC583F1
:10D2D000CCDFE9DEE7800D89828A83E493A3F60838
:10D2E000DFF9ECFAA9F0EDFB2289828A83ECFAE0FF
:10D2F000A3C8C582C8CCC583CCF0A3C8C582C8CC9E
:10D30000C583CCDFEADEE880DB89828A83E493A3ED
:10D31000F208DFF980CC88F0ED14B4040050C32487
:10D320001E83F582EB14B4050050B72415832582C3
:10D33000F582EF4E60ACEF60010EE58290D2A073F3
:10D34000000402000C060012BB020689828A83E0F8
:10D35000224003BB0402E722400789828A83E493C8
:10D3600022E322EFF88DF0A4FFEDC5F0CEA42EFE4F
:10D37000EC88F0A42EFE22BC000BBE0029EF8DF03D
:10D3800084FFADF022E4CCF875F008EF2FFFEE3308
:10D39000FEEC33FCEE9DEC984005FCEE9DFE0FD5B7
:10D3A000F0E9E4CEFD22EDF8F5F0EE8420D21CFE8B
:10D3B000ADF075F008EF2FFFED33FD4007985006F4
:10D3C000D5F0F222C398FD0FD5F0EA22C2D5EC3099
:10D3D000E709B2D5E4C39DFDE49CFCEE30E715B24D
:10D3E000D5E4C39FFFE49EFE12D377C3E49DFDE422
:10D3F0009CFC800312D37730D507C3E49FFFE49EE3
:10D40000FE22A42582F582E5F03583F58322EF4ED6
:10D410006013EDBB021089828A83EF60010EEDF08C
:10D42000A3DFFCDEFA2289F04003BB0407F709DF23
:10D43000FCA9F02250EFF309DFFCA9F022E709F67E
:10D4400008DFFA8079E9D39850F3E92FF9E82FF84B
:10D4500019E718F6DFFA8066E709F208DFFA805E5E
:10D4600088828C83E709F0A3DFFA8052E309F6088B
:10D47000DFFA804AE9D398500EE92FF9E82FF8191E
:10D48000E318F2DFFA8037E309F208DFFA802F8829
:10D49000828C83E309F0A3DFFA802389828A83E008
:10D4A000A3F608DFFA801789828A83E493A3F2083F
:10D4B000DFF9800A89828A83E0A3F208DFFA02D5C5
:10D4C0004380828093809980A380A980C280CC8091
:10D4D000E38077806380D0D3E998EA9C5039E92FC4
:10D4E000F582EA3BF583E82FF8EC3BFC0582D58218
:10D4F0000215831582E493C8C582C8CCC583CC05C8
:10D5000082D5820215831582F0C8C582C8CCC58336
:10D51000CCDFD9DED7802E89828A83ECFAE493A30C
:10D52000C8C582C8CCC583CCF0A3C8C582C8CCC549
:10D5300083CCDFE9DEE7800D89828A83E493A3F65A
:10D5400008DFF9ECFAA9F0EDFB22D3E998EA9C5048
:10D5500038E92FF582EA3BF583E82FF8EC3BFC0530
:10D5600082D5820215831582E0C8C582C8CCC583E6
:10D57000CC0582D5820215831582F0C8C582C8CC3D
:10D58000C583CCDFDADED880BC89828A83ECFAE0FE
:10D59000A3C8C582C8CCC583CCF0A3C8C582C8CCFB
:10D5A000C583CCDFEADEE8809C88F0ED14B404008B
:10D5B0005091242283F582EB14B405005085241980
:10D5C000832582F582EEFB4F700302D543EF6001A5
:10D5D0000EE58290D4C173000402000C060012FF15
:00000001FF
